:100000000C94C3030C94E4030C94E4030C94E403F5
:100010000C94E4030C94E4030C94E4030C94E403C4
:100020000C94E4030C94E4030C94E4030C94E403B4
:100030000C94E4030C94E4030C94E4030C94E403A4
:100040000C94E4030C94E4030C94E4030C94E40394
:100050000C9499070C94E4030C94E4030C94E403CB
:100060000C94200F0C94E4030C94E4030C94E4032C
:100070000C940A080C94E4030C94E4030C94DE0E34
:100080000C94E4030C94E4030C94E403AB15AE1558
:10009000DD161016DD16DD16DD16D616DD16DD169C
:1000A00098169D16A216AD16C216054F0F4F174F84
:1000B000194F1B4F1D4F1F4F214F244F6E616E0074
:1000C000696E660000407A10F35A00A0724E18095B
:1000D0000010A5D4E80000E87648170000E40B54AF
:1000E000020000CA9A3B000000E1F505000080967E
:1000F0009800000040420F000000A08601000000B0
:10010000102700000000E803000000006400000069
:1001100000000A00000000000100000000002C7632
:10012000D888DC674F0823DFC1DFAE59E1B1B7964D
:10013000E5E3E453C63AE651997696E8E6C28426AA
:10014000EB898C9B62ED407C6FFCEFBC9C9F40F286
:10015000BAA56FA5F490055A2AF75C936B6CF96702
:100160006DC11BFCE0E40D47FEF520E6B500D0EDC7
:10017000902E0300943577050080841E080000202F
:100180004E0A000000C80C333333330F986E1283CD
:100190001141EF8D2114893BE65516CFFEE6DB18A1
:1001A000D1844B381BF77C1D901DA4BBE424203266
:1001B00084725E228100C9F124ECA1E53D274E4105
:1001C0004E494E495459494E46CDCCCC3D0AD723D1
:1001D0003C17B7D13877CC2B329595E6241FB14F19
:1001E0000A000020410000C84200401C4620BCBE5E
:1001F0004CCA1B0E5AAEC59D744572726F722C208C
:10020000696E64657465726D696E61746520626F94
:100210006F7420766563746F722025640D0A004147
:10022000540024504D544B3331342C302C312C306D
:100230002C312C302C302C302C302C302C302C30DD
:100240002C302C302C302C302C302C302C302C30CE
:100250002A32380D0A0024504D544B3330302C31A3
:100260003030302C302C302C302C302A31430D0AD9
:100270000024504D544B3235312C35373630302A2E
:1002800032430D0A0052096AD53036A538BF40A363
:100290009E81F3D7FB7CE339829B2FFF87348E430B
:1002A00044C4DEE9CB547B9432A6C2233DEE4C9588
:1002B0000B42FAC34E082EA16628D924B2765BA25F
:1002C000496D8BD12572F8F66486689816D4A45CC3
:1002D000CC5D65B6926C704850FDEDB9DA5E15469E
:1002E00057A78D9D8490D8AB008CBCD30AF7E458F7
:1002F00005B8B34506D02C1E8FCA3F0F02C1AFBD53
:100300000301138A6B3A9111414F67DCEA97F2CFF0
:10031000CEF0B4E67396AC7422E7AD3585E2F937DA
:10032000E81C75DF6E47F11A711D29C5896FB76228
:100330000EAA18BE1BFC563E4BC6D279209ADBC0D3
:10034000FE78CD5AF41FDDA8338807C731B11210EB
:10035000592780EC5F60517FA919B54A0D2DE57AC8
:100360009F93C99CEFA0E03B4DAE2AF5B0C8EBBB14
:100370003C83539961172B047EBA77D626E1691422
:100380006355210C7D637C777BF26B6FC530016711
:100390002BFED7AB76CA82C97DFA5947F0ADD4A2FD
:1003A000AF9CA472C0B7FD9326363FF7CC34A5E5C9
:1003B000F171D8311504C723C31896059A07128026
:1003C000E2EB27B27509832C1A1B6E5AA0523BD65A
:1003D000B329E32F8453D100ED20FCB15B6ACBBE7F
:1003E000394A4C58CFD0EFAAFB434D338545F9022B
:1003F0007F503C9FA851A3408F929D38F5BCB6DA40
:100400002110FFF3D2CD0C13EC5F974417C4A77EE5
:100410003D645D197360814FDC222A908846EEB8F6
:1004200014DE5E0BDBE0323A0A4906245CC2D3AC30
:10043000629195E479E7C8376D8DD54EA96C56F475
:10044000EA657AAE08BA78252E1CA6B4C6E8DD7433
:100450001F4BBD8B8A703EB5664803F60E6135575B
:10046000B986C11D9EE1F8981169D98E949B1E87AB
:10047000E9CE5528DF8CA1890DBFE6426841992D50
:100480000FB054BB1678A46AD756B7C7E8DB702004
:1004900024EECEBDC1AF0F7CF52AC6874713463088
:1004A000A8019546FDD8988069AFF7448BB15BFFF2
:1004B000FFBED75C892211906B937198FD8E4379B2
:1004C000A62108B44962251EF640B340C0515A5EC9
:1004D00026AAC7B6E95D102FD65314440281E6A1BF
:1004E000D8C8FBD3E7E6CDE121D60737C3870DD5C2
:1004F000F4ED145A4505E9E3A9F8A3EFFCD9026F1E
:10050000678A4C2A8D4239FAFF81F6718722619DF4
:100510006D0C38E5FD44EABEA4A9CFDE4B604BBBB1
:10052000F670BCBFBEC67E9B28FA27A1EA8530EFD5
:10053000D4051D880439D0D4D9E599DBE6F87CA22E
:100540001F6556ACC4442229F497FF2A43A723947D
:10055000AB39A093FCC3595B6592CC0C8F7DF4EF53
:10056000FFD15D84854F7EA86FE0E62CFE14430129
:10057000A3A111084E827E53F735F23ABDBBD2D704
:100580002A91D386EB0000891112239B322446ADB9
:10059000573665BF74488CC19D5AAFD3BE6CCAE54F
:1005A000DB7EE9F7F88110080193331A22A5562C57
:1005B00047B7753E64C99C408DDBBF52AEEDDA642F
:1005C000CBFFF976E802218B30100299132667AF32
:1005D000763444BD554AADC3BC588ED19F6EEBE70F
:1005E000FA7CC8F5D983310A2091121803A7772E17
:1005F00066B5543C45CBBD42ACD99E508FEFFB66EF
:10060000EAFDD874C904428D5316619F702004A975
:10061000153227BB364CCEC5DF5EEDD7FC6888E1CE
:10062000997AABF3BA85520C4397711E60A11428D6
:1006300005B3373A26CDDE44CFDFFD56ECE99860AE
:1006400089FBBB72AA06638F7214409D512225ABB1
:10065000343006B9174EEFC7FE5CCCD5DD6AA9E38E
:10066000B8788AF19B87730E6295501C41A3352A96
:1006700024B1163807CFFF46EEDDDC54CDEBB9626E
:10068000A8F99A708B088481951AA793B62CC2A5F5
:10069000D33EE1B7F04008C919522BDB3A644EED66
:1006A0005F766DFF7C899400859BB712A6ADD2243E
:1006B000C3BFF136E0C1184809D33B5A2AE55E6C46
:1006C0004FF77D7E6C0AA583B4188691972EE3A719
:1006D000F23CC0B5D14229CB38500AD91B666FEF26
:1006E0007E744CFD5D8BB502A499961087AFF326FE
:1006F000E2BDD034C1C3394A28D11A580BE77F6E06
:100700006EF55C7C4D0CC685D71EE597F42880A15C
:10071000913AA3B3B2444ACD5B5669DF78600CE9E5
:100720001D722FFB3E8DD604C79FF516E4A99020BD
:1007300081BBB332A2C55A4C4BD7795E68E11C68C5
:100740000DF33F7A2E0EE787F61CC495D52AA1A398
:10075000B03882B193466BCF7A5448DD59622DEBA5
:100760003C700EF91F8FF706E69DD414C5ABB1227D
:10077000A0B9923083C77B4E6AD5585C49E33D6A85
:100780002CF11E780F002092D63A11241FBECFEF15
:10079000D0E4DEBFCDBF17E0A0E0B1E0E6E3F3EFC9
:1007A00000E00BBF02C007900D92A036B107D9F749
:1007B0001AE3A0E6B7E001C01D92A63DB107E1F73C
:1007C0000E948E6D0C9499790C9400000C944A64EC
:1007D0008091D63A80FF02C082E007C082FF02C04B
:1007E00083E003C083FF08C081E0809360078091AD
:1007F00024188823F9F018C01F928F9389EF91E095
:100800009F938F930E94AC7687EE95E00E94C0760E
:100810000F900F900F900F9080917307811101C07E
:10082000299A0E942510F8CF0E946254811102C0BB
:100830000E94D51080917307811101C02A9A0895F2
:10084000789484E797E10E949C09E8ECFAE384E756
:1008500097E193838283918380830E94DF060E94C5
:10086000990F0E94001082E09CE00E946C0B26EE23
:1008700033E042E05CE0BA018BE298E10E94B960AB
:1008800044E757E162E07CE08BE298E10E942B6252
:100890000E94B9110E94714F84E797E10E945D5058
:1008A0000E94F0100C94E80310923F170895809175
:1008B0003917813019F480E00E9479088091391746
:1008C000823019F480E00E949508809139178330B6
:1008D00019F480E00E94B10880913917843019F42E
:1008E00080E00E94CC0880913917853019F480E0AF
:1008F0000E94E60880913917863019F480E00E9442
:10090000000980913917873019F480E00E941A0994
:1009100080913917883019F480E00E943409809161
:100920003917893019F480E00E944E0980913917F7
:100930008A3019F480E00E946809809139178B3061
:1009400019F480E00E948209809139178C3019F4E3
:1009500080E00C94330A08958FEF8093A21A44E14B
:1009600050E060E070E04093561750935717609343
:1009700058177093591746EE50E060E070E04093CE
:10098000261850932718609328187093291849E166
:1009900050E060E070E0409317185093181860938F
:1009A000191870931A1890EC90934017809366175B
:1009B00080E8809325181092161810922E17109226
:1009C000241881E08093731780939D1A9BE0909385
:1009D000391780933817089580E008950895089591
:1009E0009FEF980F9C3010F48093391708950C9462
:1009F000B10F0C94AB0F811103C01092161808951B
:100A000081E0809316180895811103C010922E176B
:100A1000089581E080932E170895811103C01092EC
:100A200073170895813011F0823011F48093731799
:100A30000895811103C010923F170895813011F07D
:100A4000823011F480933F170895811103C01092F2
:100A50009D1A0895813011F0823011F480939D1A0F
:100A60000895F894F999FECF92BD81BD60BDFA9AC0
:100A70007894F99A0895F894F999FECF92BD81BDC2
:100A8000F89A789480B50895AF92BF92CF92DF9292
:100A9000EF92FF920F931F93CF93DF93CDB7DEB703
:100AA000E0970FB6F894DEBF0FBECDBFCE01019622
:100AB0007C0100E010E05C01C8010E943B05D70109
:100AC0008D937D010F5F1F4F00311105A9F77E0146
:100AD000B1E2EB0EF11C670100E110E0C8010E94D9
:100AE0003B05F60181936F010F5F1F4F0032110527
:100AF000A9F720E830E040E050E0B501CE01419692
:100B00000E940060FE01719680E18E0F2191D70155
:100B10009D917D01291304C08E13F8CF81E001C09F
:100B200080E0E0960FB6F894DEBF0FBECDBFDF9138
:100B3000CF911F910F91FF90EF90DF90CF90BF90DA
:100B4000AF900895EF92FF920F931F93CF93DF938F
:100B5000CDB7DEB760970FB6F894DEBF0FBECDBF3E
:100B6000CE0101967C0100E010E0C8010E943B0527
:100B7000F70181937F010F5F1F4F00311105A9F726
:100B80008C818093A21A2D8130E0AAE0B0E00E940F
:100B90004B73609356177093571780935817909321
:100BA00059172E8130E00E944B7360932618709382
:100BB000271880932818909329182F8130E00E94DD
:100BC0004B736093171870931818809319189093AB
:100BD0001A188885809340178985809366178A85BF
:100BE0008093251881E09B85911101C080E080935E
:100BF000161881E09C85911101C080E080932E172A
:100C000081E09D85911101C080E0809324188E853C
:100C1000809373178F8580939D1A888980933917E5
:100C200060960FB6F894DEBF0FBECDBFDF91CF91B7
:100C30001F910F91FF90EF9008950F931F93CF9303
:100C4000DF931F92CDB7DEB78C0169830E943B050D
:100C50006981861741F0C8010F90DF91CF911F91F4
:100C60000F910C9431050F90DF91CF911F910F914F
:100C70000895CF93DF93C0E0D0E060E0CE010E9402
:100C80001D062196C032D105C1F7DF91CF9108959D
:100C9000CF92DF92EF92FF920F931F93CF93DF9348
:100CA000CDB7DEB7E0970FB6F894DEBF0FBECDBF6D
:100CB0008E010F5F1F4F80E2F80111928A95E9F7CC
:100CC00081E089838A838B838091A21A8C836091CF
:100CD00056177091571780915817909159172AE01D
:100CE000C22ED12CE12CF12CA70196010E94857314
:100CF0002D83609126187091271880912818909163
:100D00002918A70196010E9485732E8360911718F8
:100D1000709118188091191890911A18A7019601CE
:100D20000E9485732F838091401788878091661772
:100D30008987809125188A87809116188B878091E2
:100D40002E178C87809124188D87809173178E873A
:100D500080919D1A8F8780913917888B20E830E029
:100D600040E050E0B801CE0181960E940060DE01B3
:100D70005196FE01B19680E18E0F91919D938E1355
:100D8000FCCFE12CF12CF80161918F01C7010E9489
:100D90001D06FFEFEF1AFF0A80E2E816F10499F74B
:100DA000E0960FB6F894DEBF0FBECDBFDF91CF91B6
:100DB0001F910F91FF90EF90DF90CF9008951092C8
:100DC00038171092A11A0E944405882319F00E9436
:100DD000A20504C00E94AC040E94480610923F176E
:100DE0000C9457040C94480681E0809324180C94CA
:100DF00048060E94480698E088E10FB6F894A89546
:100E0000809360000FBE90936000FFCF1092241873
:100E10000E94F90681E08093A11A08951092A11A08
:100E20000895CF92DF92EF92FF920F931F93CF938B
:100E3000DF93CDB7DEB7A0970FB6F894DEBF0FBE35
:100E4000CDBFCE0101967C0100E010E06C01C8012D
:100E50000E943B05F70181937F010F5F1F4F003216
:100E60001105A9F760E270E0C6010E94DE6AA09653
:100E70000FB6F894DEBF0FBECDBFDF91CF911F91AB
:100E80000F91FF90EF90DF90CF9008959091C80060
:100E900095FFFCCF8093CE0081E090E00895809193
:100EA000C80087FFFCCF8091CE0090E00895CF93DB
:100EB000DF931F92CDB7DEB789830E942510898109
:100EC0009091C00095FFFCCF8093C60081E090E038
:100ED0000F90DF91CF9108958091C00087FFFCCFE4
:100EE0000E9425108091C60090E00895811103C0F2
:100EF0008091C00004C0813031F48091C800881F07
:100F00008827881F089580E008958091C00087FF9A
:100F100005C00E9425108091C60008958FEF0895A6
:100F20008091C80087FF03C08091CE0008958FEFA5
:100F300008951F920F920FB60F9211240BB60F92C5
:100F40002F933F934F935F936F937F938F939F93D1
:100F5000AF93BF93EF93FF938091C00087FF47C08B
:100F60000E94251020912A1730912B178091261767
:100F7000909127172817390759F420912C17309191
:100F80002D1780912817909129172817390769F193
:100F900020912C1730912D1780912A1790912B17A3
:100FA00001972817390709F10E948507E0912C174E
:100FB000F0912D17808320912C1730912D1780915F
:100FC0002817909129172817390729F48091261797
:100FD0009091271705C080912C1790912D1701969D
:100FE00090932D1780932C1702C00E949007FF91B9
:100FF000EF91BF91AF919F918F917F916F915F9191
:101000004F913F912F910F900BBE0F900FBE0F90FD
:101010001F9018951F920F920FB60F9211240BB6C6
:101020000F922F933F934F935F936F937F938F9381
:101030009F93AF93BF93EF93FF938091C80087FF77
:1010400045C0209121113091221180911D11909164
:101050001E112817390759F42091231130912411BA
:1010600080911F11909120112817390769F1209163
:101070002311309124118091211190912211019717
:101080002817390709F10E949007E0912311F09188
:1010900024118083209123113091241180911F11FC
:1010A000909120112817390729F480911D119091F2
:1010B0001E1105C0809123119091241101969093E7
:1010C00024118093231102C00E949007FF91EF9199
:1010D000BF91AF919F918F917F916F915F914F9150
:1010E0003F912F910F900BBE0F900FBE0F901F904E
:1010F000189581110CC084E08093C50081E1809334
:10110000C4008091C0008D7F8093C000089581301D
:1011100059F484E08093CD0081E18093CC008091EC
:10112000C8008D7F8093C800089581110CC082E0B3
:101130008093C50088E08093C4008091C0008D7FBB
:101140008093C0000895813059F482E08093CD00EF
:1011500088E08093CC008091C8008D7F8093C80088
:10116000089581110CC081E08093C50083E08093D5
:10117000C4008091C0008D7F8093C00008958130AD
:1011800051F48093CD0083E08093CC008091C8001F
:101190008D7F8093C800089581110BC01092C50007
:1011A00081E88093C4008091C0008D7F8093C0004F
:1011B0000895813051F41092CD0081E88093CC00E5
:1011C0008091C8008D7F8093C800089581110BC065
:1011D0001092C50086E58093C4008091C0008D7F89
:1011E0008093C0000895813051F41092CD0086E5BF
:1011F0008093CC008091C8008D7F8093C8000895B3
:1012000081110BC01092C50080E48093C4008091CE
:10121000C0008D7F8093C0000895813051F41092FA
:10122000CD0080E48093CC008091C8008D7F8093B6
:10123000C800089581110BC01092C5008AE2809306
:10124000C4008091C0008D7F8093C00008958130DC
:1012500051F41092CD008AE28093CC008091C800B6
:101260008D7F8093C800089581110BC01092C50036
:1012700080E28093C4008091C0008D7F8093C00085
:101280000895813051F41092CD0080E28093CC001B
:101290008091C8008D7F8093C800089581110BC094
:1012A0001092C50085E18093C4008091C0008D7FBD
:1012B0008093C0000895813051F41092CD0085E1F3
:1012C0008093CC008091C8008D7F8093C8000895E2
:1012D00081110BC01092C5008FE08093C4008091F3
:1012E000C0008D7F8093C0000895813051F410922A
:1012F000CD008FE08093CC008091C8008D7F8093DB
:10130000C800089581110BC01092C5008AE0809337
:10131000C4008091C0008D7F8093C000089581300B
:1013200051F41092CD008AE08093CC008091C800E7
:101330008D7F8093C8000895CF92DF92EF92FF9245
:101340000F931F93CF93DF93CDB7DEB76C970FB694
:10135000F894DEBF0FBECDBF6C018CE1D6011D92AB
:101360008A95E9F785E2E82E81E1F82E80E096E0A3
:10137000F7019C01119221503040E1F700E917E19B
:1013800080E8D8011D928A95E9F780E00E948209E1
:101390001092CD008AE08093CC00E8ECF0E08081F0
:1013A0008D7F808396E09093C20088E98093C1008E
:1013B0009093CA008093C9008EE0FE013F96DF0142
:1013C000282F1D922A95E9F79E012F5F3F4FD901E3
:1013D0001D928A95E9F783E08A8B47E557E0588F9D
:1013E0004F8B4CE657E05A8F498F9EE0D601019013
:1013F0000D929A95E1F78C8386E497E09A87898726
:101400008FE497E09C878B878EE0F901D6011E96CA
:1014100001900D928A95E1F7E6E2F7E1F182E08230
:10142000F782E682F582E48284E297E19383828305
:10143000EDE1F1E1118300831783068315830483B3
:101440008FE098E1938382836C960FB6F894DEBFA9
:101450000FBECDBFDF91CF911F910F91FF90EF9005
:10146000DF90CF90089581110BC01092C5008AE0E3
:101470008093C4008091C00082608093C000089572
:10148000813051F41092CD008AE08093CC0080919D
:10149000C80082608093C80008950F931F93CF9374
:1014A000DF93182FC091B41AD091B51A8BA1811176
:1014B0002FC08AE390E098A38F8F1E8E1D8E1C8E06
:1014C00081E08BA38CA380917307811101C02898C0
:1014D00080917307811101C0299A209126183091BB
:1014E00027184091281850912918A0E6B9E00E94C9
:1014F0005A736056704F8F4F9F4F20E43FE140E09A
:1015000050E00E9485733D8B2C8B81E080936607B1
:101510000FB7F894209117183091181840911918A6
:1015200050911A18A0E6B9E00E945A736056704FA5
:101530008F4F9F4F20E43FE140E050E00E948573D1
:101540003F8B2E8B0FBFE091B41AF091B51A4FB7B5
:10155000F894E056FD4F24813581808191812817D0
:10156000390739F426813781828193812817390719
:1015700079F066817781248135812150310991E0AC
:1015800080E06217730709F090E0292F382F02C01E
:1015900021E030E04FBF232BB1F6E091B41AF09177
:1015A000B51A2FB7F894E056FD4FA681B7811C936A
:1015B00046815781828193814817590719F48081A8
:1015C000918103C0868197810196978386832FBF7F
:1015D00081E090E0DF91CF911F910F910895E0910C
:1015E000B41AF091B51A4FB7F89421AD32AD83AD6E
:1015F00094AD4FBF28173907D9F0E091B41AF09194
:10160000B51A9FB7F894A1ADB2AD27A930ADA21716
:10161000B30719F425A936A905C0A1ADB2AD9D0146
:101620002F5F3F4F32AF21AF8C919FBF90E0089565
:101630008FEF9FEF089587B18FEF87B910929000D9
:1016400089E18093910080E194E0909397008093EA
:10165000960080E280937100559A549A08951092F2
:1016600034171092351710923617109237171092C0
:101670006F171092701710927117109272171092C4
:101680004617109245171092800089E180938100DF
:1016900080E194E0909387008093860080E28093BD
:1016A0007C00089882B112B8EEE7F0E0808181609A
:1016B000808387E080937B008DEE80937A0008958D
:1016C0001092341710923517109236171092371760
:1016D0000E942F0B0C941B0B0F931F93CF93DF9340
:1016E000CDB7DEB72E970FB6F894DEBF0FBECDBFD5
:1016F0008C018AE195E0D801FC011D923197E9F750
:101700001093B51A0093B41A8AE390E0D80190962A
:101710009C938E935F9792961C921E929197C8010C
:101720008D9696969C938E9395979C969C938E936C
:101730009B979A969C938E939997079698969C93CD
:101740008E9397970996D6969C938E93D597DC9611
:101750009C938E93DB97DA969C938E93D9978E59B0
:101760009D4FD8969C938E93D7970996F801E05693
:10177000FD4F9183808397838683958384838E59DD
:101780009D4F9383828385E090E0019711F1D8010A
:101790009B96ED91FC919C9710829B964D915C914C
:1017A0009C9797962D913C9198974217530749F42F
:1017B00095962D913C9196979C963C932E939B9752
:1017C000E4CFF80123A534A52F5F3F4F34A723A70B
:1017D000DCCF0E94600B8EE0FE013196DF01282FE6
:1017E0001D922A95E9F793E09C832DE43AE03A872D
:1017F00029872FEE3AE03C872B87D80101900D9284
:101800008A95E1F72E960FB6F894DEBF0FBECDBFD6
:10181000DF91CF911F910F910895CF93DF93FC013A
:10182000808D8111BEC0828D811190C0DF01A056D4
:10183000BD4F14964D915C91159716962D913C9144
:1018400017974217530749F426893789232B29F420
:101850001092660713A214A251C0938D911101C07A
:10186000148E91E0938F248935892115310579F5FE
:1018700014964D915C91159716962D913C91179762
:101880004217530741F414A22689378921503109A0
:10189000378B268B20C01496CD91DC91159712962C
:1018A0002D913C911397C217D30721F42D913C91B0
:1018B000119707C01496CD91DC9115979E012F5F6B
:1018C0003F4F15963C932E931497988105C0215055
:1018D0003109358B248B9EE7918F918D9B3181F55A
:1018E00014964D915C91159716962D913C911797F2
:1018F0004217530749F41092660713A29091730799
:1019000091116FC029986DC01496CD91DC911597F7
:1019100012968D919C911397C817D90721F48D9138
:101920009C91119706C01496CD91DC911597CE012C
:10193000019615969C938E9314978881818F04C08D
:101940009E57923008F4138E81E0828F838D278D0D
:1019500030A1882379F0848D853060F0148E2A338D
:10196000310519F08AE390E002C08AE690E090A386
:10197000878F15C0828D918D982321F0948D9F5F64
:10198000948F0BC0148E2A33310519F02AE330E00E
:1019900002C02AE630E030A3278F880F828F88E0CC
:1019A000808F278D30A1858D968D820F931FAC017E
:1019B0005170568F458F208D2150208F9927803868
:1019C000910530F02FEF30E0B901681B790BCB01A6
:1019D000FC01E85FFE4F80814F3F510511F008F098
:1019E0008095DF91CF910895CF93DF93FC01809193
:1019F000A11A8823E9F020916207309163072F5FD5
:101A00003F4F3093630720936207809164078617E6
:101A10001CF4609364070CC02036310548F0109226
:101A200063071092620718161CF4815080936407B4
:101A3000DF01A35FBA4F2D913C911197EF01C55F74
:101A4000DA4F39832883C1A5D2A587A190A5C817ED
:101A5000D90719F485A196A104C0C1A5D2A5CE01CC
:101A6000019692A781A798819602C001112497FD43
:101A7000039695958795959587958D939C93DF0112
:101A8000AF5EBA4F5C9111964C911197EF01C15F17
:101A9000DA4F58834983820F931F252F342F37FF46
:101AA00002C02F5F3F4F35952795820F931F8D936F
:101AB0009C93DF01AD5EBA4F21E030E018161906A5
:101AC00014F420E030E08D919C911197880F991FBC
:101AD000822B932B11969C938E93C3A5D4A56883D8
:101AE00023A534A587A190A52817390719F485A146
:101AF00096A103C083A594A5019694A783A78D9171
:101B00009C9111979C0136952795369527958227AC
:101B1000932783709927EF01CB5EDA4F039769F41F
:101B2000888199818032910510F4019601C0019756
:101B30009983888312A211A205C081A192A1019666
:101B400092A381A38881998108968034910518F425
:101B50009983888323C18F73992799838883EF01A1
:101B6000C95EDA4F8881880F88839C9197702BEF2C
:101B7000290F233010F0933011F48160888388811D
:101B8000982F96958927809581709685990F892B36
:101B900086878E37C9F521AD32AD85A996A928175C
:101BA000390739F423AD34AD87A990AD281739072B
:101BB00039F123AD34AD81AD92AD019728173907C6
:101BC000F9F0A3ADB4AD8EE78C9323AD34AD87A906
:101BD00090AD2817390719F485A996A903C083ADDC
:101BE00094AD019694AF83AF91E0918B83898C3053
:101BF00020F4128A8F5F838B01C0928B81E09FC09B
:101C0000118A128A138A9AC08F778F3711F4118A3A
:101C10000FC0928980917307992321F0811105C02B
:101C2000289A03C0811101C028988189811103C0BD
:101C3000128A138AB3C08685982F9F739E3309F446
:101C4000ADC080FF03C080898068808B97859F5FCF
:101C500097878089983008F477C092E8980F92307F
:101C600010F08B3199F521AD32AD85A996A92817D1
:101C7000390739F423AD34AD87A990AD281739075A
:101C8000E1F023AD34AD81AD92AD0197281739074E
:101C9000A1F0A3ADB4AD8BE18C9323AD34AD87A996
:101CA00090AD2817390719F485A996A903C083AD0B
:101CB00094AD019694AF83AF09C0118A128A138A3A
:101CC00080917307811104C0289803C081E001C08E
:101CD00080E041AD52AD25A936A94217530739F42A
:101CE00043AD54AD27A930AD42175307F1F043ADD2
:101CF00054AD21AD32AD2150310942175307A9F03F
:101D00009089A3ADB4AD9C9343AD54AD27A930AD3C
:101D10004217530719F425A936A904C023AD34ADE1
:101D20002F5F3F4F34AF23AF0AC0118A128A138A44
:101D300080917307811102C0289801C080E0108A49
:101D40001786882321F02AC08695808B27C0DF0163
:101D5000A85EBA4F8D919C911197816011969C93CA
:101D60008E9321AD32AD85A996A92817390739F48C
:101D700023AD34AD87A990AD2817390741F023ADC5
:101D800034AD81AD92AD01972817390739F483AD91
:101D900094AD92AF81AF11961C921E9281A192A137
:101DA000813C910540F012A211A2128A8091730722
:101DB000811101C02898DF91CF9108951F920F9251
:101DC0000FB60F9211240BB60F922F933F934F93A0
:101DD0005F936F937F938F939F93AF93BF93EF9393
:101DE000FF9380916607882379F08091B41A9091CF
:101DF000B51A0E940D0C88B980917307811101C03A
:101E0000299A5D9A5C9809C080917307811101C07D
:101E100029988FE788B95D985C9AFF91EF91BF91FF
:101E2000AF919F918F917F916F915F914F913F9172
:101E30002F910F900BBE0F900FBE0F901F90189513
:101E40001F920F920FB60F9211240BB60F922F9381
:101E50003F934F935F936F937F938F939F93AF9332
:101E6000BF93EF93FF9380E286BB80916607811159
:101E700015C06091790060588091B41A9091B51A9C
:101E80000E94F40C809161078F5F803C18F480936E
:101E9000610704C0109261070E9456120E945510FB
:101EA0008091341790913517A0913617B09137175C
:101EB0000196A11DB11D8093341790933517A093FF
:101EC0003617B093371780914517909146170196B2
:101ED000909346178093451781159B44B8F08091E5
:101EE0006F1790917017A0917117B09172170196AA
:101EF000A11DB11D80936F1790937017A093711758
:101F0000B09372171092461710924517FF91EF91F8
:101F1000BF91AF919F918F917F916F915F914F9101
:101F20003F912F910F900BBE0F900FBE0F901F90FF
:101F300018958AB1806C8AB983EA8093B00081E0F9
:101F40008093B100809125188093B300809166172B
:101F50008093B40008958093251880958093B300F2
:101F60000895809366178093B40008952FB7F8946E
:101F7000609134177091351780913617909137170B
:101F80002FBF08958F929F92AF92BF92CF92DF9210
:101F9000EF92FF92CF93DF9300D000D0CDB7DEB7A2
:101FA0009B01AC0169833A834B835C830E94B60F2B
:101FB0006B017C01A3E1B0E029813A814B815C8116
:101FC0000E945A734B015C010E94B60FDC01CB01E9
:101FD0008C199D09AE09BF0988159905AA05BB058D
:101FE00098F30F900F900F900F90DF91CF91FF908B
:101FF000EF90DF90CF90BF90AF909F908F9008951B
:1020000088EF92E0A0E0B0E080936F0790937007B4
:10201000A0937107B093720784B18F6184B985B1C1
:10202000807E85B983EC84BD81E085BD80914017B9
:1020300087BD089581E08093730708951092730718
:1020400008958093401787BD08958091730781118B
:1020500011C02C9A0E94B60FDC01CB0188509D4F15
:10206000AF4FBF4F8093670790936807A0936907AE
:10207000B0936A07089580917307811101C02C986D
:1020800008952C9A0E94B60FDC01CB0188509D4F19
:10209000AF4FBF4F8093670790936807A09369077E
:1020A000B0936A0708952C9808950F931F93809119
:1020B0006B0790916C07A0916D07B0916E074091EE
:1020C0006F075091700760917107709172078417C4
:1020D0009507A607B707D4F00E94B60F00916707CF
:1020E000109168072091690730916A070617170752
:1020F0002807390714F40E943B1010926B071092C6
:102100006C0710926D0710926E070BC00196A11D0F
:10211000B11D80936B0790936C07A0936D07B093EC
:102120006E071F910F910895CF9381E080937307FD
:102130002A980E9453102998289868EC70E080E053
:1021400090E00E94C20FC2E02A9A62E370E080E051
:1021500090E00E94C20F2A980E94411062E370E052
:1021600080E090E00E94C20F0E945310289A62E320
:1021700070E080E090E00E94C20F2898299A62E304
:1021800070E080E090E00E94C20F299862E370E066
:1021900080E090E00E94C20FC13011F0C1E0D4CFC6
:1021A0002A9A10927307CF9108950E94251080916A
:1021B0007307811101C02A9864EF71E080E090E01C
:1021C0000E94C20F0E943B1080917307811101C0D1
:1021D0002A9A64EF71E080E090E00E94C20FE5CFA0
:1021E00081B1866081B90E94D64F811103C081B14F
:1021F000886181B9089582B186958170089582B110
:1022000082FB882780F908950E94D64F811105C06E
:1022100082B183FB882780F9089580E008950E94A9
:10222000D64F811104C082B182958170089580E0FB
:102230000895119A0895129A08950E94D64F811117
:1022400001C0139A08950E94D64F811101C0149ABB
:10225000089511980895129808950E94D64F8111FB
:1022600001C0139A08950E94D64F811101C0149A9B
:1022700008950E94D64F811107C00E94FB10811162
:102280000C9429110C94191108950E94D64F8111B4
:1022900007C00E94FF1081110C942B110C941B118C
:1022A00008950E94041181110C942D110C941D119C
:1022B0000E940F1181110C9433110C9423118F92F1
:1022C0009F92AF92BF92CF92DF92EF92FF920F93C5
:1022D0001F939B01AC018FB7F894C0903417D09036
:1022E0003517E0903617F09037178FBFA3E1B0E0B5
:1022F0000E945A732FB7F894809034179090351736
:10230000A0903617B09037172FBF950184010C1994
:102310001D092E093F09061717072807390750F32B
:102320001F910F91FF90EF90DF90CF90BF90AF90F3
:102330009F908F900895CF93C2E080917307811191
:1023400001C02A986AEF70E080E090E00E945F117F
:1023500080917307811101C02A9A64E170E080E0E6
:1023600090E00E945F11C13011F0C1E0E6CFCF9143
:10237000089584B1806A84B9269881E58CBD0E9A4F
:102380000F98179A08950E949B110E94BD548111C5
:102390000C94D5100895CF938130D1F4C4E080918E
:1023A0007307811101C02A9861E470E080E090E039
:1023B0000E945F1180917307811101C02A9A6EE11A
:1023C00070E080E090E00E945F11C15041F705C0CD
:1023D000811103C0CF910C949B11CF91089581E09E
:1023E0000E94CB110C94205780910001869581703A
:1023F00091E08927089581E090910001911180E09A
:1024000008958091780708950E94F411882389F037
:1024100041E062EB76E086EB9AE10E940A35811199
:1024200004C081E08093780702C010927807809101
:102430007807089540E062EB76E080E090E00E944B
:102440000A35811104C01092780781E0089580E078
:1024500008950E94041281110C94EF1108950E94B6
:102460001A1281110C94C311089580917707882363
:1024700021F0109277070E94291280917607882315
:1024800021F0109276070E942F1280917507882301
:1024900021F0109275070E94EF1180917407882334
:1024A00021F0109274070C94C3110895CF9380917A
:1024B00079078F5F809379070E94F21680E00E946F
:1024C000C814809300018091790762E30E946573CC
:1024D000911116C010927907C0917807C11107C0F9
:1024E0000E94F411882319F081E0809377070E94FD
:1024F000F411811105C0CC2319F081E08093760797
:10250000CF9108950F931F93CF93DF93CDB7DEB78D
:1025100060970FB6F894DEBF0FBECDBF2FB7F8940B
:1025200080916F1790917017A0917117B0917217E9
:102530002FBF8D879E87AF87B88BBE016F5F7F4FA0
:10254000CE010D960E94296B4B81552747FD509572
:10255000652F752F8BE0440F551F661F771F8A95D7
:10256000D1F78C81992787FD9095A92FB92FDC0190
:1025700099278827482B592B6A2B7B2B8A819927EF
:1025800087FD9095A92FB92F35E0880F991FAA1FB5
:10259000BB1F3A95D1F7482B592B6A2B7B2B89818E
:1025A000992787FD9095A92FB92FB695A79597954F
:1025B0008795482B592B6A2B7B2B8F819885805DC3
:1025C0009740AA2797FDA095BA2FF9E1880F991F88
:1025D000AA1FBB1FFA95D1F7482B592B6A2B7B2BCF
:1025E0008E818F5F992787FD9095A92FB92F15E1CF
:1025F000880F991FAA1FBB1F1A95D1F78A019B014B
:10260000082B192B2A2B3B2BC901B80160960FB65A
:10261000F894DEBF0FBECDBFDF91CF911F910F9118
:1026200008958EBD0DB407FEFDCF8EB50895169AA0
:102630008FEF0C9411130F931F93CF93DF93EC0143
:102640008B0184E180937B078FEF0E9411138F3FF2
:1026500029F480917B078111F7CF1EC08E3FE1F4F2
:102660008FEF8EBD0DB407FEFDCF9EB598838EBD56
:102670000DB407FEFDCF22969EB5FE0131979083E3
:102680000250110971F78FEF0E9411138FEF0E9412
:10269000111381E090E002C080E090E0DF91CF91E3
:1026A0001F910F91089582E380937A078FEF0E9424
:1026B0001113282F8F3F21F080917A078111F6CFD7
:1026C00081E090E02F3F11F080E090E00895CF93FB
:1026D000DF9300D0CDB7DEB716988FEF0E941113AD
:1026E0000E945313009739F489839A830E94171329
:1026F00089819A8102C081E090E00F900F90DF9174
:10270000CF910895FF920F931F93CF93DF93C82F1C
:10271000D42F152F062FF72E87FF09C040E050E079
:10272000BA0187E30E9482138230A0F5CF77CC30C4
:1027300099F48C2F80640E9411138F2D0E94111325
:10274000802F0E941113812F0E9411138D2F0E9440
:102750001113CC2369F008C00E9417130E9467135D
:10276000892B39F78FEF16C0C83021F081E003C004
:1027700085E901C087E80E941113CC3019F48FEF6E
:102780000E941113CAE08FEF0E94111387FF02C04D
:10279000C150C9F7DF91CF911F910F91FF9008951C
:1027A0001F93CF93DF93EC01162F0E9453130097D2
:1027B00059F1812F0E9411131D3F21F1CE019E5F1F
:1027C00028812EBD0DB407FEFDCF2296FE01319764
:1027D00020812EBD0DB407FEFDCFC817D90781F7A4
:1027E0008FEF0E9411138FEF0E9411138FEF0E9441
:1027F00011138F7131E020E0853009F030E0832F34
:10280000922F02C081E090E0DF91CF911F91089557
:10281000DF92EF92FF920F931F93CF93DF9300D03D
:1028200000D0CDB7DEB78111A6C01CBC80910101DC
:1028300081FD9EC084B1806A84B9269881E58CBDF3
:1028400082E58CBD1AE08FEF0E9411131150D9F769
:1028500040E050E0BA0180E00E948213813009F02C
:1028600075C084E680937B074AEA51E060E070E03F
:1028700088E00E948213813009F040C08E010F5F12
:102880001F4F780184E0D82ED00E8FEF0E941113D5
:10289000F70181937F01DE12F8CF8B81813009F03F
:1028A00055C08C818A3A09F051C080917B07811113
:1028B00006C080917B07882309F448C00AC040E025
:1028C00050E060E070E489EA0E9482138111EDCF4C
:1028D000F0CF40E050E0BA018AE30E9482138111F8
:1028E00035C08FEF0E941113F80181938F01DE1222
:1028F000F8CF898186FD2CC014E02BC040E050E069
:10290000BA0189EA0E948213823018F011E001E0D6
:1029100002C012E009EA80917B07811105C0809115
:102920007B07882399F009C040E050E0BA01802F6E
:102930000E9482138111EFCFF2CF40E052E060E0BD
:1029400070E080E10E948213882319F010E001C03A
:102950001CE010937C070E941713112341F0809113
:1029600001018E7F8093010180E58CBD01C01CBCFC
:102970008091010101C081E00F900F900F900F90A6
:10298000DF91CF911F910F91FF90EF90DF9008950D
:10299000811103C080910101089581E00895EF92B3
:1029A000FF920F931F93CF937B01BA01A90181116D
:1029B00038C001151105A9F18091010180FD33C0D6
:1029C00080917C0783FD07C089E0440F551F661F77
:1029D000771F8A95D1F70230110510F4C1E101C0CB
:1029E000C2E18C2F0E948213811114C060E072E05A
:1029F000C7010E941B13892B29F08EEFF81A015092
:102A00001109A1F7C23131F440E050E0BA018CE085
:102A10000E9482130E94171381E0012B29F480E0A9
:102A200003C084E001C083E0CF911F910F91FF901C
:102A3000EF900895CF92DF92EF92FF920F931F9342
:102A4000CF93DF93EB0169017A01811156C0011523
:102A5000110509F452C08091010180FD50C08091A0
:102A6000010182FD4EC080917C0783FD07C099E083
:102A7000CC0CDD1CEE1CFF1C9A95D1F70130110522
:102A800099F4B701A60188E10E94821381112EC03A
:102A90006EEFCE010E94D01331E020E0892B09F0C7
:102AA00030E0032F122F22C0867031F0A80160E0C1
:102AB00070E087E90E948213B701A60189E10E94B4
:102AC0008213811113C06CEFCE010E94D013892BA9
:102AD00021F0DE5F01501109B1F76DEF80E090E069
:102AE0000E94D013892B11F401E010E00E9417130B
:102AF00081E0012B39F480E005C084E003C083E06D
:102B000001C082E0DF91CF911F910F91FF90EF9074
:102B1000DF90CF900895EF92FF920F931F93CF9382
:102B2000DF93CDB7DEB760970FB6F894DEBF0FBE68
:102B3000CDBF811147C18091010180FD45C17A015E
:102B4000862F90E08F30910508F037C1FC01EA5BD9
:102B5000FF4F0C9406740E94671324C140E050E0BC
:102B6000BA0189E00E948213882311F011E026C186
:102B700060E170E0CE0101960E941B13892BB1F336
:102B800099819295969596959370888549852A8521
:102B90009130E1F48F7390E0A0E0B0E0DC01992780
:102BA00088270196A11DB11D50E0542F4427BA017A
:102BB000620F711D860F971FA11DB11DFAE0880FCE
:102BC000991FAA1FBB1FFA95D1F7ABC04295469536
:102BD00046954370F4E08F9FC0011124840F911D2E
:102BE00001964F81437050E0542F4427550F550FE5
:102BF000840F951FA0E0B0E03E81432F4F703B85CE
:102C0000331F3327331F340F2370220F230F275016
:102C100004C0880F991FAA1FBB1F2A95D2F781C035
:102C200010917C0740E050E0BA0112FF2BC08DE804
:102C30000E94821381119ACF8FEF0E94111360E1DD
:102C400070E0CE0101960E941B13892B09F48ECFF0
:102C500010E38FEF0E9411131150D9F72B852295A5
:102C60002F7080E190E0A0E0B0E004C0880F991FD1
:102C7000AA1FBB1F2A95D2F7F70180839183A283F5
:102C8000B3839CC089E00E94821381116FCF60E101
:102C900070E0CE0101960E941B13892B09F466CFC8
:102CA0008B852C8511FF1FC0221F2227221F022F78
:102CB00010E00F5F1F4F8F73080F111D080F111DBC
:102CC0008E858295869586958370815002C0000F0F
:102CD000111F8A95E2F720E030E0F70100831183AD
:102CE0002283338323C0922F9370229526952770D9
:102CF00030E0F8E09F9F200D311D11242F5F3F4FE2
:102D00008C7790E095958795959587950196289F66
:102D1000A001299F500D389F500D1124CA01A0E039
:102D2000B0E0F70180839183A283B38310E046C0B3
:102D300080917C07FA018083F9CF40E050E0BA012E
:102D400089E004C040E050E0BA018AE00E948213AA
:102D500081110CCF60E170E022C040E050E0BA0188
:102D60008AE30E948213811101CF87010C5F1F4FFC
:102D70008FEF0E941113F70181937F01E017F10794
:102D8000B9F7D4CF40E050E0BA018DE80E94821339
:102D90008111ECCE8FEF0E94111360E470E0C70147
:102DA0000E941B1311E0892B49F0C0CF1CBC8091FD
:102DB0000101816080930101B9CF14E00E941713D3
:102DC000812F03C084E001C083E060960FB6F894C1
:102DD000DEBF0FBECDBFDF91CF911F910F91FF904E
:102DE000EF90089580917B07882319F0815080939C
:102DF0007B0780917A07882319F0815080937A07A6
:102E000090910101892F8B7F079B03C0892F897FB8
:102E100001C08360809301010895FC016381862FC6
:102E200090E0A0E0B0E0BA2FA92F982F8827228148
:102E3000822BBA2FA92F982F88272181822BBA2F76
:102E4000A92F982F88272081BC01CD01622B0895DE
:102E50000F93FC01278130E040E050E060E070E03B
:102E600080E090E008E00E940F74A6812A2B0E9467
:102E70000F74A5812A2B0E940F74A4812A2B0E9413
:102E80000F74A3812A2B0E940F74A2812A2B0E9407
:102E90000F74A1812A2B0E940F74E0812E2B0F91B9
:102EA0000895FC01408351836283738308950F93D7
:102EB0001F93CF93DF93FC01D22FC32FB42FA52FE5
:102EC000CB01008398014D2F5C2F6B2F7A2F08E0E8
:102ED0000E942A7421830E942A7422830E942A74E9
:102EE00023830E942A7424830E942A7425830E94CB
:102EF0002A7426830E942A742783DF91CF911F9121
:102F00000F910895480F591FFC016193CF01E417F9
:102F1000F507D1F70895DC01FB012D91819130E097
:102F2000B901681B7109CB014150510911F000979B
:102F3000A1F308950F931F93FC019A01AB01225056
:102F40003109410951098789908DA18DB28D029770
:102F5000A109B109281739074A075B0768F4A18559
:102F6000B2850E945A7303A514A525A536A5600F46
:102F7000711F821F931F03C060E070E0CB011F919F
:102F80000F910895FC019C01255F3F4F80E0982F31
:102F900090FB979597F98191890FE217F307B9F79D
:102FA0000895CF93DF93FC01418150E04F5F5F4F65
:102FB00065E0440F551F6A95E1F780E090E060E01E
:102FC00070E062307105A1F0DC01A170BB2780FFC9
:102FD00002C0A0E0B0E8EF01C60FD71F2881969588
:102FE0008795EC01C20FD11DCE018A0F9B1F02C035
:102FF00063E070E06F5F7F4F6417750710F3DF9138
:10300000CF910895CF93DF93DC01ED91FC9111975F
:103010003097D1F09F012F5F3F4FE90121978881C1
:10302000803278F08A33B9F7908180ED890F8A3049
:1030300058F43296E217F30739F4903329F42D93BC
:103040003C9380E090E002C08FEF9FEFDF91CF9143
:1030500008950F931F93CF93DF93EC018B01892B7E
:10306000F1F0E881F9813097D1F080818823B9F0BF
:103070002A813B81858196812817390781F48181D6
:103080000E94C81480FD0BC02881398180E0F801BE
:1030900031832083DF91CF911F910F91089589E0B3
:1030A00020E030E0F4CF0F931F93CF93DF93EA013A
:1030B000890141E653E00E94894E8F3F910541F01E
:1030C00038F00230110558F09883898382E008C0F7
:1030D000009729F0012B19F0888381E001C080E07E
:1030E000DF91CF911F910F9108952F923F924F92B0
:1030F0005F926F927F928F929F92AF92BF92CF9288
:10310000DF92EF92FF920F931F93CF93DF93DC0137
:103110008D909C901197FB01128E9E960D911D91A2
:103120002D913C91D197012B022B032B09F4A1C1C6
:10313000EB018C01D4018C91843009F09AC01D966A
:10314000ED90FC901E97A12CB12CB0E4CB2ED12C8D
:1031500000E010E080E090E088248A94912CD70170
:1031600093962C9130E0A216B30608F044C0B0E666
:10317000CB16B2E0DB0608F043C096012F7133276F
:10318000232B19F4E2E0CE0ED11CF701EC0DFD1D4E
:103190004180512C542C44242081422AF2E0CF0E4D
:1031A000D11C2FEFA21AB20A009729F49201385DC0
:1031B00021153840F0F0A801465E5F4F4C0F5D1FAF
:1031C000612C712CA0E0B0E0DC0199278827BC01BC
:1031D000CD0164297529862997299401201B310B7B
:1031E0000E94531890E0009759F0080F191F412CC6
:1031F000512CC201B4CF892B19F40115110521F40A
:103200008FE38A8F01E010E0FE01E00FF11F128EC4
:103210001D86F70184818C8784FD05C0C701C8968F
:103220000E94281708C020E030E040E050E060E055
:1032300070E080E090E0288339834A835B836C836D
:103240007D838E839F83D7011D968C911D9790E07F
:10325000982F88271C962C911C97822B9B878A87F6
:103260001F968C911F9790E0982F88271E962C917F
:10327000FDC0F801E05CFF4F80819181A281B381A4
:103280008F3F9F4FAF4FBF4F09F44AC0A12CB12CC5
:10329000C12CD12CE12CF12C66246A94712CD40120
:1032A0001B96ED91FC911C97EA0DFB1D808191818D
:1032B000009771F1C114D10429F49C01385D2115E6
:1032C0003840F8F0A701465E5F4F4C0F5D1FA0E04D
:1032D000B0E01601412C512C210133242224BC01E1
:1032E000CD01622973298429952993012E193F095B
:1032F0000E94531890E0009749F0E80EF91E80E014
:1033000090E022E0A20EB11C6C01C9CFE12CF12C9F
:10331000CD2811F0E12CF12CFE01EE0DFF1D128ED7
:1033200020E030E080E090E06EE2AC014F5F5F4F64
:10333000D801D296ED91FC91D397E80FF91F8081C7
:1033400090E080329105B9F08530910511F485EE59
:1033500090E04930510549F42C30310530F4FE013C
:10336000E20FF31F65872F5F3F4FFE01E20FF31F50
:1033700085872F5F3F4FCA014B305105B1F6FE01E3
:10338000E20FF31F15868A8D811142C0232B31F085
:10339000BE01665E7F4FE0E0F0E010C08FE38A8FF1
:1033A000E1E0F0E029C090E09C01215431092A318C
:1033B000310558F0DB018D93BD013196CB010D979E
:1033C000DC018C918111EFCF17C0D801D2962D91DD
:1033D0003C91D397D9011C962C9130E0E930F1054E
:1033E00018F448E050E002C040E150E024233523C7
:1033F000232B01F38096DECFEC0FFD1F128ED80138
:10340000D296ED91FC91D3978485811101C01D86E0
:10341000D801D296ED91FC91D39783858C87D29673
:103420008D919C91D3974C960E940D174B015C0196
:1034300068839982AA82BB821C821D821E821F829F
:10344000D801D296ED91FC91D397878990E0982F7F
:1034500088272689822B9B878A87D296ED91FC91BB
:10346000D397818D90E0982F8827208D822B998784
:103470008887DF91CF911F910F91FF90EF90DF90A0
:10348000CF90BF90AF909F908F907F906F905F9004
:103490004F903F902F9008950F931F93CF93DF93FA
:1034A000EC01E881F9818F010F5F1F4F6081862F4A
:1034B00090E0009731F061E673E00E94BC4E009707
:1034C00031F019830883BC0180E090E003C06FEF06
:1034D0007FEFCB01DF91CF911F910F9108950F9353
:1034E0001F93CF93DF938C01C0E0D0E0F80161918E
:1034F00071918F016115710529F180E090E00E94C2
:10350000D14EAE0141705527C0FF02C040E050E8E7
:10351000D695C7959B0133272C0F3D1F240F351FD0
:10352000A9014170552720FF02C040E050E83695C0
:103530002795C72FDD27B9016C0F7D1FEB01C40F45
:10354000D51FD4CFCE01DF91CF911F910F91089558
:10355000FB01480F591F2191DC012D93CD01A417C8
:10356000B507C9F70895FB01438D50E0542F442758
:10357000928D492B60E070E0833079F4858990E08A
:10358000982F88272489822BA0E0B0E0DC019927BE
:103590008827482B592B6A2B7B2BCB01BA01089526
:1035A000FB01228F338FDC018C91833029F4CA0117
:1035B000AA27BB27848B958B08950F931F93CF93D6
:1035C000DF938C01EB01DC018D919C91C4960E94EC
:1035D0000D176E837F8388879987F8018081918199
:1035E000C8960E9428172A873B874C875D876E877D
:1035F0007F87888B998BD801ED91FC9181A1827096
:103600008D831E8A1F8A188E198EDF91CF911F918C
:103610000F9108958F929F92AF92BF92EF92FF9277
:103620000F931F93CF93DF93FC0123812223C1F1DA
:10363000EC017C01F7E3EF0EF11C2BA93CA94DA98D
:103640005EA901E010E0B70189810E941A1581117D
:1036500029C01B828BA99CA9ADA9BEA90B8D1C8D6D
:103660002D8D3E8D8BA09CA0ADA0BEA0AC01BD0158
:10367000481959096A097B094017510762077307FE
:1036800078F46A81623061F4A9019801280F391F2A
:103690004A1F5B1F01E010E0B70189810E941A15E3
:1036A00080E001C081E0DF91CF911F910F91FF90E9
:1036B000EF90BF90AF909F908F9008958F929F92C0
:1036C000AF92BF92FF920F931F93CF93DF93EC01C2
:1036D0004A015B018BA99CA9ADA9BEA9481759074E
:1036E0006A077B07E9F0CE010E940A1BF82E8111C0
:1036F00018C001E010E0A5019401BE01695C7F4F94
:1037000089810E94CF14882331F0FF24F394882408
:103710008A94982C54018BAA9CAAADAABEAA01C077
:10372000F12C8F2DDF91CF911F910F91FF90BF90C2
:10373000AF909F908F9008954F925F926F927F927B
:103740008F929F92AF92BF92CF92DF92EF92FF92B1
:103750000F931F93CF93DF936C0148015901DB0155
:10376000CA010297A109B1098C019D014CE036956F
:103770002795179507954A95D1F7F60147A550A9C2
:1037800061A972A9400F511F621F731F8C019D0117
:10379000E3E03695279517950795EA95D1F7E80167
:1037A000D1708770992711E001C0110F8A95EAF74F
:1037B00001E02A013B01FFEF4F1A5F0A6F0A7F0AFF
:1037C000C6010E945E1B811125C0F601EC0FFD1F92
:1037D00097A9492F412321E030E011F420E030E0A7
:1037E000E216F306C9F0912797ABF6010383F1E0E7
:1037F0008F1A9108A108B10881F0110F31F72196B5
:1038000011E0C11592E0D90701F7C0E0D0E0B301A3
:10381000A201CFCF81E001C082E0DF91CF911F9163
:103820000F91FF90EF90DF90CF90BF90AF909F905F
:103830008F907F906F905F904F9008952F923F925E
:103840004F925F926F927F928F929F92AF92BF92B0
:10385000CF92DF92EF92FF920F931F93CF93DF935C
:1038600000D000D01F92CDB7DEB7FC016A017B010A
:10387000208131813C832B834230510561057105E4
:1038800008F464C1AB81BC8157964D915D916D91F7
:103890007C915A97C416D506E606F70608F056C17D
:1038A0008C91823009F45CC018F4813041F04EC133
:1038B000833009F47EC0843009F4A5C047C1860175
:1038C000169507950C0D1D1DC801892F9927869502
:1038D000EB81FC8143A154A165A176A1480F591F3A
:1038E000611D711DCF010E945E1B882321F06FEFC7
:1038F0007FEFCB0134C15801FFEFAF1ABF0A11703F
:10390000EB81FC81E00FF11F17A9C501892F9927D1
:103910008695AB81BC8193964D915D916D917C9123
:103920009697480F591F611D711DCD010E945E1BA6
:103930008111DDCFB1E0BB22EB81FC81EA0DFB1DE3
:1039400087A9612F70E0782BC0FE06C024E0769531
:1039500067952A95E1F701C07F7080E090E0FFC095
:1039600077276F2D5E2D4D2DEB81FC8183A194A1D6
:10397000A5A1B6A1480F591F6A1F7B1FCF010E9446
:103980005E1B8111B4CFCC0CDD1CE894C0F8F1E0D3
:10399000DF22EB81FC81EC0DFD1D90AD692F70E005
:1039A000762F6627EB81FC81EC0DFD1D87A9682B26
:1039B000D4CFEB81FC8183A194A1A5A1B6A1B701CD
:1039C000A60117E076956795579547951A95D1F713
:1039D000480F591F6A1F7B1FCF010E945E1B811178
:1039E00086CFCC0CDD1CCC0CDD1CFCEFCF22F1E033
:1039F000DF22C601C7962B813C81820F931F0E9454
:103A00000D179F70ACC032844384548465847684DF
:103A100007851089B189BD83232D342D452D562D61
:103A2000672D702F812F9B2FA0E025800E946D7441
:103A300041F04681578160857185452B462B472B88
:103A400011F4211083C0468157816085718546013C
:103A50005701841A950AA60AB70AAB81BC81199648
:103A60000D90BC91A02DBA83A983B2E02B1230C077
:103A7000232D342D452D562D672D702F812F9D819F
:103A8000AFEF0E944F7409E00E942A74B22FA32F57
:103A9000E42F152F89819A819C0140E050E06B2F23
:103AA0007A2F8E2F912F0E948573281539054A058C
:103AB0005B0508F44BC082169306A406B50609F40C
:103AC0004AC0C701B6016F5F7F4F8F4F9F4F47C0FE
:103AD00093E0291209C082899389A489B58988163F
:103AE0009906AA06BB0668F386899789A08DB18DD1
:103AF000892B8A2B8B2B79F5EB81FC8183A194A1F7
:103B0000A5A1B6A1B701A60127E0769567955795BF
:103B100047952A95D1F7480F591F6A1F7B1FCF0180
:103B20000E945E1B8111E3CECC0CDD1CCC0CDD1C95
:103B3000FCEFCF22F1E0DF22C601C7962B813C814A
:103B4000820F931F0E940D179F7709C061E070E0FC
:103B500080E090E004C06FEF7FEF8FEF9FE70F9062
:103B60000F900F900F900F90DF91CF911F910F91B9
:103B7000FF90EF90DF90CF90BF90AF909F908F908D
:103B80007F906F905F904F903F902F9008954F924D
:103B90005F926F927F928F929F92AF92BF92CF92DD
:103BA000DF92EF92FF920F931F93CF93DF93EC017D
:103BB0006A017B0108811981F8018081843029F034
:103BC00080E090E0A0E2B0E004C080E090E0A0E0FF
:103BD000B0E1C816D906EA06FB0610F082E0AAC0DA
:103BE000D701C6018F719927AA27BB27892B8A2B5A
:103BF0008B2BA1F7CEA2DFA2E8A6F9A68E809F802C
:103C0000A884B98481149104A104B10469F5F80170
:103C100080818330E8F4F80187819085A0E0B0E0EE
:103C2000B701A601E5E07695679557954795EA9522
:103C3000D1F7481759076A077B0780F6F80187A173
:103C400090A5A1A5B2A58EA79FA7A8ABB9AB48C068
:103C5000F80187A190A5A1A5B2A51D820097A10595
:103C6000B105C9F24C015D01F80141845284612C17
:103C7000712C39E0440C551C661C771C3A95D1F721
:103C8000B501A401C414D504E604F70410F1CE0173
:103C90000E941E1C4B015C016F3F7F4F8F4F9F4F57
:103CA00009F447C082E088169104A104B10408F425
:103CB00095CFF8018789908DA18DB28D88169906D0
:103CC000AA06BB0608F08ACFC418D508E608F7088C
:103CD000D7CFC8010E949A176EA77FA788AB99AB70
:103CE0008AA69BA6ACA6BDA68EA59FA5A8A9B9A984
:103CF0000097A105B10509F471CFB701A60129E02C
:103D000076956795579547952A95D1F7840F951F16
:103D1000A61FB71F8EA79FA7A8ABB9ABF1E0DF2204
:103D200087E3C80ED11CC00ED11EDBAACAAA80E050
:103D300001C081E0DF91CF911F910F91FF90EF9033
:103D4000DF90CF90BF90AF909F908F907F906F90BB
:103D50005F904F900895CF93DF93EC011B828FEF1C
:103D60009FEFDC018BAB9CABADABBEABCE010E9439
:103D70005E1B811134C0FE01EA5CFD4F808190E042
:103D8000982F882731972081822B85359A4A49F5CB
:103D90004BE050E065E076E0CE01C7960E948B17BD
:103DA000892B09F18FA98B3E19F0885E8230F8F4D7
:103DB00043E050E061E176E0CE0183599F4F0E94DD
:103DC0008B17892B91F045E050E065E176E0CE015C
:103DD00087579F4F0E948B17892B49F406C084E0B8
:103DE00007C083E005C081E003C080E001C082E03D
:103DF000DF91CF9108952F923F924F925F926F92F1
:103E00007F928F929F92AF92BF92CF92DF92EF926A
:103E1000FF920F931F93CF93DF93CDB7DEB7E29757
:103E20000FB6F894DEBF0FBECDBF6B01142FDB01C0
:103E30001D921C920E9402187C0197FD84C2FC0115
:103E4000EE0FFF1FE152F44F208031802114310426
:103E500009F47BC2F601318220821E7FD1018C9150
:103E6000882369F011968C910E94C81480FD07C0C8
:103E7000112309F46CC282FF6AC28AE02CC4F101EA
:103E80001082E1828E2D0E94081480FD62C21123EF
:103E900011F082FDF2CF40E050E0BA01C1010E9472
:103EA000AB1E823009F043C08E010F5F1F4F7801B7
:103EB000810103501E4F510123ECA21A2DEFB20ACB
:103EC0006701F80134978081882321F0C8010E949E
:103ED0000D1703C060E070E0CB01D6016D937D93B8
:103EE0008D939D936D01005F1F4F0A151B0549F7C8
:103EF0008E010F5E1F4FD7014D905D906D907D90AC
:103F00007D01498E5A8E6B8E7C8E41145104610462
:103F1000710441F0B301A201C1010E94AB1E8230C5
:103F200010F411C083E0E016F10629F7D0C3198E12
:103F30001A8E1B8E1C8E843011F481E0CCC382302B
:103F400010F08DE0C8C3F101EE5BFF4F813051F4FA
:103F5000910129583F4F81918111F3CFE217F30767
:103F6000D1F7F9C1D101AD5BBF4F8C9190E0982F93
:103F700088272081822B8115924019F7F101E25B9D
:103F8000FF4F8080912C982C882431978081882A3B
:103F90008114910419F0A12CB12C07C0C101855ADC
:103FA0009F4F0E940D174B015C01D1015B968D92D2
:103FB0009D92AD92BC925E97F101E95BFF4F00814B
:103FC000F10102838FEF800F823008F0BACFEC5BF3
:103FD000FF4F1081812F90E01A969C938E93199732
:103FE000009709F4AECF9C0121503109822393231D
:103FF000892B09F0A6CF3596808190E0382F2227B3
:10400000319780812901482A5A8A498A18965C92F8
:104010004E921797C2018F709927892B09F091CF83
:104020003396808190E0982F882731972081822BCA
:104030002C01612C712C892B39F4C101895A9F4FB5
:104040000E940D172B013C01F101EA5BFF4FE0815B
:10405000F0E0FE2FEE27D101AB5BBF4F8C91E82B38
:10406000309709F46ECFA02FB0E0A50194010E9413
:104070005A736D8F7E8F8F8F98A36F01E12CF12C77
:10408000C9A2DAA2EBA2FCA289899A89B4E096952A
:104090008795BA95E1F7C80ED91EE11CF11CD7012E
:1040A000C601CD8CDE8CEF8CF8A0C80ED91EEA1E9E
:1040B000FB1E4C145D046E047F0408F442CFC30160
:1040C000B2016C197D098E099F09212F30E040E073
:1040D00050E00E948573211531054105510509F411
:1040E00030CF263F0FEF300740070FE0500708F0B2
:1040F00028CF263F1FEF31074105510540F4263FE9
:104100008FE038074105510520F411E003C013E0AA
:1041100001C012E029013A0192E0490E511C611CD4
:10412000711CD10157964D925D926D927C925A9777
:10413000298D3A8D4B8D5C8D5F962D933D934D93DC
:104140005C939297DA01C90129A13AA14BA15CA124
:10415000820F931FA41FB51FF10183A394A3A5A3EE
:10416000B6A3498D5A8D6B8D7C8D4C0D5D1D6E1DDA
:104170007F1D43A754A765A776A7133029F5EE59ED
:10418000FF4F808190E0982F882731972081822BE4
:10419000892B09F0D6CEC988DA88CD2809F0D1CE8E
:1041A000C1018D599F4F0E940D17D10197966D93B4
:1041B0007D938D939C939A97E2E0440C551C661C6A
:1041C000771CEA95D1F72DC0C988DA88CD2809F483
:1041D000B8CECD8CDE8CEF8CF8A0C80ED91EEA1EAE
:1041E000FB1EC7A2D0A6E1A6F2A6123029F4440C09
:1041F000551C661C771C15C0A3E0B0E0A30192011A
:104200000E945A73DC01CB01B695A79597958795C7
:10421000E1E04E22552466247724480E591E6A1E7A
:104220007B1EFFEF4F0EF1E05F1E611C711C59E019
:1042300076946794579447945A95D1F784149504CB
:10424000A604B70408F47DCE8FEF9FEFDC01F101E7
:10425000838B948BA58BB68B8787908BA18BB28B2E
:1042600080E88483133009F052C0E859FF4F808101
:1042700090E0982F882731972081822B019709F0B1
:1042800046C0498D5A8D6B8D7C8D4F5F5F4F6F4F50
:104290007F4FC1010E945E1B811139C0D10114966C
:1042A0001C92F101EA5CFD4F808190E0982F8827F5
:1042B00031972081822B85359A4A49F5C101C796ED
:1042C0000E940D17623572458146914401F5C10186
:1042D000855E9D4F0E940D1762377247814491465B
:1042E000B1F4C101815E9D4F0E940D17D10153961B
:1042F0006D937D938D939C935697C1018D5D9D4FDA
:104300000E940D17F1016787708B818B928BD10111
:104310001C938091DD0B9091DE0B01969093DE0B48
:104320008093DD0B16969C938E9315978DE797E0FF
:104330001C969C938E931B978DE799E01E969C93F9
:104340008E931D9704C08BE0C6C18CE0C4C180E091
:10435000C2C183E0C0C1F101E056FF4F808190E00F
:10436000982F882731972081822B8115914009F061
:10437000E8CDF101ED55FF4F81E090E0008002C0F3
:10438000880F991F0A94E2F78115924009F0D9CD60
:10439000C10181589F4F0E942817498C5A8C6B8C01
:1043A0007C8C53014201C12CD12C7601498A9A8A16
:1043B000AB8ABC8ACD8ADE8AEF8AF88E5201CB881E
:1043C000DC88E12CF12C00E010E00E9446742D8F77
:1043D00039A3742E652E562E472E8DA39EA3562DDF
:1043E000652D742D2F3F3F4F4F4F5F4F6105710576
:1043F0008105910511F008F0A4CDC10185579F4FAB
:104400000E940D17D1015B966D937D938D939C93C4
:104410005E97F101EB55FF4F8081F101828381307E
:1044200009F08FCDEC55FF4F01E010E0008002C095
:10443000000F111F0A94E2F71A961C930E93199716
:104440000115110509F47DCDC1018D569F4F0E94C4
:104450000D179B01AC016E3FBFEF7B078B07BFE7DA
:104460009B0708F06ECDDC01CB010296A11DB11DAA
:10447000F101878B908FA18FB28F898C9A8CAB8C36
:10448000BC8C878E90A2A1A2B2A2C10181579F4F7E
:104490002FA338A749A75AA70E940D17860E971E6B
:1044A000A81EB91E898A9A8AAB8ABC8AF10183A6A2
:1044B00094A6A5A6B6A6C10189579F4F0E940D17C5
:1044C000898C9A8CAB8CBC8C860E971EA81EB91E4C
:1044D000F10183A294A2A5A2B6A2A988BA88CB882A
:1044E000DC8845015601C12CD12C76018BA69CA6F7
:1044F000ADA6BEA6CFA6D8AAE9AAFAAAD8012FA12E
:1045000038A549A55AA50E945A737B018C0120E069
:1045100030E0A901698BFA8A0B8B1C8B2D8B3E8BAB
:104520004F8B588F9401A50160E070E080E090E02F
:1045300057016801E12CF12C00E010E00E94467464
:1045400059016A017B018C012D8D39A1472D562D12
:10455000652D742D8DA19EA10E94647408F4F1CC88
:10456000C10189569F4F0E940D17D10197966D93F7
:104570007D938D939C939A97C12CD12C760100E06A
:1045800010E00115110511F5F10181859285A0E07A
:10459000B0E0C816D906EA06FB0608F0D2CC47A15F
:1045A00050A561A572A5C1010E949A17AB01BC017B
:1045B0004C0D5D1D6E1D7F1DC1010E945E1B811192
:1045C000BCCCFFEFCF1ADF0AEF0AFF0AF101E00FC0
:1045D000F11F87A9813821F0005E1F4F1170D1CFE4
:1045E000C801855B9F4F820D931D0E940D176B01C3
:1045F0007C01623071058105910508F4A2CCF101BE
:104600008789908DA18DB28DC816D906EA06FB0662
:1046100008F097CCA185B285A701960122503109F7
:10462000410951090E945A7303A514A525A536A571
:10463000DC01CB01800F911FA21FB31F87A790AB96
:10464000A1ABB2ABF10183A194A1A5A1B6A1B70121
:10465000A601E7E07695679557954795EA95D1F7D6
:10466000480F591F6A1F7B1FC1010E945E1B8111E9
:1046700064CCC6018F779927880F991F880F991FDF
:10468000C796820D931D0E940D176F3FFFEF7F07A6
:104690008F079F0771F00FEFC01AD00AE00AF00AE7
:1046A0006C157D058E059F0509F04BCC6B017C01D7
:1046B000C9CFD10153966D937D938D939C9356975B
:1046C000F1016787708B818B928B14E020CE843050
:1046D00009F037CC32CCE2960FB6F894DEBF0FBEAD
:1046E000CDBFDF91CF911F910F91FF90EF90DF90A1
:1046F000CF90BF90AF909F908F907F906F905F9082
:104700004F903F902F9008952F923F924F925F923B
:104710006F927F928F929F92AF92BF92CF92DF92D1
:10472000EF92FF920F931F93CF93DF9300D000D0AF
:10473000CDB7DEB71C016A017B0128013901423087
:1047400051056105710508F4EEC0FC018789908D63
:10475000A18DB28D481759076A077B0708F0E3C09F
:104760008081823009F47AC018F4813029F0DBC0EE
:10477000853008F495C0D7C05A01B694A794A40E0A
:10478000B51EC501892F99278695D10193964D9124
:104790005D916D917C919697480F591F611D711D18
:1047A000C1010E945E1B182F8111BEC04501BFEFE1
:1047B0008B1A9B0AE1E0BE22A20CB31CD701C601F2
:1047C00081709927AA27BB2789839A83AB83BC83EF
:1047D000C0FE0BC0D501D7968C91282F2F70B0E169
:1047E0004B9EC0011124822B01C0842DF50187ABA3
:1047F00081E0D10113968C93139793964D915D911F
:104800006D917C919697C401892F99278695480FC1
:10481000591F611D711DC1010E945E1B182F81115E
:1048200083C0B1E09B22F101E80DF91D89819A81D5
:10483000AB81BC81892B8A2B8B2B41F054E0769481
:104840006794579447945A95D1F706C067A9607F3B
:10485000852D8F70462E482A47AA60C077276F2D76
:104860005E2D4D2DF10183A194A1A5A1B6A1480F04
:10487000591F6A1F7B1FC1010E945E1B182F8111E7
:1048800053C0CC0CDD1CE894C0F8F1E0DF22F1014C
:10489000EC0DFD1D47AAF101EC0DFD1D50AE3EC013
:1048A000F10183A194A1A5A1B6A127E07695679512
:1048B000579547952A95D1F7480F591F6A1F7B1FB7
:1048C000C1010E945E1B182F81112EC0D1018C9155
:1048D000CC0CDD1CCC0CDD1C8430A1F0BFE07B22B5
:1048E000C6018C7F9170C796820D931D0E940D1793
:1048F000DC01CB0188279927AA27B07F482A592AAB
:104900006A2A7B2AECEFCE22E1E0DE22C601C796BE
:10491000B301A201820D931D0E94511781E0D101C4
:1049200013968C9301C012E0812F0F900F900F907F
:104930000F90DF91CF911F910F91FF90EF90DF903B
:10494000CF90BF90AF909F908F907F906F905F902F
:104950004F903F902F9008952F923F924F925F92E9
:104960006F927F928F929F92AF92BF92CF92DF927F
:10497000EF92FF920F931F93CF93DF9300D000D05D
:10498000CDB7DEB79C838B836A017B0109831A83D1
:10499000322E232E82E0882E912CA12CB12C412C7A
:1049A000512C32014394EB81FC8186899789A08D3B
:1049B000B18D0097A105B105A1F182309105A10546
:1049C000B10558F095018401081B190B2A0B3B0B0C
:1049D0000C0D1D1D2E1D3F1D04C009811A81232DA4
:1049E000322DB301A201481B590B6A0B7B0B4C0DF6
:1049F0005D1D6E1D7F1DEB81FC81808191810E9478
:104A0000842381110FC0EB81FC8186899789A08D59
:104A1000B18D0197A109B109868B978BA08FB18FBA
:104A2000C2CF80E00F900F900F900F90DF91CF9149
:104A30001F910F91FF90EF90DF90CF90BF90AF90BC
:104A40009F908F907F906F905F904F903F902F90AE
:104A500008952F923F924F925F926F927F928F9222
:104A60009F92AF92BF92CF92DF92EF92FF920F93FD
:104A70001F93CF93DF9300D000D000D0CDB7DEB727
:104A80001C016A017B0128013901DC010D90BC91F8
:104A9000A02DBE83AD83423051056105710510F430
:104AA00082E003C1ED81FE818789908DA18DB28D59
:104AB000481759076A077B0798F7012B022B032B2E
:104AC00029F4C982DA82EB82FC825BC0AD81BE81AF
:104AD0008C91843021F4F1018581823091F30FEFC4
:104AE0001FEF9801B301A2018D819E810E94842352
:104AF000882339F3DAC0613071058105910581F2AF
:104B00006F3F7F4F8F4F9F4F09F46EC0AD81BE81C5
:104B10008C91843009F06AC0ED81FE81838994898B
:104B2000A589B6894789508D618D728D4250510992
:104B30006109710984179507A607B70750F4019614
:104B4000A11DB11D838B948BA58BB68B8481816055
:104B50008483FFEFCF1ADF0AEF0AFF0AC814D904D3
:104B6000EA04FB0409F04EC075016401ED81FE8189
:104B70008789908DA18DB28D88169906AA06BB06ED
:104B800068F4B701A601C1010E941E1C4B015C0123
:104B9000611571058105910509F0ADCFAD81BE812B
:104BA0008C91843009F080C04BC0F1018581811166
:104BB0005EC0C680D780E084F184C414D504E604C6
:104BC000F70409F46DC0B701A601C1010E941E1CC3
:104BD000623071058105910508F462CF6F3FFFEFE8
:104BE0007F078F079F07B1F581E05FC000E010E00D
:104BF0009801B701A601CD010E948423882309F4FE
:104C00008BCF53C0AD81BE818C918430A1F49701CC
:104C1000860189819A81AB81BC81081B190B2A0B03
:104C20003B0BE12CF12CAC01BD018D819E810E94DA
:104C30009C1B81113AC089829A82AB82BC8294CF3C
:104C4000411451046104710409F0AFCFD1011596EC
:104C50001C922AC02FEFC21AD20AE20AF20A6C157D
:104C60007D058E059F0501F56B017C01A6CF833084
:104C7000D9F4F10146815781608571854416550646
:104C80006606770688F082899389A489B589840F9E
:104C9000951FA61FB71F84159505A605B70520F01B
:104CA00082E0D10115968C9380E026960FB6F89499
:104CB000DEBF0FBECDBFDF91CF911F910F91FF904F
:104CC000EF90DF90CF90BF90AF909F908F907F90AC
:104CD0006F905F904F903F902F9008958F929F928A
:104CE000AF92BF92CF92DF92EF92FF920F931F93FA
:104CF000CF93DF93EC014E815F8168857985CA8807
:104D0000DB88EC88FD88C40ED51EE61EF71E4C1508
:104D10005D056E057F0591F04A015B018FEF881AF2
:104D2000980AA80AB80A95018401888199810E948D
:104D30008423811105C0B501A401E9CF1D8280E063
:104D4000DF91CF911F910F91FF90EF90DF90CF9067
:104D5000BF90AF909F908F9008956F927F928F92A7
:104D60009F92AF92BF92CF92DF92EF92FF920F93FA
:104D70001F93CF93DF9300D000D0CDB7DEB73C01B7
:104D800049835A836B837C830E940A1B49815A8121
:104D90006B817C81811139C0C3010E949A174B013C
:104DA0005C01F30163AB74AB85AB96AB6301F7E3D6
:104DB000CF0ED11C40E052E060E070E0C6010E94DE
:104DC0008217E12CF12CF30181859285E816F90612
:104DD00048F081E0F30121853285E216F306B1F453
:104DE00080E014C001E010E0A50194012E0D3F1DEC
:104DF000411D511DB601F30181810E941A158111D7
:104E0000E8CF8FEFE81AF80ADECF81E00F900F901D
:104E10000F900F90DF91CF911F910F91FF90EF9026
:104E2000DF90CF90BF90AF909F908F907F906F90CA
:104E300008953F924F925F926F927F928F929F92CE
:104E4000AF92BF92CF92DF92EF92FF920F931F9398
:104E5000CF93DF93CDB7DEB72A970FB6F894DEBFB6
:104E60000FBECDBF6C0149835A836B837C83DC0109
:104E70000D90BC91A02DBA87A987452B462B472BB7
:104E8000B9F41F964D905D906D907C9052974114AF
:104E9000510461047104A9F157968D919D910D9073
:104EA000BC91A02D481659066A067B0670F129C0F0
:104EB00049815A816B817C810E941E1C4B015C01DF
:104EC000623071058105910508F43AC26F3F7F4F4A
:104ED0008F4F9F4F29F46FEF7FEF8FEF9FEF3BC214
:104EE000E985FA858789908DA18DB28D88169906FE
:104EF000AA06BB0608F429C249805A806B807C80D0
:104F000004C0412C512C32014394E985FA858389F0
:104F10009489A589B689892B8A2B8B2B11F460E0A3
:104F200010C2A985BA852C9157968D919D910D90AF
:104F3000BC91A02D243009F02FC1A3019201225071
:104F40003109410951092D833E834F8358870297C8
:104F5000A109B109281739074A075B0720F01D820C
:104F60001E821F8218868D809E80AF80B884332475
:104F70003394E985FA8587A590A9A1A9B2A9B501BD
:104F8000A4011CE076956795579547951A95D1F73A
:104F9000480F591F6A1F7B1FCF010E945E1B8111A2
:104FA0005DC0D501C40143E0B695A7959795879557
:104FB0004A95D1F79C013170C40187709927F32D70
:104FC00001C0FF0F8A95EAF78F2FA985BA855796FA
:104FD0004D915D916D917C915A977A018B01B2E070
:104FE000EB1AF10801091109E985FA85E20FF31FAF
:104FF00097A99823B501A4014F5F5F4F6F4F7F4F73
:105000004E155F056007710710F4880F06C040E079
:1050100050E0BA0120E032E080E0911106C0E2E009
:105020008E0E911CA11CB11C21C08D809E80AF8072
:10503000B884481559056A057B05A9F0882319F03D
:105040004A015B01D1CF2F5F3F4F211582E0380726
:1050500010F481E0F5CF4A015B018BCF88248A945C
:10506000982C540103C0812C912C5401D501C4010A
:105070000197A109B1098E3F9F4FAF4FBF4F08F075
:1050800064C1EE24E394F12C01E010E020E030E074
:10509000B501A40189859A850E949C1B823009F480
:1050A0004FC1813009F417CF29813A814B815C814E
:1050B000232B242B252B19F492E0D6011DC0F601D9
:1050C00095819230D9F4B301A2014F5F5F4F6F4FCA
:1050D0007F4F84169506A606B70681F04681578154
:1050E00060857185441A550A660A770AD601428A94
:1050F000538A648A758A93E015969C93F60195818C
:10510000923009F425C146895789608D718D0981D6
:105110001A812B813C810F5F1F4F2F4F3F4F80160D
:105120009106A206B306B1F441155105610571055A
:1051300029F04F5F5F4F6F4F7F4F04C042E050E058
:1051400060E070E0D60156964D935D936D937C932D
:105150005997FEC0452B462B472B49F481E090E040
:10516000A0E0B0E0F601868B978BA08FB18F950100
:10517000840149815A816B817C81C6010E94AC24E3
:105180008111DBC081E090E0A0E0B0E0F601868B09
:10519000978BA08FB18FA7C089809A80AB80BC808D
:1051A000481459046A047B0409F043C053014201C6
:1051B0002FEF821A920AA20AB20A88169906AA0644
:1051C000BB0628F092E0892E912CA12CB12CB501C0
:1051D000A401C6010E941E1C613071058105910564
:1051E00009F4AEC06F3F3FEF73078307930709F4DD
:1051F00072CE672B682B692BB9F0E985FA85878514
:105200009089A189B28982309105A105B10588F004
:105210004789508D618D728D84179507A607B70752
:1052200040F42C013D0105C081149104A104B10496
:10523000E9F553014201FFEF8F1A9F0AAF0ABF0A37
:10524000E985FA858789908DA18DB28D881699069A
:10525000AA06BB0660F0F2E04F1651046104710427
:1052600008F45DCE82E0882E912CA12CB12CB501E2
:10527000A401C6010E941E1C8B019C0161157105D1
:105280008105910599F0613071058105910529F03D
:105290006F3F7F4F8F4F9F4F19F4B801C9015BC01B
:1052A00084149504A604B70431F639CE0FEF1FEF2E
:1052B0009801B501A40189859A850E9484238111F2
:1052C0003CC089819A81AB81BC810097A105B10561
:1052D00051F095018401AC01BD0189859A850E9438
:1052E000842381112AC0A985BA851F968D929D922B
:1052F000AD92BC925297FD0183899489A589B689A4
:105300004789508D618D728D425051096109710933
:10531000481759076A077B0738F00197A109B109B7
:10532000838B948BA58BB68BA985BA8514968C91AB
:105330001497816014968C9308C0813009F4CBCD0A
:1053400061E070E080E090E006C0B401C50103C0F8
:10535000882349F2F5CF2A960FB6F894DEBF0FBE28
:10536000CDBFDF91CF911F910F91FF90EF90DF9014
:10537000CF90BF90AF909F908F907F906F905F90F5
:105380004F903F9008954F925F926F927F92AF92AD
:10539000BF92CF92DF92EF92FF920F931F93CF9322
:1053A000DF93EC0108811981CEA0DFA0E8A4F9A465
:1053B00080E2C80ED11CE11CF11CF8018081843010
:1053C00029F080E090E0A0E2B0E004C080E090E04E
:1053D000A0E0B0E1C816D906EA06FB0620F01EA63A
:1053E0001FA618AA19AA8EA59FA5A8A9B9A90097B2
:1053F000A105B10509F4AAC05B01B701A60151706E
:1054000066277727452B462B472B09F090C001963E
:10541000A11DB11D8EA79FA7A8ABB9AB4AA55BA5DF
:105420006CA57DA5F8014115510561057105C1F413
:1054300087819085A0E0B0E0B701A60135E07695C0
:105440006795579547953A95D1F7481759076A07D1
:105450007B0708F46CC01EA61FA618AA19AA76C05E
:10546000818592850197A0E0B0E02601370129E00F
:1054700076946794579447942A95D1F7842195217F
:10548000A621B721892B8A2B8B2B09F050C0CE0186
:105490000E941E1C2B013C016230710581059105A3
:1054A00010F482E056C08FEF48165806680678065A
:1054B00011F481E04EC0F8018789908DA18DB28DE5
:1054C000481659066A067B0628F1AB2821F24AA540
:1054D0005BA56CA57DA5CE010E9419272B013C017F
:1054E000611571058105910599F16130710581059D
:1054F0009105B9F28FEF4816580668067806C9F28A
:10550000B301A201C8010E94AD268111D2CF8D81C5
:1055100084608D834AA65BA66CA67DA6B301A2011A
:10552000C8010E949A176EA77FA788AB99ABCEA23D
:10553000DFA2E8A6F9A6E1E0DE22F7E3CF0ED11C58
:10554000C00ED11EDBAACAAA80E003C084E001C05D
:1055500087E0DF91CF911F910F91FF90EF90DF9047
:10556000CF90BF90AF907F906F905F904F900895D5
:10557000CF92DF92EF92FF920F931F93CF93DF931F
:10558000EC016B01E880F98040E050E0BA010E9434
:10559000C71D81112FC000E010E04EA55FA568A9CE
:1055A00079A9C7010E945E1B811124C0F701908177
:1055B000EAA9FBA9943031F490819095991F99271D
:1055C000991F07C0208191E0253E11F0211190E044
:1055D0009170992331F00F5F1F4F0C151D0519F4C1
:1055E0000CC000E010E061E070E0CE010E94C32931
:1055F000882399F2843009F487E0DF91CF911F91DD
:105600000F91FF90EF90DF90CF900895AF92BF92EF
:10561000CF92DF92EF92FF920F931F93CF93DF937E
:10562000EC0108811981CEA0DFA0E8A4F9A4FC0157
:10563000E05CFF4F40815181628173814F3F8FEF6A
:1056400058076807780729F485EEB82EAA24A39492
:1056500021C0CE010E94C71D81112BC0F5CFF801DA
:105660009081EAA9FBA99430F9F490819F77908307
:10567000F801A3824EA15FA168A579A54C155D052F
:105680006E057F05B0F460E070E0CE010E94C32992
:1056900081110CC04EA55FA568A979A9C8010E9417
:1056A0005E1B8823E1F202C0B082E2CF843009F4AD
:1056B00082E0DF91CF911F910F91FF90EF90DF90EB
:1056C000CF90BF90AF900895EF92FF920F931F93EA
:1056D000CF93DF93EC010E940A1B982F81115CC0CD
:1056E0008881833009F04EC08C81813009F04AC036
:1056F00040E052E060E070E07E0187E3E80EF11CDC
:10570000C7010E94821785E5FE01EB5CFD4F808397
:105710008AEA3196808382E58FAB88AF81E689AFD4
:1057200091E49AAF22E77B972083319620833196CC
:105730009083319680834B895C896D897E89CE0107
:10574000815E9D4F0E9451174F85588969897A89DA
:10575000CE018D5D9D4F0E9451178F8D98A1A9A1FB
:10576000BAA19C01AD012F5F3F4F4F4F5F4F2BAB55
:105770003CAB4DAB5EAB01E010E0B70189810E940C
:105780001A151C8240E050E060E089810E948B1570
:1057900091E0811101C090E0892FDF91CF911F919D
:1057A0000F91FF90EF900895CF92DF92EF92FF92CA
:1057B0000F931F93CF93DF938C01DC01ED91FC914C
:1057C000E584F684C7010E94D117F7018283938391
:1057D000C180F801E05CFF4F40815181628173819B
:1057E000C8010E94C71DC82FD12CD1E0C1112AC009
:1057F000D8019E964D915D916D917C91D1978D913F
:105800009C910E945E1BC82F81111CC040E250E099
:10581000B701F80182A993A90E94A81AD801ED91B5
:10582000FC91D383C114D10469F0B0E2EB0EF11CFA
:1058300060E070E0C8010E94C329C82FE1E0CE1AE1
:10584000D108D4CF8C2FC33008F082E0DF91CF9104
:105850001F910F91FF90EF90DF90CF900895CF921E
:10586000DF92EF92FF920F931F93CF93DF93EC01A0
:1058700088819981FC01058516854EA55FA568A9DB
:1058800079A90E945E1B811191C06AA97BA9FB01C5
:105890008081853809F063C040E250E0C8010E9471
:1058A000A81AF801E180F12CFFEFEF1AFF0AF5E0EA
:1058B000EE0CFF1CFA95E1F7C70180569109813083
:1058C000924008F04CC060E070E0CE010E94C32915
:1058D000843009F444C0811169C04EA55FA568A950
:1058E00079A9888199810E945E1B81115FC06AA994
:1058F0007BA9FB018081803C91F540E250E0C8012A
:1059000080960E94A81AF80183A190E08C966FE01F
:1059100070E00E947173E5E0660F771FEA95E1F78A
:10592000E616F706E0F050E4C52ED12C60E070E0FA
:10593000CE010E94C329843091F0811137C04EA559
:105940005FA568A979A9888199810E945E1B811150
:105950002DC06AA97BA9FB018081813C11F082E006
:1059600025C0F0E6CF16F2E0DF0638F440E250E062
:10597000C8018C0D9D1D0E94A81A20E2C20ED11CE8
:10598000CE14DF0498F281E6C81682E0D80668F4E7
:10599000C8010E94D117F801238130E0322F22275D
:1059A0004281242B82179307D1F680E0DF91CF91BB
:1059B0001F910F91FF90EF90DF90CF9008954F923D
:1059C0005F927F928F929F92AF92BF92CF92DF921F
:1059D000EF92FF920F931F93CF93DF93EC016B0134
:1059E000E880F9800FEF1FEF84E0B82E9DE0792E5C
:1059F0004E0160E4860E911C4EA55FA568A979A9A9
:105A0000411551056105710509F4CFC0C7010E9418
:105A10005E1BB82E8111CBC0EAA9FBA98081882327
:105A200009F4CCC0D7019C91943019F5C114D1046C
:105A300021F0833809F0AFC0C6C0853809F0ABC08B
:105A40008EA19FA1A8A5B9A5FE01E05CFF4F8083B0
:105A50009183A283B383CE010E942F2C8111B1C008
:105A6000D7011D96ED91FC911E9784818F738C83D5
:105A7000AAC093859F739C83853E09F48BC08E32A8
:105A800009F488C021E030E0492F4F71483011F00F
:105A900020E030E02C153D0509F07CC09F3009F076
:105AA00068C086FF0EC00585182F1F7B4EA15FA121
:105AB00068A579A5D4014D935D936D937C9313975D
:105AC00002C0811367C08585081364C0D7011B9687
:105AD000AD90BC901C97838D90E0982F8827228DE5
:105AE000822B892B09F056C0808190E08F7B019733
:105AF000789E9001799E300D1124AAE14A2EA2E0F1
:105B00005A2E41E050E0D2018D912D01BF01680F66
:105B1000711DDB0111968C91119790E0982F8827C9
:105B20006C91862B4115510579F02F3F310590F589
:105B3000A901440F551F4A0D5B1DDA018D939C93FB
:105B4000AC012F5F3F4F02C0019621F567E2461678
:105B500062E05606C1F6808186FF2EC02F3F3105D8
:105B6000C8F4220F331FF501E20FF31F11821082D8
:105B700023C0111105C0CF010E94C217081719F1E7
:105B8000C05CDF4F8FEF9FEFDC0188839983AA838E
:105B9000BB8319C01FEF60E070E0CE010E94C329F3
:105BA000B82E882309F428CF02C0BB2061F01EA6BE
:105BB0001FA618AA19AA07C01150EDCF84E0B82E6D
:105BC000F6CFB82EF4CF8B2DDF91CF911F910F918F
:105BD000FF90EF90DF90CF90BF90AF909F908F900D
:105BE0007F905F904F9008952F923F924F925F92D7
:105BF0006F927F928F929F92AF92BF92CF92DF92DD
:105C0000EF92FF920F931F93CF93DF93CDB7DEB741
:105C10002F970FB6F894DEBF0FBECDBF9F878E873C
:105C2000DC018D909C9040E050E0BA010E94C71DBD
:105C300081117FC1F4018081843009F06CC08385BB
:105C400094850E946F1A5C0160E070E08E859F85EC
:105C50000E94DF2C382E81115CC0D4011D96ED917D
:105C6000FC911E9785A190E0982F882724A1822B74
:105C70008A159B0549F7C3A0D12C00E010E080E411
:105C8000E82EF12C0C151D05B1F1C7018F71992774
:105C9000892B19F4B2E0EB0EF11CD4011D96ED91A5
:105CA000FC911E97EE0DFF1D618170E0762F662737
:105CB0008081682B80E090E00E94D14E2B013C0156
:105CC000F401438554859801220F331FFA01E20F36
:105CD000F31F6081718180E090E00E94D14E4616F2
:105CE00057066806790609F0AFCFF2E0EF0EF11C17
:105CF0000F5F1F4FC7CF000F111FD4011B96ED91EF
:105D0000FC911C97E00FF11F80819181892B09F094
:105D10009BCF832D0EC1AE84BF8420E4A20EB11CA4
:105D20008FEF9FEFDC01F50180839183A283B38322
:105D30002FEF29833FEF3D8744244A94542C3201AE
:105D40002E853F852C5C3F4F3B872A87AE85BF85DC
:105D50009E964D915D916D917C91D197C4010E9469
:105D60005E1B8111E6C0EE85FF85E2A8F3A8D7018E
:105D70008C91882309F4D5C01B963C91932F9F7377
:105D80009483853E09F4B9C033FF04C09F3009F005
:105D9000B4C003C09F3009F098C0AE85BF85DF96C0
:105DA0009C91DF9796FDB3C086FF11C0F701F58582
:105DB000F9838F7B8D8796968D919D910D90BC91E7
:105DC000A02DF50180839183A283B38303C02D8529
:105DD000821399C0D7011D968C912981281395C0F3
:105DE000D4011B96CD90DC901C97F701838D90E039
:105DF000982F8827328D832B892B09F086C08081CC
:105E00008F7390E00197FDE0F89F8001F99F100DDE
:105E100011242AE132E03B832A8341E050E0AA8149
:105E2000BB818D91BB83AA83F701E80FF11D8181AE
:105E300090E0982F882730811C01232A41155105B5
:105E400059F10F3F110508F060C0B10180E090E00A
:105E50000E94D14E6C837D838E839F8398012F5F38
:105E60003F4F39872887000F111FF601E00FF11F00
:105E700080819181BC0180E090E00E94D14E2C8114
:105E80003D814E815F812617370748075907E9F59D
:105E9000A1010885198503C023202094B1F52A812A
:105EA0003B812752324009F0BACFD7018C9186FF4F
:105EB0003CC0452BD1F1000F111FF601E00FF11F7F
:105EC00080819181892B89F120C02D85211106C007
:105ED000C7010E94C2173981381729F1AE85BF85E5
:105EE000DF968C9180FD09C04BE050E06A857B8590
:105EF000C7010E948B17892BB1F0F50140825182B6
:105F00006282738202C03FEF12C02FEF2D8760E0E4
:105F100070E08E859F850E94C329882309F416CFDF
:105F200008C084E006C080E004C03D8531503D8754
:105F3000EECF2F960FB6F894DEBF0FBECDBFDF9128
:105F4000CF911F910F91FF90EF90DF90CF90BF9076
:105F5000AF909F908F907F906F905F904F903F9009
:105F60002F9008952F923F924F925F926F927F925F
:105F70008F929F92AF92BF92CF92DF92EF92FF9259
:105F80000F931F93CF93DF93CDB7DEB7CE54D109D4
:105F90000FB6F894DEBF0FBECDBFDC016D907C90D4
:105FA0001197DF962C91207A09F0D0C2D3011B966D
:105FB000ED91FC911C97E12CF12C21913191232B37
:105FC00021F0BFEFEB1AFB0AF8CF4C01F3018081FF
:105FD000843009F032C1C7010E966FE070E00E9474
:105FE00071738B016E5F7F4FC4010E94B82A8111CB
:105FF000AEC29401205C3F4F0F5F174F45E0000F8A
:10600000111F4A95E1F7F40186A197A1A0A5B1A5BA
:10601000801B910BA109B109F90180839183A283AF
:10602000B383D40115968C91159782FFAFC08B7FF7
:1060300015968C93833071F0F40142A553A564A5A5
:1060400075A50FEF1FEF9801C4010E94AC248823AF
:1060500039F07DC2C4010E946E26811178C2ECCF56
:10606000F40186819781A085B185892B8A2B8B2BA2
:1060700009F48CC0808191819A838983828D938D6C
:10608000A48DB58D8F839887A987BA87068D178DC4
:1060900020A131A10E8300270B871C872D873E8707
:1060A0001F86188A198A1A8A1F8A188E198E1A8EC4
:1060B00042A153A164A175A125964CAF5DAF6EAF0F
:1060C0007FAF2597CE0101960E94C71D81113FC267
:1060D000CE0101960E942F2C811139C2D30119964D
:1060E000AD90BC901A97C501A0E0B0E029E0880F00
:1060F000991FAA1FBB1F2A95D1F75C016D019C0156
:10610000A60160E070E080E090E0F401A284B38436
:10611000C484D584E684F784008911890E9446747A
:10612000228733874487558766877787808B918B53
:10613000D3011D96ED91FC911E9789019A01AB0147
:10614000BC01CF01C8960E945717F4010285138540
:10615000248535854685578560897189D3011D96CB
:106160008D919C911E9788960E945717D3011D967A
:10617000ED91FC911E97D40115968C91816081A3BD
:10618000CE0101960E94D42B8111E1C1F301E38479
:10619000F4840585168540E450E060E070E0C801B5
:1061A0000E94821785E8D8018C9380EC90968C939E
:1061B00041E050E020E030E080E490E0B1ECF80114
:1061C000E80FF91FB083FC013196E00FF11F029632
:1061D00010824115510559F0F701E20FF11DE20F50
:1061E000F11D408151814115510509F02F5FF801E2
:1061F000E80FF91F408351830296BC016F71772726
:10620000672B39F7A1E0A30FF701E20FF11DE20FB1
:10621000F11D60817181672B11F03A2FD0CFF80109
:1062200023A33E5F3183C7010E946F1AD801949661
:106230008C93949795969C9387C16401B4E3CB0E9D
:10624000D11C4CE050E0B601CE0101960E94A81A84
:106250008C8580FFAEC080E4F40187AF212C312C07
:106260002101239485E4A82EB12CAC0EBD1EF8E0CC
:10627000AF0EB11C8101D3011B962C911B971C966C
:106280003C914BE050E0BE016F5F7F4FC6012E9600
:106290002FAF2E972F963FAF2F970E94A81A2E96BA
:1062A0002FAD2E972F963FAD2F97B6E02B163104CA
:1062B0004104510418F1F901B201A10181919191B8
:1062C0000097D9F020E130E0440F551F661F771F7B
:1062D000DC01A170BB274A0F5B1F611D711D9695E4
:1062E000879560FF06C0A1E24A27A0E15A27A1E0F6
:1062F0006A272150310941F7E1CF8A01F50127E0F2
:1063000030E0902F9F7080E3890F8A3310F087E38D
:10631000890F215031098293A4E016950795AA951B
:10632000E1F70115110569F7E5E4F0E0EC0FFD1F59
:10633000E20FF31FBEE7B083F60180E090E0821722
:10634000930721F4F601E80FF91F0CC04191403288
:10635000C9F30196F4CF80E28193CF018C199D0996
:10636000089768F428303105B0F7A5E4B0E0AC0F29
:10637000BD1FA20FB31F8C912F5F3F4FEDCFC40104
:106380000E94F42D81110EC0EFEF2E1A3E0A4E0A24
:106390005E0AF4E62F1631044104510409F06ACF75
:1063A00087E0D5C0843009F0D2C08C85D401DF9657
:1063B0008C938C8581FF0AC0C7010C966DE070E05C
:1063C0000E9471738B010F5F1F4F02C001E010E04C
:1063D000B801C4010E94B82A8111B9C00150110945
:1063E00009F487C0F40146A157A160A571A5C801B1
:1063F000E5E0880F991FEA95E1F7481B590B610901
:106400007109C4010E94C71D8111A1C0C6010E946B
:10641000C217F82E6FE0562E7DE0A72EBB24B39452
:10642000D4019E964D915D916D917C91D197C30160
:106430000E945E1B81118BC0E02ED401D296ED919B
:10644000FC91D397D3011B966D917C911C97F58697
:1064500053861486128E138E9801332721503109EA
:10646000A29EC001A39E900D11245AE1252E52E058
:10647000352E20E030E02F3FBFEF3B0749F09C0175
:10648000220F331F260F371FD9012D913C91019602
:10649000D1014D911D01DF01A40FB11D2C93119667
:1064A0003C932115310511F42FEF3FEFB7E22B1686
:1064B000B2E03B0601F72F3F3F4F49F0880F991F8D
:1064C000DB01A80FB91F8D919C91892B19F48E2D9A
:1064D0008064E82EE082D3011396BC9260E070E005
:1064E000C4010E94C329811132C00150110909F071
:1064F00097CFD4019E964D915D916D917C91D197EE
:10650000C3010E945E1B811122C040E250E060E0A6
:1065100070E0F40182A993A90E9482174BE050E039
:10652000B601D401D2968D919C91D3970E94A81A5E
:10653000D401D296ED91FC91D397DF968C9188711E
:10654000848781E0F301838380E001C086E0C25B41
:10655000DF4F0FB6F894DEBF0FBECDBFDF91CF91F6
:106560001F910F91FF90EF90DF90CF90BF90AF9071
:106570009F908F907F906F905F904F903F902F9063
:1065800008952F923F924F925F926F927F928F92D7
:106590009F92AF92BF92CF92DF92EF92FF920F93B2
:1065A0001F93CF93DF93CDB7DEB72C970FB6F89438
:1065B000DEBF0FBECDBF8C01DC010D90BC91A02DC4
:1065C000BC83AB83FB012E2F9F2F81918F32D9F398
:1065D0008C35C9F3422E592EF80116821782108687
:1065E0001186168A178A108E118EF20180818032F0
:1065F00080F098012C5C3F4F3E832D83245F3F4FFA
:1066000038872F832B813C81235F3F4F3A8729872F
:106610008AC080E8D801DF968C9340E050E0BA0150
:10662000C8010E94C71DDDC1C114D10409F008C111
:106630008E9709F405C1929182918E9721F041E0E5
:10664000E41AF108C1F74BE050E060E270E08D81A0
:106650009E810E94821758E0A52EB12C20E030E0E8
:10666000212C46018FEF881A980ACC0CDD1CF3010F
:10667000EC0DFD1D80819181009709F0E5C0F801C6
:1066800084A9853E11F485E084ABF8E0AF16B1042F
:1066900011F4220C220C822D8C708C3009F467C10D
:1066A000822D8370833009F462C131FE64C1D80148
:1066B000DF963C92C8010E94F42DF80197AD81113C
:1066C00067C192FD8EC1D801848184FF7CC1EB81BA
:1066D000FC818081843009F060C116968D919D9176
:1066E0000D90BC91A02DF801828F938FA48FB58F50
:1066F00082859385A485B58588272581822B868F01
:10670000978FA0A3B1A3EF81F88580819181A281A9
:10671000B381F80182A393A3A4A3B5A3B80189858B
:106720009A850E94DD1A5A824982D801ED91FC9126
:1067300063847484E12CF12CCE0101960E944C1AE2
:106740006F3FBFEF7B078B079B0709F41FC16115E4
:106750007105E1E08E07910558F0F701EE0FFF1F7C
:10676000E60DF71D9183808397012F5F3F4F7901DD
:10677000AB016032710558F16F32710541F16C3532
:10678000710529F16038710558F49B01EBE1F6E0E1
:106790004191442329F050E042175307C9F7F6C04E
:1067A0003FEFE316F10408F0F1C0F701EE0FFF1F11
:1067B000E60DF71D71836083C70101967C01BCCF94
:1067C0002C3561F49FEF491A590A5A82498249804F
:1067D0005A80D2012C912F3299F7F4CF40325105D3
:1067E00010F0312C02C0E4E03E2EF701EE0FFF1F47
:1067F000E60DF71DE114F10459F092918291803277
:10680000910511F08E9721F4B1E0EB1AF108F2CF67
:10681000F701EE0FFF1FE60DF71D11821082E11444
:10682000F10409F4B3C0D301C12CD12C8D919D91F9
:106830008032910509F0F8CE2FEFC21AD20AF6CFB6
:10684000332D3360332EF7CE8032910539F08E32FE
:10685000910549F48E149F0409F4BDC0932D9360F3
:10686000392E6401FECE2A153B0520F48E149F04B8
:10687000F9F4ABC0ABE0AA16B10439F4B32DB360A0
:106880003B2E9BE0A92EB12CFACE8E149F0439F03A
:10689000E32DE3603E2EE814F90408F4F0CE220C58
:1068A000220C47018BE0A82EB12C28E030E0D9CF94
:1068B0008038910578F1F32DF260DF2EBC0180E085
:1068C00090E041E653E02B873C870E94894E2B8560
:1068D0003C8587FF09C08F779927FC01E656FE4F5C
:1068E000808190E03D2C16C08F3F9105A1F098F07B
:1068F000A501415051092417350728F0232D2360A5
:10690000322E9501AECFF801E20FF31F94AB2F5F4B
:106910003F4F25C0D32C009749F0E4E2F6E04191C7
:10692000442351F050E048175907C9F74D2D4360F3
:10693000D42E8FE590E013C0AC01415451094A3187
:10694000510518F4A22DA2602A2EAC01415651091E
:106950004A31510520F4B22DB1602B2E8097F801F9
:10696000E20FF31F84AB2F5F3F4F3D2C7ACF232DD7
:106970002260322E9ACE20FE03C0332D3061332E9A
:1069800022FE95CE432D4860342E91CE86E029C05C
:10699000843039F592FF17C024C0D80196966D91C6
:1069A0007C9197977170695C7F4F2B813C81620F5E
:1069B000731F0E94B31AD80116966D937D938D9321
:1069C0009C931997B0CE85E00CC0BBE0AB16B10428
:1069D00009F065CF53CFEBE0AE16B10409F05FCFFD
:1069E0004DCF2C960FB6F894DEBF0FBECDBFDF9112
:1069F000CF911F910F91FF90EF90DF90CF90BF90BC
:106A0000AF909F908F907F906F905F904F903F904E
:106A10002F900895CF93DF93CDB7DEB727970FB6AA
:106A2000F894DEBF0FBECDBF9C838B837E836D83C6
:106A30007A836983CE0101964F830E9402184F81A9
:106A400097FD22C0880F991FFC01E152F44F01907D
:106A5000F081E02D309709F01082EB81FC813097B6
:106A600009F01082FC01E152F44F2B813C8131830B
:106A70002083442359F040E0BE016D5F7F4FCE017B
:106A800005960E94FB1E03C08BE001C080E02796A4
:106A90000FB6F894DEBF0FBECDBFDF91CF91089542
:106AA0002F923F924F925F926F927F928F929F921E
:106AB000AF92BF92CF92DF92EF92FF920F931F930C
:106AC000CF93DF93CDB7DEB7C655D1090FB6F89493
:106AD000DEBF0FBECDBF29967FAF6EAF299700975F
:106AE00009F40FC3142F4C01042F0F73F02E402F05
:106AF000BE016B5B7F4FCE01895B9F4F0E94FB1EE7
:106B0000811109C327968EAD9FAD27979A838983FC
:106B100029966EAD7FAD2997CE0101960E94C132B4
:106B2000E82F811105C021968FAD219787FDE6E002
:106B3000812F8C7109F4E8C0EE2369F0E43029F468
:106B4000CE0101960E94B22FE82F1F2D1860F12E62
:106B5000EE2339F0E3C28D81817109F0D8C212FDB4
:106B6000D2C2F3FEDDC02796EEADFFAD2797808140
:106B7000843009F071C0D401ED93FC93B401CF01CE
:106B80000D960E94DD1A2796EEADFFAD27978585FD
:106B900096854EE150E060E070E002960E94821718
:106BA0002796EEADFFAD2797858596854AE150E0A3
:106BB00060E070E086960E9482172796EEADFFADEA
:106BC00027970584F685E02D80E284830E94821257
:106BD000AB01BC012796EEADFFAD27978585968565
:106BE00008960E9451172796EEADFFAD27970584B2
:106BF000F685E02D81E081A3CE0101960E94D42B81
:106C0000E82F81118BC2F40146815781608571851F
:106C1000411551056105710509F482C000E010E0DD
:106C20009801C4010E942925E82F27962EAD3FAD7B
:106C30002797D40116964D915D916D917C9119978E
:106C40004150510961097109D9011F964D935D9316
:106C50006D937C93529762C06BA97CA90E94B31A72
:106C60002B013C010E948212AB01BC018BA99CA9A3
:106C70000E960E945117EBA9FCA980E283876BA9AD
:106C80007CA920E030E0A90127968EAD9FAD279723
:106C90000E94D01AEBA9FCA9148E158E168E178EA1
:106CA0002796EEADFFAD279781E083834114510411
:106CB00061047104A9F1A3A8B4A8C5A8D6A800E0EE
:106CC00010E09801B301A201CE0101960E9429258E
:106CD000E82F811123C2B601A50127968EAD9FAD85
:106CE00027970E945E1BE82F2796AEADBFAD279772
:106CF000F1E04F1A5108610871081F964D925D929C
:106D00006D927C9252970AC0E11108C28D8184FD78
:106D1000FCC111FF05C080FDFAC102C0E111FEC136
:106D2000F3FE03C00F2D0064F02E2796EEADFFADED
:106D3000279743A954A965A976A9D401D8964D935C
:106D40005D936D937C93DB970BA91CA9DD961C9337
:106D50000E93DC978081843049F54F815885698591
:106D60007A855A964D935D936D937C935D974B8591
:106D70005C856D857E8544278E81482B5E964D937C
:106D80005D936D937C93919725964CAD5DAD6EAD03
:106D90007FAD259792964D935D936D937C939597D8
:106DA000B401CF010D960E94DD1A26C0B8010E94E1
:106DB000B31AF4016683778380879187C8014C9664
:106DC0000E940D178B019C01D4011A966C931A979F
:106DD0001B961C931B971C962C931C971D963C93FB
:106DE0001D971E961C921E971F961C921F975096D9
:106DF0001C92509751961C922796EEADFFAD2797A7
:106E0000D4011196FC93EE938581968113969C9301
:106E10008E9312979696FC92969797961C929797B8
:106E2000D4961D921D921D921C92D79798961C92F3
:106E3000989799961C9299979A961C929A979B96D6
:106E40001C929B979C961C929C979D961C929D973A
:106E50009E961C929E979F961C929F97F5FE59C1F5
:106E60001A967C901A971B96BC916296BFAF629758
:106E7000D4011C96BC916396BFAF6397D4011D9655
:106E8000BC916496BFAF6497D4011E96BC91659681
:106E9000BFAF6597D4011F96BC916696BFAF66974A
:106EA000D40150966C9050975196BC916796BFAFA5
:106EB0006797272D62963FAD629763964FAD6397B4
:106EC00064965FAD649765966FAD659766967FAD86
:106ED0006697862D9B2FA0E00E946D7409F419C15E
:106EE000D40198967C92989799963C9399979A9604
:106EF0004C939A979B965C939B979C966C939C97CC
:106F00009D967C939D979E966C929E979F969C9340
:106F100081859285A0E0B0E029E0880F991FAA1F23
:106F2000BB1F2A95D1F7F401268037804084518415
:106F30008C019D012A968FAF2A972B961FAF2B9716
:106F40002C962FAF2C972D963FAF2D97272D62961D
:106F50003FAD629763964FAD639764965FAD64975C
:106F600065966FAD659766967FAD6697862D679639
:106F70009FAD67972A96AFAC2A972B96BFAC2B97FD
:106F80002C96CFAC2C972D96DFAC2D97E12CF12CC5
:106F900000E010E00E94647409F008F454C0B201EB
:106FA000A101C4010E941E1C1B012C01623071054D
:106FB0008105910538F06F3F7F4F8F4F9F4F21F034
:106FC000E0E003C0E2E001C0E1E0272D62963FADC2
:106FD000629763964FAD639764965FAD64976596CD
:106FE0006FAD659766967FAD6697862D67969FAD68
:106FF00067972A96AFAC2A972B96BFAC2B972C9607
:10700000CFAC2C972D96DFAC2D97E12CF12C00E026
:1070100010E00E945B74722E62963FAF6297639697
:107020004FAF639764965FAF649765966FAF659750
:1070300066967FAF6697682E67969FAF6797EE2339
:1070400009F484CF01C0E0E0D401D0962D923D92A6
:107050004D925C92D397E11161C0272D62963FADAE
:107060006297317040E050E060E070E080E090E0D6
:10707000A0E00E946D7409F44CC0B201A1012796F2
:107080008EAD9FAD27970E949A176B017C01672BED
:10709000682B692B09F441C0272D62963FAD62979A
:1070A00063964FAD639764965FAD649765966FADD9
:1070B000659766967FAD6697862D67969FAD6797B5
:1070C00009E00E942A742A962FAF2A972B963FAF89
:1070D0002B972C964FAF2C972D965FAF2D972D9613
:1070E0000CAD1DAD2EAD3FAD2D97C00ED11EE21ED5
:1070F000F31ED401D496CD92DD92ED92FC92D797F7
:1071000008C089E00FC0E8E009C0E4E007C0E7E09C
:1071100005C080E007C0E82F01C0E2E0D4011D9265
:107120001C928E2FCA5ADF4F0FB6F894DEBF0FBEE7
:10713000CDBFDF91CF911F910F91FF90EF90DF9026
:10714000CF90BF90AF909F908F907F906F905F9007
:107150004F903F902F9008952F923F924F925F92C1
:107160006F927F928F929F92AF92BF92CF92DF9257
:10717000EF92FF920F931F93CF93DF93CDB7DEB7BC
:107180002E970FB6F894DEBF0FBECDBF4C017C87A3
:107190006B873A013E872D87D9011D921C92BE0153
:1071A0006F5F7F4F0E942918811193C1F40187A15D
:1071B00081118FC186A180FF8BC1228533854485D3
:1071C00055856685778580899189A0A4B1A4C2A4DC
:1071D000D3A4E4A4F5A406A517A50E945B74F22F1E
:1071E000E32F6A017B018C01930140E050E060E0F5
:1071F00070E080E090E0AF2EBE2E0E94647409F033
:1072000008F4D6C0CF01692E782ED2C0D40198964A
:10721000FC9198979996EC9199979A965C909A9789
:107220009B96CC909B979C96DC909C979D96EC901F
:107230009D979E96FC909E979F964C903E2F317006
:107240002F2F40E050E060E070E080E090E0A0E0B0
:107250000E946D7409F010C13E2F452D5C2D6D2DDF
:107260007E2D8F2D942D09E00E942A742B833C8360
:107270004D835E836F83788789879A8789819A8116
:10728000DC0119960D911C911A97015011092B815F
:107290003C81022313230115110509F48EC0C98016
:1072A000DA80F40140A951A962A973A9C6010E941C
:1072B0009A17611571058105910509F49FC01B019D
:1072C0002C01200E311E411C511C7301EF2CFF2498
:1072D000E694E114F10409F4C8C0D60119968D9121
:1072E0009C911A979701200F311F8217930718F46A
:1072F0007C01E01AF10A8701A20191016B857C856E
:10730000F60181810E94CF14811183C0E981FA8145
:10731000838181118AC0FE2CEE24FF0C6E187F0839
:10732000AD85BE858D919C9111978E0D9F1D8D937E
:107330009C93EB85FC85EE0DFF1DFC87EB87970189
:1073400040E050E060E070E080E090E0D40198968A
:10735000AC9098979996BC9099979A96CC909A975A
:107360009B96DC909B979C96EC909C979D96FC90AE
:107370009D979E960C919E979F961C919F970E9419
:10738000467498962C93989799963C9399979A96C9
:107390004C939A979B965C939B979C966C939C9727
:1073A0009D967C939D979E968C939E979F969C937B
:1073B0006114710409F02ACF89C02F2F3E2F452D6B
:1073C0005C2D6D2D7E2D8F2D942DA0E00E946D746F
:1073D00041F4D40116966D917D918D919C911997F0
:1073E00008C0F40140A951A962A973A9C4010E946F
:1073F0001E1C623071058105910528F482E0D401DC
:1074000097968C9366C06F3FBFEF7B078B079B07F8
:1074100021F481E0F40187A35CC0D401D0966D9380
:107420007D938D939C93D3973ACF83A994A9A5A9D3
:10743000B6A982199309A409B509A70160E070E013
:1074400084179507A607B70708F065CFBF01695CE9
:107450007F4F982F8827990F40E052E02B853C857D
:10746000820F931F0E94A81A56CFD401D4962D9252
:107470003D924D925C92D797F40180A591A59170B1
:1074800020E032E0281B390B73012615370508F47C
:107490007901D401D4964D915D916D917C91D797EE
:1074A00089819A810E945E1B8111B3CFF40160A58E
:1074B00071A57170695C7F4F89819A81680F791F0E
:1074C000A7018B859C850E94A81A28CF80E001C067
:1074D00087E02E960FB6F894DEBF0FBECDBFDF91CA
:1074E000CF911F910F91FF90EF90DF90CF90BF90C1
:1074F000AF909F908F907F906F905F904F903F9054
:107500002F9008952F923F924F925F926F927F92A9
:107510008F929F92AF92BF92CF92DF92EF92FF92A3
:107520000F931F93CF93DF93CDB7DEB767970FB657
:10753000F894DEBF0FBECDBF4C017C876B871A016C
:107540003E872D87D9011D921C92BE016F5F7F4F30
:107550000E942918811146C2F40187A1811142C2FB
:1075600086A181FF3EC2E981FA818081843009F4DD
:1075700063C1D40198960C91989799961C9199970C
:107580009A962C919A979B963C91C101A0E0B0E00D
:10759000800F911FA21FB31F80179107A207B30787
:1075A00008F04AC118012094309446C1D40198963D
:1075B000FC9198979996EC9199979A96AC909A9796
:1075C0009B96BC909B979C96CC909C979D96DC90AC
:1075D0009D979E961C919E979F967C903E2F317012
:1075E0002F2F40E050E060E070E080E090E0A0E00D
:1075F0000E946D7409F0C6C13E2FA501B601812F0E
:10760000972D09E00E942A742B833C834D835E836F
:107610006F83788789879A8789819A81DC01199697
:10762000ED90FC901A97B1E0EB1AF1082B813C81A8
:10763000E222F322E114F10409F403C189819A8161
:10764000FC0103A914A925A936A9D401D4964D910A
:107650005D916D917C91D797041715072607370721
:1076600009F446C1E981FA81FC83EB83D401D09609
:107670004D915D916D917C91D397CF010E949A17A6
:10768000611571058105910509F410C12B013C01BB
:107690004E0C5F1C611C711C6101CD2CDD24C69455
:1076A000C114D10409F42AC1EB81FC818185928542
:1076B00096012E0D3F1D8217930718F46C01CE180A
:1076C000DF088601A30192016B857C85AB81BC81BB
:1076D00011968C910E941A158111F2C089819A81AC
:1076E000FC0143A954A965A976A94419550966095D
:1076F0007709860120E030E04017510762077307E1
:1077000078F4542F4427550F6B857C85640F751FC3
:1077100040E052E0C7960E94A81AE981FA811382DC
:107720008601102F0027110F201A310AAD85BE8562
:107730008D919C911197800F911F8D939C93EB8558
:10774000FC85E00FF11FFC87EB87980140E050E0DB
:1077500060E070E080E090E0D4019896AC9098975B
:107760009996BC9099979A96CC909A979B96DC9014
:107770009B979C96EC909C979D96FC909D979E96CF
:107780000C919E979F961C919F970E944674989685
:107790002C93989799963C9399979A964C939A978D
:1077A0009B965C939B979C966C939C979D967C93E1
:1077B0009D979E968C939E979F969C939F971A96C3
:1077C000BC91BB83F401F385FF87D4011C96BC9167
:1077D000B88BF401F585F98BD4011E96BC91BA8B58
:1077E000F401F785FB8BD4015096BC91BC8BF4015E
:1077F000F189FD8B29013A01B62FA72F8E8B9F8B24
:10780000AB80BF84C888D988EA88FB880C891F2F81
:107810000E94647430F425013601BE2DAF2D0E8B0D
:10782000FF8BF4014286538664867586B687A787E8
:10783000AE89A08BBF89B18B2114310409F0B6CE7B
:1078400027C02F2F3E2FA501B601812F972DA0E035
:107850000E946D7481F4D40116966D917D918D9185
:107860009C9119976115710581059105D1F440E04E
:1078700050E0BA0105C0F40140A951A962A973A959
:10788000C4010E941927611571058105910549F40C
:10789000D40196968C919697806496968C9380E00E
:1078A000A1C0613071058105910521F482E0F401E8
:1078B00087A398C06F3FFFEF7F078F079F0729F4CB
:1078C00081E0D40197968C938DC0F40160AB71ABCD
:1078D00082AB93AB0681178120853185012B022B6A
:1078E000032B09F0ABCE6683778380879187A6CE82
:1078F0000E940A1B882309F4B5CEE2CFD4019896E2
:107900002C91989799963C9199979A964C919A9721
:107910009B965C919B979C966C919C979D967C9175
:107920009D971A96AC901A971B96BC901B971C9625
:10793000CC901C971D96DC901D971E96EC901E9780
:107940001F96FC901F9750960C91509751961C9142
:1079500051979E968C919E979F969C910E946474DD
:1079600060F08B819C810E940A1B8111A9CFE98163
:10797000FA8143AA54AA65AA76AAF40144AA55AA90
:1079800066AA77AAD40198968D919C919997917047
:10799000E0E0F2E0E81BF90B8101E215F30508F4E1
:1079A0008F01D401D4964D915D916D917C91D797C3
:1079B00089819A810E945E1B811182CFF40180A58A
:1079C00091A59170C79629813A81A8016B857C8524
:1079D000820F931F0E94A81AE981FA8121E0238374
:1079E000A3CE87E067960FB6F894DEBF0FBECDBF7B
:1079F000DF91CF911F910F91FF90EF90DF90CF908B
:107A0000BF90AF909F908F907F906F905F904F90BE
:107A10003F902F900895CF92DF92EF92FF920F93B5
:107A20001F93CF93DF9300D0CDB7DEB7FC01228147
:107A3000338137FD31C08C01C480D5807901FFEFDF
:107A4000EF1AFF0AFC01E20FF31F66838CE3E816CE
:107A5000F104CCF09E012F5F3F4FA701B8016A5F90
:107A60007F4FF801808191810E94823A81E090E00D
:107A700029813A812E153F0511F480E090E0EE2433
:107A8000FF24E81AF90AF801F382E282FFEFCF1A25
:107A9000DF0AF801D582C4820F900F90DF91CF9159
:107AA0001F910F91FF90EF90DF90CF9008950F936B
:107AB0001F93CF93DF9300D0CDB7DEB7FC01428197
:107AC000538157FF03C08FEF9FEF18C08C01BC019B
:107AD0006A5F7F4F9E012F5F3F4FFC018081918144
:107AE0000E94823A8111EFCFF8012281338189818E
:107AF0009A812817390739F7848195810F900F9063
:107B0000DF91CF911F910F9108958F929F92AF9225
:107B1000BF92EF92FF920F931F93CF93DF93CDB756
:107B2000DEB7C654D1090FB6F894DEBF0FBECDBF85
:107B30007C01BE016B5B7F4F0E942918811125C11A
:107B4000D70196969C9196FF20C10E9482124B010C
:107B50005C0127968EAD9FAD2797FC012081D70150
:107B6000243009F0D0C015968C91833071F0F70164
:107B700040A951A962A973A90FEF1FEF9801C7018E
:107B80000E94AC24882339F000C1C7010E946E26F0
:107B90008111FBC0ECCFD7018D919C9111979A83F5
:107BA00089835A968D919D910D90BC91A02D8F83C4
:107BB0009887A987BA87F701068D178D20A131A173
:107BC0000E8300270B871C872D873E871F86188A08
:107BD000198A1A8A1F8A188E198E1A8E42A153A1E9
:107BE00064A175A125964CAF5DAF6EAF7FAF2597B1
:107BF000CE0101960E94C71D8111C7C0CE0101961A
:107C00000E942F2C8111C1C02796EEADFFAD2797A2
:107C1000A585B68514968C911497806214968C93E2
:107C200025853685D70115968C918160D90191966D
:107C30008C93D70116964D915D916D917C9119971A
:107C400085859685C4960E945117F7010285138594
:107C50002485358546855785608971892796EEADDF
:107C6000FFAD279785859685C8960E945717D7013F
:107C70001A960C911A971B961C911B971C962C9187
:107C80001C971D963C911D971E964C911E971F9612
:107C90005C911F9750966C91509751967C912796C6
:107CA000EEADFFAD27978585968588960E9457177C
:107CB0002796EEADFFAD279785859685B501A40182
:107CC0000C960E9451172796EEADFFAD2797A5851C
:107CD000B68555961C920584F685E02D108A118A8A
:107CE000128A138ACE0101960E94D42B81114DC0B5
:107CF00027968EAD9FAD27970E94642BF70196A122
:107D00009F7B96A342C0D8964D915D916D917C91D9
:107D1000DB970E945E1B811138C0F70104AD15ADE1
:107D2000D8011B968C911B9780621B968C932681A1
:107D3000378140855185B801808191810E94D01A98
:107D4000F7014285538564857585C8014C960E946C
:107D50005117B501A401C80146960E945117D801D8
:107D600052961C92529753961C9227968EAD9FADB9
:107D7000279721E0FC0123830E94642BD70196966C
:107D80009C9196979F7B96969C93CA5BDF4F0FB60C
:107D9000F894DEBF0FBECDBFDF91CF911F910F9141
:107DA000FF90EF90BF90AF909F908F9008950F93AA
:107DB0001F93CF93DF9300D0CDB7DEB78C010E9425
:107DC000853D81110BC0BE016F5F7F4FC8010E94CE
:107DD0002918811103C0F801118210820F900F90B1
:107DE000DF91CF911F910F9108952F923F924F9263
:107DF0005F926F927F928F929F92AF92BF92CF923B
:107E0000DF92EF92FF920F931F93CF93DF93CDB743
:107E1000DEB7A2970FB6F894DEBF0FBECDBF1C0130
:107E20000B871C872D873E874F87588B4B01BE01E0
:107E30006F5F7F4F0E94291881111CC3D101979653
:107E40008C91811117C3E981FA818081843041F0DE
:107E5000E981FA81FAA3E9A38081843089F42DC0F5
:107E6000D101D0964D915D916D917C91D3970FEF9B
:107E70001FEF9801C1010E94AC24882349F3FAC284
:107E80002B853C854D855E856F857889C4012F3FA4
:107E90003F4F4F4F5F4F610571058105910569F0B7
:107EA00060F0EFEFEB87FFEFFC870FEF0D871FEF21
:107EB0001E871F86188A812C912CD1011A964C900E
:107EC0001A971B965C901B971C966C901C971D969E
:107ED0007C901D971E96EC911E971F96FC911F9704
:107EE0005096BC91BD8BD1015196BC91BE8B2B8518
:107EF0003C854D855E856F857889C401520163019B
:107F00007F010D891B2F0E94647469F060F0D1011C
:107F100096968C9181FD07C04B865C866D867E8629
:107F2000EF87F88B4801F101F0A5FB83D101999609
:107F30004C9099979A965C909A979B966C909B9789
:107F40009C967C909C979D96BC91BD8BF101F6A56B
:107F5000FE8BF101B7A510A611A612A613A614A6B2
:107F600015A616A617A62B853C854D855E856F85C3
:107F70007889C401A0E00E946D7421F4412C512C39
:107F80003201FEC1E9A1FAA14185528560E070E0AD
:107F90008A019B0189E0000F111F221F331F8A9560
:107FA000D1F7098B1A8B2B8B3C8B2B81342D452DD4
:107FB000562D672D7D898E899B2FA0E00E946D74C0
:107FC00009F497C029893A894B895C8959016A016A
:107FD000E12CF12C87012B81342D452D562DAFEF4F
:107FE0000E944F742D8B3E8B4F8B588F2B013C0181
:107FF0002B853C854D855E856F857889C4010E94FF
:108000004F74AB82BC82CD82DE82EF82F886098714
:108010001A87E12CF12C00E010E00E94A973298F4F
:108020003A8F4B8F5C8F6D8F7E8F8F8F98A32D89AA
:108030003E894F89588DB201C3010E94A97359012D
:108040006A017B018C01298D3A8D4B8D5C8D6D8D84
:108050007E8D8F8D98A10E94647408F44AC00989AE
:108060001A892B893C890150110921093109A02E57
:10807000A094B12EB094C22EC094D32ED0943D893A
:10808000A3224E89B4225F89C522688DD622D101F0
:108090009896AC9298979996BC9299979A96CC920A
:1080A0009A979B96DC929B979C964C929C979D9658
:1080B0005C929D979E966C929E979F967C929F97BE
:1080C0002B853C854D855E856F857889C40172015D
:1080D00083010E945B742B873C874D875E876F8787
:1080E000788B4C01D0964D905D906D907C90D3979D
:1080F00032C0F1014680578060847184411451047C
:108100006104710419F540E050E0BA01C1010E9418
:1081100019272B013C01613071058105910529F476
:1081200082E0D10197968C93A5C16F3FBFEF7B078B
:108130008B079B0721F481E0F10187A39BC1D1014B
:1081400016966D937D938D939C931997F10140AA98
:1081500051AA62AA73AA411451046104710409F47A
:108160000DCF29893A894B895C8989019A0140E0C0
:1081700050E0BA010B831C832D833E834F835887C5
:1081800069877A872B853C854D855E856F857889E3
:10819000C401AB80BC80CD80DE80E12CF12C00E0FE
:1081A00010E00E94647409F008F4A5C02B853C859A
:1081B0004D855E856F857889C401AB80BC80CD809C
:1081C000DE80E12CF12C00E010E00E945B742B8734
:1081D0003C874D875E876F87788B4C019501A601A0
:1081E00060E070E080E090E0D1019896AC909897C4
:1081F0009996BC9099979A96CC909A979B96DC907A
:108200009B979C96EC909C979D96FC909D979E9634
:108210000C919E979F961C910E944674298B3D8BD2
:10822000B42FA52F698F7E8B8F8B9A8FF10120A79A
:1082300031A742A753A764A775A786A797A7F6A15A
:10824000F88FF1FF27C0F101A284B384C484D584E0
:10825000E684F784008911895A2F0E94647471F0B2
:1082600068F022873387B487A58766877787808BF6
:10827000918BE88DE064D1019696EC93B301A20155
:10828000C1010E9419272B013C01672B682B692B28
:1082900041F429C0B301A201C1010E941E1C2B019F
:1082A0003C01BFEF4B165B066B067B0609F443CF20
:1082B000E2E04E1651046104710408F431CFE98103
:1082C000FA818789908DA18DB28D481659066A066C
:1082D0007B0608F025CFD101D0964D925D926D922C
:1082E0007C92D3974FCF1B861C861D861E861F86C9
:1082F000188A812C912C2B853C854D855E856F8558
:108300007889C401F101A0A4B1A4C2A4D3A4E4A4B7
:10831000F5A406A517A50E94467420A731A742A779
:1083200053A764A775A786A797A72B853C853170AF
:1083300040E050E060E070E080E090E0A0E00E946B
:108340006D7409F41BCEB301A20189819A810E9448
:108350009A176B017C01672B682B692B09F4E0CE1F
:108360002B853C854D855E856F857889C40109E044
:108370000E942A7429013A014C0C5D1C6E1C7F1C62
:10838000D1019896FC9198979996EC9199979A9625
:10839000BC91BB83D1019B96BC91BB87D1019C96BC
:1083A0008C909C979D969C909D979E96BC91BC8727
:1083B000D1019F96BC91BD87D1011A96AC901A97B6
:1083C0001B96BC901B971C96CC901C971D96DC901E
:1083D0001D971E96EC901E971F96FC901F97509627
:1083E0000C91509751961C9151972F2F3E2F4B81F6
:1083F0005B85B4018C859D850E946474F9F0F0F072
:108400001A96FC931A971B96EC931B971C964C9309
:108410001C971D965C931D971E968C921E971F9617
:108420009C921F9750968C93509751969C9351977E
:1084300096968C919697806496968C933E2F317089
:108440002F2F40E050E060E070E080E090E0A0E09E
:108450000E946D7471F0F10184A995A9A6A9B7A92C
:10846000481659066A067B0621F044AA55AA66AA50
:1084700077AA80E0A2960FB6F894DEBF0FBECDBFFC
:10848000DF91CF911F910F91FF90EF90DF90CF90F0
:10849000BF90AF909F908F907F906F905F904F9024
:1084A0003F902F9008950F931F93CF93DF9300D0A9
:1084B00000D0CDB7DEB77C836B83009709F467C02B
:1084C0008C0140E0BE016F5F7F4FCE0103960E949A
:1084D000FB1E811158C089819A81F80191838083A4
:1084E0006B817C81C8010E94C132811156C0F801A4
:1084F00087AD87FD38C0848184FF44C029813A81DB
:10850000F9018081F801843029F586819781A08561
:10851000B185828F938FA48FB58F428553856485F3
:10852000758544278581482B468F578F60A371A39B
:10853000D801A05CBF4F8D919D910D90BC91A02D55
:1085400082A393A3A4A3B5A3B801C9010D960E9469
:10855000DD1A09C062A973A90E94B31AF8016683E3
:10856000778380879187E981FA8185819681F801F7
:108570009383828340E050E0BA01C8010E94C71D86
:10858000843039F485E0F8011182108209C089E055
:1085900007C08111F8CF80E003C08430A1F7F2CF8B
:1085A0000F900F900F900F90DF91CF911F910F912F
:1085B00008950F931F93CF93DF9300D0CDB7DEB70D
:1085C0008C01BE016F5F7F4F0E942918811103C08B
:1085D000F801118210820F900F90DF91CF911F91BF
:1085E0000F910895CF92DF92EF92FF921F93CF9356
:1085F000DF9300D0CDB7DEB77C016B01BE016F5FAA
:108600007F4F0E942918182F81111EC0C114D10458
:1086100039F440E050E0BA01C7010E94C71D13C001
:1086200060E070E0C7010E94DF2C982F9B7F59F417
:10863000B601C7010E94751860E070E0C7010E9492
:10864000C329843009F0182F812F0F900F90DF91EC
:10865000CF911F91FF90EF90DF90CF900895EF9210
:10866000FF921F93CF93DF93CDB7DEB7C654D109E6
:108670000FB6F894DEBF0FBECDBF27969FAF8EAF6B
:1086800027977B0140E0BE016F5F7F4FCE018B5B80
:108690009F4F0E94FB1E182F81111AC027966EADA6
:1086A0007FAD2797CE0101960E94C132182F81110C
:1086B0000FC021968FAD219787FD09C0E114F10409
:1086C00039F0B701CE0101960E94751801C016E07D
:1086D000812FCA5BDF4F0FB6F894DEBF0FBECDBF50
:1086E000DF91CF911F91FF90EF9008952F923F92CD
:1086F0004F925F926F927F928F929F92AF92BF92B2
:10870000CF92DF92EF92FF920F931F93CF93DF935D
:10871000CDB7DEB7E1970FB6F894DEBF0FBECDBF81
:108720009AA789A77DA76CA78A0140E0BE01695D71
:108730007F4FCE0189960E94FB1E8BA781111BC122
:10874000EFA1F8A5D801ED93FC9383899489A589BD
:10875000B6894788508C618C728C5301420122E0AB
:10876000821A9108A108B10888169906AA06BB06C4
:1087700038F0ECA5FDA580839183A283B383FBC071
:1087800080818130B9F5FA83E98342E0442E512C8F
:10879000612C712CC12CD12C7601B301A201CE0128
:1087A00001960E941E1C6F3FFFEF7F078F079F07F8
:1087B00009F4CBC0613071058105910509F4C7C08A
:1087C000672B682B692B29F42FEFC21AD20AE20A11
:1087D000F20A8FEF481A580A680A780AEFA1F8A53A
:1087E0008789908DA18DB28D481659066A067B0641
:1087F000A0F2B1C0843009F04FC047A550A961A9CB
:1088000072A900E010E0C12CD12C760138E0232EB3
:10881000312C0115110579F42A013B019FEF491A0A
:10882000590A690A790A8FA198A50E945E1B8111D5
:1088300091C0B301A201EFA1F8A5E00FF11FE7A9D4
:1088400024013501C10188199909411451046104B9
:108850007104A9F0E0FD05C0AFEFCA1ADA0AEA0A0E
:10886000FA0AE695B1E04B1A5108610871089C01BB
:10887000240D351D232B49F75301420103C0812CE0
:10888000912C54010F5F1F4F117081149104A104AA
:10889000B10409F0BECF5FC083A094A0A5A0B6A08C
:1088A00000E010E0C12CD12C760101151105A9F4CE
:1088B000D501C4010196A11DB11D8EA79FA7A8AB2C
:1088C000B9ABB501A4018FA198A50E945E1B8111CF
:1088D00041C08EA49FA4A8A8B9A8EFA1F8A5608163
:1088E000C801C7966230B1F4DF01A80FB91F119615
:1088F0008C9190E0982F8827E00FF11F67A9862BB5
:10890000892B29F49FEFC91AD90AE90AF90A0E5FDF
:108910001F4F12C08E0F9F1F0E940D17DC01CB014D
:10892000BF70892B8A2B8B2B29F4AFEFCA1ADA0A76
:10893000EA0AFA0A0C5F1F4F1170B1E04B1A510896
:108940006108710809F0B1CF06C021E001C022E042
:108950002BA701C08BA7ACA5BDA5CD92DD92ED9252
:10896000FC921397EFA1F8A5C38AD48AE58AF68A08
:108970008481816084838BA5E1960FB6F894DEBF75
:108980000FBECDBFDF91CF911F910F91FF90EF9060
:10899000DF90CF90BF90AF909F908F907F906F901F
:1089A0005F904F903F902F9008952F923F924F925B
:1089B0005F926F927F928F929F92AF92BF92CF926F
:1089C000DF92EF92FF920F931F93CF93DF9300D02C
:1089D0001F92CDB7DEB74C01BE016F5F7F4F0E9483
:1089E0002918811185C0F40177A071107CC086A17F
:1089F00081FF7BC030A441A452A463A4B4A5A5A563
:108A000026A4F7A5FB83F401A284B384C484D5848F
:108A1000E684F78400891189232D342D452D562DA8
:108A20006B2F7A2F822D9B810E94647408F05FC0A7
:108A3000A0E00E946D7489F446815781608571853C
:108A400000E010E09801C4010E942925782EF4016D
:108A500016821782108611862FC0F40140A951A9F1
:108A600062A973A9C4010E941E1CAB01BC014F3F47
:108A7000FFEF5F076F077F0741F041305105610548
:108A8000710531F482E0782E17C07724739414C0F6
:108A9000E981FA818789908DA18DB28D4817590798
:108AA0006A077B0748F4F40100A911A922A933A998
:108AB000C4010E942925782EF40180A5828781A512
:108AC000838782A5848783A5858784A5868785A5D6
:108AD000878786A5808B87A5818B86A1806486A3E6
:108AE000772029F077A2872D03C087E001C080E0BE
:108AF0000F900F900F90DF91CF911F910F91FF90EA
:108B0000EF90DF90CF90BF90AF909F908F907F902D
:108B10006F905F904F903F902F900895CF92DF928B
:108B2000EF92FF920F931F93CF93DF93CDB7DEB7F2
:108B3000C25BD1090FB6F894DEBF0FBECDBFCF54D4
:108B4000DF4F99838883C15BD04042E0BE0161550D
:108B50007F4FCE018F549F4F0E94FB1E8111CEC0CC
:108B6000C155DF4F88819981CF5AD04027969FAF5A
:108B70008EAF2797CF54DF4F68817981C15BD0409A
:108B8000CE018B5B9F4F0E94C1328111B7C0CC5781
:108B9000DF4F8881C458D04087FD06C02A968FAD2C
:108BA0002A9780FD88C002C086E0A8C0C155DF4F6B
:108BB000E881F981CF5AD040C757DF4FF983E88366
:108BC000C958D0408081843081F4BE0167577F4FFF
:108BD000CF010D960E94DD1AC157DF4FC880D980A2
:108BE000EA80FB80CF58D04008C0E9966EAD7FADDB
:108BF000E9970E94B31A6B017C012A968FAD2A97E0
:108C000084FF5BC0C155DF4FE881F981CF5AD04066
:108C1000FA83E983CF82D886E986FA868081843018
:108C2000B1F5CD56DF4F8881C359D0408B87CC56E4
:108C3000DF4F8881C459D0408C87CB56DF4F888165
:108C4000C559D0408D87CA56DF4F8881C659D0405C
:108C50008E87C956DF4F8881C759D0408F87C85645
:108C6000DF4F8881C859D040888BC756DF4F888135
:108C7000C959D040898BC656DF4F8881CA59D04028
:108C80008A8BC257DF4F8881CE58D0408E8340E018
:108C900050E0BA01CE0101960E94C71D81112EC07D
:108CA00060E070E0CE0101960E94DF2C882319F06D
:108CB000843019F023C087E021C0CE018B5B9F4F29
:108CC0000E94062B81111AC0C114D104E104F104E1
:108CD00049F4C155DF4F88819981CF5AD0400E9415
:108CE000642B0CC000E010E09801B701A601CE0192
:108CF00087579F4F0E942925882359F3CE54DF4F71
:108D00000FB6F894DEBF0FBECDBFDF91CF911F919C
:108D10000F91FF90EF90DF90CF9008954F925F9268
:108D20006F927F928F929F92AF92BF92FF920F931A
:108D30001F93CF93DF93CDB7DEB7CE56D1090FB6D1
:108D4000F894DEBF0FBECDBFAF969FAF8EAFAF978B
:108D500042E0BE0165597F4FCE0183599F4F0E946B
:108D6000FB1EF82E81112FC1AD968EAD9FADAD9734
:108D70009A838983AF966EAD7FADAF97CE01019692
:108D80000E94C132882309F41AC1843009F01AC143
:108D9000AD968EAD9FADAD9727969FAF8EAF2797BF
:108DA00040E050E0BA01CE018B5B9F4F0E94192733
:108DB0004B015C01672B682B692B79F081E08816E9
:108DC0009104A104B10461F0EFEF8E169E06AE0689
:108DD000BE0641F4FF24F39405C047E0F42E02C020
:108DE00032E0F32E0E9482122B013C01F110DCC014
:108DF000B501A401AD968EAD9FADAD970E94AD2695
:108E0000F82E8111D1C0AD968EAD9FADAD97FC010E
:108E10002081243009F447C04BE050E060E270E06C
:108E2000C7960E948217AD968EAD9FADAD971EE29C
:108E3000FC0117ABEE5BFF4F20E12083B301A201E1
:108E4000835B9F4F0E945117AD968EAD9FADAD973E
:108E5000BC01695C7F4FA50194010E94D01AAD96B8
:108E60008EAD9FADAD97BC01695C7F4F40E250E095
:108E7000895A9F4F0E94A81AAD968EAD9FADAD97AF
:108E8000FC01E85AFF4F10832F81388549855A85A8
:108E9000BC01695A7F4F0E94D01AAD96EEADFFAD6E
:108EA000AD9781E08383CE0101960E94B22FF82E08
:108EB00081117AC0AD96EEADFFADAD978081843063
:108EC00009F050C085859685B301A2010C960E94D9
:108ED0005117AD96EEADFFADAD9785859685B50181
:108EE000A401C4960E945117AD96EEADFFADAD97AB
:108EF0004185528560E070E099E0440F551F661F80
:108F0000771F9A95D1F785859685C8960E94511747
:108F1000AD96EEADFFADAD974185528560E070E056
:108F200029E0440F551F661F771F2A95D1F78585C5
:108F3000968588960E945117AD96EEADFFADAD9720
:108F4000A585B68583E091968C930584F685E02D02
:108F500080E18483CE0101960E94D42BF82E8111EA
:108F600032C01BC08BA99CA9B301A20146960E94E6
:108F700051176BA97CA9A5019401AD968EAD9FAD4B
:108F8000AD970E94D01AEBA9FCA980E18387AD962A
:108F9000EEADFFADAD9781E08383AD968EAD9FAD15
:108FA000AD970E94642B0EC000E010E09801B5015F
:108FB000A401CE018B5B9F4F0E94292504C088E04D
:108FC000F82E01C0F82E8F2DC259DF4F0FB6F8943E
:108FD000DEBF0FBECDBFDF91CF911F910F91FF90EC
:108FE000BF90AF909F908F907F906F905F904F90C9
:108FF0000895DF92EF92FF920F931F93CF93DF9329
:10900000CDB7DEB7CE5CD1090FB6F894DEBF0FBE88
:10901000CDBFC553DF4F99838883CB5CD040C3530A
:10902000DF4F79836883CD5CD040CE0183539F4F5F
:109030000E94021842E0BE0167537F4FCE01855364
:109040009F4F0E94FB1E81117BC1C753DF4F888158
:109050009981C95CD04027969FAF8EAF2797C553A3
:10906000DF4F68817981CB5CD040CE018B5B9F4F15
:109070000E94C132811164C1CC57DF4F8881C4582E
:10908000D040807A09F057C1C753DF4FE881F9819A
:10909000C95CD0408081843009F08CC065857685BC
:1090A00040E450E0CE0187579F4F0E94A81A44E445
:1090B00050E0BE016B5B7F4FCE0101960E94A81A63
:1090C000C353DF4F68817981CD5CD040CE010196DA
:1090D0000E94C132811121C04F81588569857A85EE
:1090E0002F968CAD9DADAEADBFAD2F9748175907EC
:1090F0006A077B0709F021C14FA158A569A57AA588
:10910000AF968CAD9DADAEADBFADAF9748175907CB
:109110006A077B0709F011C103C0843009F010C150
:10912000CE0101960E94B22F81110AC1C753DF4FB1
:10913000E881F981C95CD0400584F685E02DE180A5
:10914000F3A005A110E0102F002784A1082B40E414
:1091500050E0BE0167577F4FCF010E94A81AC75346
:10916000DF4FE881F981C95CD0400584F685E02DA8
:10917000E182C753DF4FE881F981C95CD040A58502
:10918000B6859396FC92A585B68594960C93949794
:1091900095961C930584F685E02D848184FD02C09C
:1091A00080628483CE0101960E94D42B882309F427
:1091B000B2C0C6C0E9966EAD7FADE99740E250E01F
:1091C000CE0187579F4F0E94A81A44E450E0BE0189
:1091D0006B5B7F4FCE0101960E94A81AC353DF4FED
:1091E00068817981CD5CD040CE0101960E94C13268
:1091F000811121C04F81588569857A852F968CAD64
:109200009DADAEADBFAD2F97481759076A077B07D5
:1092100009F093C04FA158A569A57AA5AF968CAD6A
:109220009DADAEADBFADAF97481759076A077B0735
:1092300009F083C003C0843009F082C0CE010196DA
:109240000E94B22F81117CC00BA91CA969E870E0B3
:109250006C0F7D1F635F7F4F43E150E0C8010D96A7
:109260000E94A81ACC56DF4F8881C459D04084FF91
:109270008062F8018387C753DF4FE880F980C95CBB
:10928000D040DD24D394F701D382F801838584FF95
:1092900042C02F964CAD5DAD6EAD7FAD2F978F81E7
:1092A0009885A985BA85481759076A077B0799F1F8
:1092B000B801F70180810E94B31AAB01BC01C7015C
:1092C0000E949A17AB01BC0141155105610571055A
:1092D000B1F1C7010E945E1BC753DF4FE881F981DE
:1092E000C95CD04081112CC0DF01A85ABF4F8C91BE
:1092F0008E3289F42F81388549855A85BF01695A94
:109300007F4FCF010E94D01AC753DF4FE881F98108
:10931000C95CD040D382CE018B5B9F4F0E94062B4D
:1093200081110EC0C753DF4F88819981C95CD0403D
:109330000E94642B05C086E003C088E001C082E083
:10934000C253DF4F0FB6F894DEBF0FBECDBFDF9123
:10935000CF911F910F91FF90EF90DF9008952F9282
:109360003F924F925F927F928F929F92AF92BF9265
:10937000CF92DF92EF92FF920F931F93CF93DF93E1
:10938000CDB7DEB7C854D1090FB6F894DEBF0FBE13
:10939000CDBF29969FAF8EAF29977B014A0140E050
:1093A000BE016B5B7F4FCE01895B9F4F0E94FB1E0E
:1093B000782E8111C1C0E114F10409F48AC0279606
:1093C0008EAD9FAD27979A8389831F821886198651
:1093D0001A8640E050E0BA01CE0101960E94C71DF6
:1093E000811173C061E070E0CE0101960E94DF2C14
:1093F00081116BC02796EEADFFAD27978081843039
:1094000009F04DC0C12CD12C00E010E0A12CB12CF2
:10941000EBA9FCA9818190E0A816B906C0F52FEF51
:10942000A21AB20AC501880F991FE80FF91F4181DE
:1094300050E0542F44278081482BC114D10429F4D3
:10944000CA01985D81159840F0F060E070E0C601B7
:10945000A0E0B0E0DC01992788271A012B01282A17
:10946000392A4A2A5B2AC201B10124E030E0A7016F
:10947000400F511F0E94531890E0009731F0080FE1
:10948000191F40E050E06A01C3CF00E010E0CD2892
:1094900011F000E010E0F701E00FF11F19C08BA9F7
:1094A0009CA9F7013B96A701DC012D91CD01DA01C2
:1094B0002D93AD01AE17BF07B9F71082EE15FF056A
:1094C00041F082918032C9F304C08430A1F5F701E4
:1094D00010828114910481F127968EAD9FAD27975C
:1094E000DC015F964D915D916D917C9192970E9408
:1094F0005E1B782E811120C027968EAD9FAD2797D9
:10950000FC012081233029F0243031F027E230E0C3
:1095100005C023E430E002C024E630E0295C3F4F80
:10952000820F931F0E940D17D4016D937D938D932D
:109530009C93139701C0782E872DC85BDF4F0FB621
:10954000F894DEBF0FBECDBFDF91CF911F910F9179
:10955000FF90EF90DF90CF90BF90AF909F908F9053
:109560007F905F904F903F902F9008958F929F92A1
:10957000AF92BF92EF92FF920F931F93CF93DF931F
:10958000CDB7DEB7CE55D1090FB6F894DEBF0FBE0A
:10959000CDBF6F969FAF8EAF6F9742E0BE01655A09
:1095A0007F4FCE01835A9F4F0E94FB1E81112AC11B
:1095B0006D96EEADFFAD6D9780819E012B5B3F4FA9
:1095C0007901843009F045C046E150E060E070E088
:1095D000C9010E94821700E010E06F96EEADFFAD6A
:1095E0006F978081803208F476C0CE01835A9F4FF6
:1095F0000E944C1A6115710531E083079105C0F096
:109600006F3FEFEF7E078E079E0711F486E0FAC0EA
:109610000A301105D8F74C01AA24BB24F801EE0F3B
:10962000FF1FEE0DFF1D808291820F5F1F4F05C04F
:10963000611571058105910549F3AB01EFE8F1E092
:109640002191222309F4B7C030E024173507C1F770
:10965000DDCF4BE050E060E270E0C9010E9482176C
:1096600000E010E06F96EEADFFAD6F978081803225
:10967000F8F0CE01835A9F4F0E944C1A6115710574
:10968000F1E08F07910510F60E94D14E41E653E0BC
:109690000E94894E009709F4B9CFE8E8F1E02191E2
:1096A000222309F496C030E028173907C1F7AECF5E
:1096B000F7018081853E09F4A9CFE00FF11F8F01EA
:1096C0000E191F09EE15FF0521F082918032B9F3C2
:1096D00002C000E010E06D968EAD9FAD6D979A834D
:1096E00089831F82188619861A8640E050E0BA01E5
:1096F000CE0101960E94C71D811184C061E070E017
:10970000CE0101960E94DF2C811115C06D96EEAD41
:10971000FFAD6D9720818BA99CA9243011F4FC0129
:109720002DC0012B21F04BE050E0B70136C025EEF3
:10973000FC01208334C0843009F064C00115110598
:10974000C1F161E070E0CE0101960E94B82A81115A
:1097500059C040E250E060E070E08BA99CA90E94F3
:1097600082176D96EEADFFAD6D978081EBA9FCA9D8
:10977000843061F483E88083EBA9FCA901838BA981
:109780009CA946E150E0B701029607C088E08387B4
:109790004BE050E0B7018BA99CA90E94A81A6D96D6
:1097A0008EAD9FAD6D9721E0FC0123830E94642B59
:1097B00029C080E027C00B30110508F027CFF80141
:1097C000EE0FFF1FEE0DFF1D608371830F5F1F4FB4
:1097D00004CF8F3F910591F088F00A30110508F011
:1097E00015CFF701E00FF11F90830F5F1F4FF701B7
:1097F000E00FF11F80830F5F1F4F34CF0B30110537
:10980000B0F304CFC25ADF4F0FB6F894DEBF0FBEDD
:10981000CDBFDF91CF911F910F91FF90EF90BF903F
:10982000AF909F908F9008958F929F92AF92BF922A
:10983000CF92DF92EF92FF920F931F93CF93DF931C
:1098400000D000D000D0CDB7DEB77C014A015B016B
:1098500081E0A81AB1088701C12CD12CCA14DB04FD
:10986000D4F49E012B5F3F4F41E050E0BE016F5F9B
:109870007F4FC4010E94AC388D819E81019759F4BD
:1098800089810F5F1F4FF801319780839FEFC91ABD
:10989000D90A8A3019F7F8011082CD2811F0C701D2
:1098A00002C080E090E026960FB6F894DEBF0FBEAF
:1098B000CDBFDF91CF911F910F91FF90EF90DF907F
:1098C000CF90BF90AF909F908F900895EF92FF92AE
:1098D0001F93CF93DF93CDB7DEB7C654D1090FB630
:1098E000F894DEBF0FBECDBF182F7B0146E450E0D9
:1098F00060E070E0CE0101960E948217FA82E98250
:10990000612FCE0101960E940B3DCE0101960E946F
:10991000573DCA5BDF4F0FB6F894DEBF0FBECDBF19
:10992000DF91CF911F91FF90EF900895EF92FF92FA
:109930000F931F93CF93DF93CDB7DEB7C654D109F2
:109940000FB6F894DEBF0FBECDBF7C018B0146E49D
:1099500050E060E070E0CE0101960E9482171A8309
:1099600009838701F80161918F01CE010196662379
:1099700019F00E940B3DF6CF0E94573DCA5BDF4FA6
:109980000FB6F894DEBF0FBECDBFDF91CF911F9110
:109990000F91FF90EF9008952F923F924F925F9218
:1099A0006F927F928F929F92AF92BF92CF92DF92EF
:1099B000EF92FF920F931F93CF93DF93CDB7DEB754
:1099C000CC56D1090FB6F894DEBF0FBECDBFCD5730
:1099D000DF4FE880F980C358D04046E450E060E0B3
:1099E00070E0CE0101960E948217CF57DF4F888129
:1099F0009981C158D0409A8389836E0125E8C20EAF
:109A0000D11C1E0187E4280E311CD7016C916623FE
:109A100009F461C1653221F0BFEFEB1AFB0AACC05B
:109A2000F7011181103331F43396D70112961C914E
:109A300001E00BC0F7011D3219F0329600E005C0BD
:109A40003396D70112961C9102E01A3219F0812C3C
:109A5000912C0CC0D6018D909C907F01BFEFEB1A2A
:109A6000FB0A1081F60132966F0114C07F0180ED70
:109A7000810F8A3078F43AE0432E489CC001499C1B
:109A8000900D11244C01810E911C20E3821A910843
:109A90001191ECCF812F8F7D8C3431F40460D7018C
:109AA0001C91F70131967F01112309F414C18FE94C
:109AB000810F8A3118F420EE210F01C0212F2F349D
:109AC000E9F050F4233409F449C0243409F45CC0AB
:109AD000223409F457C04FC0253509F455C0283544
:109AE00009F447C0233509F046C05601F2E0AF0E35
:109AF000B11CD6016D907C90F30102C038E045C0E6
:109B0000CF018619970921912111FACF6C0101FD2E
:109B10000EC06C01BFEFCB1ADB0A8815990538F42B
:109B200060E2CE0101960E940B3DC601F2CFF30127
:109B300061913F01662369F0CE0101960E940B3DC1
:109B4000F6CF60E2CE0101960E940B3DFFEFCF1AE7
:109B5000DF0AC814D904A8F3650157CF560122E0E3
:109B6000A20EB11CD6016C91CE0101960E940B3D54
:109B7000F3CF30E10AC0612FCE0101960E940B3D68
:109B80005601EACF32E001C03AE002FF0CC05601B4
:109B9000B4E0AB0EB11CF6016081718182819381CA
:109BA000243401F515C0C60102965C01243449F441
:109BB000D6018D919C91BC01882777FD8095982FC7
:109BC00007C0F60180819181BC0180E090E00AC06D
:109BD00097FF08C090958095709561957F4F8F4F46
:109BE0009F4F0860A9963FAE2EAEA997C12CD12CED
:109BF000432E512C612C712CAD964CAE5DAE6EAEE9
:109C00007FAEAD97AD962CAD3DAD4EAD5FADAD9792
:109C10000E9485732B013C01E62FCA01B901AAE01D
:109C20004A1651046104710430F0183711F0E7E06E
:109C300001C0E7E2E40DBFEFCB1ADB0AE05DA996B5
:109C4000AEADBFADA997ED93A996BFAFAEAFA99743
:109C5000232B242B252B21F0B0E2CB16D10491F637
:109C600003FF09C0F101EC0DFD1D2DE2422E4082E3
:109C7000C60101966C0100FD03C090E2792E02C07E
:109C800080E3782E01FD0EC0C6018C010F5F1F4FCF
:109C90008815990540F4672DCE0101960E940B3D71
:109CA000C801F3CF8601C20CD31CD6016E916D01A1
:109CB000CE0101960E940B3DC214D304B1F70815E2
:109CC000190508F049CF672DCE0101960E940B3D82
:109CD0000F5F1F4FF4CFCE0101960E94573DC4592C
:109CE000DF4F0FB6F894DEBF0FBECDBFDF91CF912F
:109CF0001F910F91FF90EF90DF90CF90BF90AF90AA
:109D00009F908F907F906F905F904F903F902F909B
:109D10000895CF92DF92EF92FF926038710581052E
:109D2000910510F4CB0123C06115710521E0820774
:109D30009105D8F441365340C1F4E5EDF4E020E05C
:109D400030E0C190D190E12CF12C6C157D058E0591
:109D50009F0529F02F5F3F4F2038310591F7B9015A
:109D600060587F4FCB01992702C080E090E0FF90C0
:109D7000EF90DF90CF9008958038910588F061369C
:109D8000734061F48F3F910509F040F4880F991FEB
:109D9000FC01EB52FC4F80819181089580E090E0BE
:109DA0000895CF93DF936115710521E08207910536
:109DB00008F058C0EB01611570418105910518F05C
:109DC000A7E2B2E002C0A3EEB2E04D915C91119720
:109DD0004115510509F443C0C417D50708F43FC025
:109DE0001496FD01329720813181E32FFF2733271D
:109DF000B901640F751FC617D70748F5E930F1059B
:109E000070F5EB5AFF4F0C940674CE01841B950B32
:109E1000880F991FA80FB91FCD91DC9120C09E011A
:109E2000241B350B21703327C21BD30B18C060973E
:109E300016C0A09714C0E09712C06A9710C0289669
:109E40000EC0C055D1090BC0C056DC4108C0EF2B75
:109E500009F0BBCF220F331FA20FB31FB6CFBE0135
:109E600080E090E0DF91CF9108958F929F92AF9222
:109E7000BF92CF92DF92EF92FF920F931F939B01BD
:109E8000AC018FB7F894C0903417D0903517E0909C
:109E90003617F09037178FBFA3E1B0E00E945A73D6
:109EA0002FB7F8948090341790903517A0903617FC
:109EB000B09037172FBF950184010C191D092E0989
:109EC0003F09061717072807390750F31F910F910D
:109ED000FF90EF90DF90CF90BF90AF909F908F90CA
:109EE000089581B1877E81B9149A039B5EC004995D
:109EF0005CC080E00E94CC0868EC70E080E090E0FC
:109F00000E94354F8FE192E09F938F930E94AC7631
:109F10008BE296E00E94C07664E670E080E090E01C
:109F20000E94354F8CE396E00E94C07664E670E0B4
:109F300080E090E00E94354F85E596E00E94C07673
:109F400064E670E080E090E00E94354F8CE696E099
:109F50000E94C07664E670E080E090E00E94354F99
:109F600085E896E00E94C07664E670E080E090E0CC
:109F70000E94354F85E996E00E94C07664E670E065
:109F800080E090E00E94354F89EA96E00E94C0761A
:109F900064E670E080E090E00E94354F0B9A1398E1
:109FA00081E08093E10B0F900F9008958091E10B79
:109FB00008958FB7F89440913417509135176091F8
:109FC0003617709137178FBF2FB7F89480913417D9
:109FD00090913517A0913617B09137172FBF841B7A
:109FE000950BA60BB70B8C369740A105B10560F316
:109FF00008950D9880B185FB882780F90895159AFA
:10A00000089515980895809102010895CF93DF93E4
:10A01000CDB7DEB72C970FB6F894DEBF0FBECDBF1D
:10A020008091000C90E08C599F4F98878F8380918E
:10A03000111881508E83809110188C8380912A187A
:10A040008B8380914D178A838091251789838FEFA9
:10A050009FEF9C878B87CE0101960E94056C2FB7DE
:10A06000F89460936F1770937017809371179093A3
:10A0700072172FBF81E08093010C2C960FB6F894D5
:10A08000DEBF0FBECDBFDF91CF9108958091020159
:10A0900081110C94FF4F0C9401509F938F938091EA
:10A0A0007417909175170E969F938F930E94577611
:10A0B0000F900F900F900F900895CF939093751776
:10A0C0008093741780E8EDEEFCE1DF01982F1D927C
:10A0D0009A95E9F7EDE6FDE1DF011D928A95E9F732
:10A0E00010924717109248171092491710924A176A
:10A0F00010925E1710925F171092601710926117FE
:10A1000010923B1710923C1710923D1710923E1779
:10A110001092010C0E94F94F882359F1C1E0C093BD
:10A12000E30B0D9A8091731781508230E8F481E03F
:10A130000E94CC080E94D94F81E792E00E944D50C6
:10A140000E94D94F81E00E944E090E94D94F86E5B6
:10A1500092E00E944D5082E292E00E944D50C093E6
:10A160000201CF910C94FF4F10920201CF910C94F9
:10A1700001501092E30B10920201CF9108958033A9
:10A1800050F08A3310F4805308959FEB980F963067
:10A1900010F48753089580E008952F923F924F92D4
:10A1A0005F926F927F928F929F92AF92BF92CF9267
:10A1B000DF92EF92FF920F931F93CF93DF93CDB770
:10A1C000DEB76F970FB6F894DEBF0FBECDBF082F76
:10A1D00080913F17813071F48DE69DE19F938F93BD
:10A1E0008EEA96E09F938F930E94AC760F900F902B
:10A1F0000F900F9080913F17823031F4602F70E004
:10A200008DE69DE10E94936A053008F4E0C210E0FB
:10A21000680124E0C21AD108F601E359F24E8081A8
:10A220008A3209F0D4C20359124EF8013397808163
:10A230000E94BF5030E1839F70011124F8013297D2
:10A2400080810E94BF50F701E80FF11DCF0141E06E
:10A25000242F30E02C153D053CF4F901E359F24E72
:10A26000208182274F5FF4CF892B09F0B0C263EBC6
:10A2700076E08DE69DE10E94F775892B09F4D4C143
:10A280006CE270E08DE69DE10E94E1756CE270E0A9
:10A2900001960E94E175FC0181818D8B82818E8BFC
:10A2A0001F8A83818A8B84818B8B1C8A86818E8313
:10A2B00087818F8380858887818589871A866CE26C
:10A2C00070E0CF0101960E94E175FC01F181F88FE9
:10A2D0006CE270E001960E94E175FC0181818B8740
:10A2E00082818C8783818D871E8684818F8785817B
:10A2F000888B198A8781898380858A8381858B836E
:10A3000082858C831D826CE270E0CF0101960E94F1
:10A31000E175FC01F181F98F6CE270E001960E9419
:10A32000E17501969B8F8A8F0E94D7748150863089
:10A3300020F481E08093B31A02C01092B31A809186
:10A34000B31A882309F470C1CE0145960E94D774D0
:10A350008C0190934C1780934B17CE0142960E942C
:10A36000D7749D8F8C8F90939F1A80939E1ACE01E5
:10A3700006960E94D774BC01882777FD8095982F98
:10A380000E94527220E030E44CE156E40E94AF712A
:10A3900020E030E040E752E40E94DE722B013C01F5
:10A3A0006093621770936317809364179093651797
:10A3B000CE010B960E94D7741C0190935D17809379
:10A3C0005C17CE010F960E94D7749F8F8E8F90934B
:10A3D0005B1780935A17CE0101960E94D774BC0177
:10A3E000882777FD8095982F0E94527220E030E4F4
:10A3F0004CE156E40E94AF7120E030E040E752E4C7
:10A400000E94DE724B015C016093521770935317E8
:10A410008093541790935517B801882777FD80953E
:10A42000982F0E9452726B017C012C8D3D8DB901D9
:10A43000882777FD8095982F0E94527220E030E0A7
:10A4400040E752E40E94AF719B01AC01C701B60125
:10A450000E9443716B017C0120E030E041E655E44D
:10A46000C301B2010E94AF719B01AC01C701B601EB
:10A470000E94437160936717709368178093691700
:10A4800090936A17B101882777FD8095982F0E94D5
:10A4900052722B013C01EE8DFF8DBF01882777FDA5
:10A4A0008095982F0E94527220E030E040E752E4FD
:10A4B0000E94AF719B01AC01C301B2010E944371C4
:10A4C0002B013C0120E030E041E655E4C501B40138
:10A4D0000E94AF719B01AC01C301B2010E944371A4
:10A4E00060936B1770936C1780936D1790936E1732
:10A4F0006CE270E08A8D9B8D0E94E1758C010F5F8C
:10A500001F4FC8010E94D7748093A01A6CE270E0BC
:10A51000C8010E94E1758C010F5F1F4FC8010E94A6
:10A52000D37460931F187093201880932118909310
:10A5300022186CE270E0C8010E94E1758C010F5F87
:10A540001F4FC8010E94D37460932F177093301768
:10A5500080933117909332176CE270E0C8010E942B
:10A56000E1756CE270E001960E94E17501960E942F
:10A57000D37460934117709342178093431790935D
:10A58000441720912F173091301740913117509177
:10A5900032170E94437160934E1770934F17809348
:10A5A000501790935117F88DF0933317298D2093FE
:10A5B00023186091671770916817809169179091BF
:10A5C0006A17FE3429F020E030E040E85FEB04C079
:10A5D00020E030E040E85FE30E94DE72609367179E
:10A5E000709368178093691790936A1760916B173F
:10A5F00070916C1780916D1790916E17398D35346D
:10A6000029F020E030E040E85FEB04C020E030E0DB
:10A6100040E85FE30E94DE7260936B1770936C17E3
:10A6200080936D1790936E176AEB76E08DE69DE14F
:10A630000E94F775892B09F4CAC08091B31A882348
:10A6400009F4B5C06CE270E08DE69DE10E94E17511
:10A650008C010F5F1F4F8091010C811108C0C80150
:10A660000E94D3740E9421722B013C0103C0412C33
:10A67000512C32016CE270E0C8010E94E1756CE27D
:10A6800070E001960E94E1756CE270E001960E9414
:10A69000E1756CE270E001960E94E1756CE270E099
:10A6A00001960E94E1756CE270E001960E94E175EE
:10A6B0008C010F5F1F4FC8010E94D374609347172E
:10A6C000709348178093491790934A1726E53EE008
:10A6D0004DEE5FE30E94DE7260935E1770935F172A
:10A6E00080936017909361176CE270E0C8010E943C
:10A6F000E1758C010F5F1F4FC8010E94D3746093F6
:10A700003B1770933C1780933D1790933E176CE274
:10A7100070E0C8010E94E1752091010C211108C070
:10A7200001960E94D3740E9421724B015C0103C008
:10A73000812C912C54018091010C811148C0C301DE
:10A74000B20120E137E240E050E00E94857320939F
:10A750002A1824E6C22ED12CE12CF12CA701960157
:10A760000E94857320934D17C301B201A701960182
:10A770000E94857360932517C501B40120E137E27B
:10A7800040E050E00E94857320931018A7019601C5
:10A790000E94857320931118C501B401A701960189
:10A7A0000E9485736093000C0E94065010C01092A6
:10A7B0004717109248171092491710924A17109293
:10A7C0005E1710925F1710926017109261176F96C4
:10A7D0000FB6F894DEBF0FBECDBFDF91CF911F91B2
:10A7E0000F91FF90EF90DF90CF90BF90AF909F9030
:10A7F0008F907F906F905F904F903F902F90089533
:10A80000CF938A3001F5EDEEFCE1ADE6BDE18DE1DF
:10A81000ED36F80719F081918D93F9CFC0E8EDEE90
:10A82000FCE1DF018C2F1D928A95E9F78091E20B04
:10A830000E94CD50EDE6FDE1DF011D92CA95E9F7DA
:10A840001092E20B0CC0E091E20BE7FD08C091E032
:10A850009E0F9093E20BF0E0E351F34E8083CF9193
:10A8600008954FB7F89420912111309122118091D1
:10A870002311909124114FBF2817390711F19FB769
:10A88000F894E0912111F091221120911F11309143
:10A890002011E217F30729F420911D1130911E11A8
:10A8A00007C0E0912111F09122119F012F5F3F4FCE
:10A8B000309322112093211180819FBF0E94005468
:10A8C000D0CF0895EF92FF920F931F93CF93DF9312
:10A8D0001F92CDB7DEB785E1E82EF12C8091EA0B0F
:10A8E000811129C09FB7F894009134171091351742
:10A8F00020913617309137179FBF9FB7F89440913A
:10A9000034175091351760913617709137179FBFE4
:10A91000401B510B620B730B4C36574061057105A0
:10A9200060F389830E94351291E0E91AF108898168
:10A93000E114F10499F60F90DF91CF911F910F91DF
:10A94000FF90EF900895EF92FF920F931F937B017A
:10A9500023E0EE0CFF1C2A95E1F700E010E09C01DB
:10A9600040E850E060E57EE183EA9AE10E945E5BA8
:10A970001F910F91FF90EF9008958091EA0B089539
:10A9800060E57EE180E69EE10E94825880E1E2EF90
:10A99000FDE1A2E0BEE101900D928A95E1F70895F4
:10A9A000CF93DF93EC01A2E0BEE1FC019C01205FAC
:10A9B0003F4F8D91908189278193E217F307C9F763
:10A9C000BE0180E69EE10E94C25980E1FE01A2E044
:10A9D000BEE101900D928A95E1F7DF91CF91089544
:10A9E0000F931F93CF93DF93CDB7DEB760970FB66A
:10A9F000F894DEBF0FBECDBF8C0180E1F801DE010F
:10AA0000119601900D928A95E1F7B80180E69EE1DA
:10AA10000E94DB5AE2E0FEE1D8019801205F3F4F3F
:10AA200081919C9189278D93A217B307C9F780E183
:10AA3000FE013196A2E0BEE101900D928A95E1F708
:10AA400060960FB6F894DEBF0FBECDBFDF91CF91F9
:10AA50001F910F9108951F93CF93DF9300D0CDB72F
:10AA6000DEB70E940112182F882309F476C041E056
:10AA700061EC76E082E19EE10E9450358093ED1D0D
:10AA80008430D9F582E19EE10E94D73E46E061EC38
:10AA900076E082E19EE10E9450358093ED1D8111A8
:10AAA00023C01092E60B1092E70B1092E80B109265
:10AAB000E90B1092101F1092111F1092121F10928A
:10AAC000131F1A8219829E012F5F3F4F44E050E00E
:10AAD00060E17FE182E19EE10E94823A8093ED1D78
:10AAE00082E19EE10E94D73E41E061EC76E082E1A6
:10AAF0009EE10E9450358093ED1D8091ED1D8111E6
:10AB00002CC01A8219829E012F5F3F4F44E050E013
:10AB100060E17FE182E19EE10E94AC388093ED1D0F
:10AB200082E19EE10E94D73E8091ED1D811115C00A
:10AB300089819A81049789F48091101F9091111F47
:10AB4000A091121FB091131F8093E60B9093E70B17
:10AB5000A093E80BB093E90B05C082E19EE10E944F
:10AB6000D73E10E0812F0F900F90DF91CF911F9172
:10AB70000895CF93DF9300D0CDB7DEB742E061EC0C
:10AB800076E082E19EE10E9450358093ED1D8111B7
:10AB900038C08091E60B9091E70BA091E80BB09143
:10ABA000E90B0496A11DB11D8093E60B9093E70B72
:10ABB000A093E80BB093E90B8093101F9093111FA3
:10ABC000A093121FB093131F1A8219829E012F5F48
:10ABD0003F4F44E050E060E17FE182E19EE10E946E
:10ABE000823A8093ED1D82E19EE10E94D73E8091E2
:10ABF000ED1D811106C089819A81049711F481E0CD
:10AC000001C080E00F900F90DF91CF9108952F92B7
:10AC10003F924F925F926F927F928F929F92AF92EC
:10AC2000BF92CF92DF92EF92FF920F931F93CF9339
:10AC3000DF9300D01F92CDB7DEB70E9401128823A8
:10AC400009F484C00E94B9558B83882309F47EC01F
:10AC500041E069ED76E082E19EE10E94503580930B
:10AC6000ED1D811173C040901C1E50901D1E609000
:10AC70001E1E70901F1E4091E60B5091E70B6091D5
:10AC8000E80B7091E90B8A019B0140E050E060E025
:10AC900070E082E19EE10E94F53E8093ED1D8111FE
:10ACA0004FC0D301C2010497A109B1091C012D01B4
:10ACB00020913A1E30913B1E40913C1E50913D1E0A
:10ACC00060913E1E70913F1E8091401E9091411EEA
:10ACD00051016201E12CF12C00E010E00E9464744B
:10ACE00078F51A8219829E012F5F3F4F44E050E0B1
:10ACF00060E17FE182E19EE10E94AC388093ED1D2E
:10AD000082E19EE10E94D73E8091ED1D81111EC01F
:10AD10006091101F7091111F8091121F9091131F4D
:10AD20006093EE1D7093EF1D8093F01D9093F11DC5
:10AD30000E94CA7481E08093E50B1092E40B0BC073
:10AD400082E19EE10E94D73E0E94D51082E19EE101
:10AD50000E94D73E1B828B810F900F900F90DF9146
:10AD6000CF911F910F91FF90EF90DF90CF90BF9008
:10AD7000AF909F908F907F906F905F904F903F909B
:10AD80002F900895CF930E940112C82F811102C005
:10AD9000C0E00FC041E062EF76E082E19EE10E94F8
:10ADA00050358093ED1D8111F3CF82E19EE10E9429
:10ADB000D73E8C2FCF9108951F93CF93DF9300D070
:10ADC000CDB7DEB70E940112182F882389F141E028
:10ADD0006BE077E082E19EE10E9450358093ED1DAB
:10ADE000811126C01A8219829E012F5F3F4F40E1D8
:10ADF00050E060E17FE182E19EE10E94AC38809307
:10AE0000ED1D82E19EE10E94D73E8091ED1D8111F2
:10AE10000FC089819A81409759F4A0E5BEE1E0E135
:10AE2000FFE180E18E0F91919D938E13FCCF01C0C5
:10AE300010E0812F0F900F90DF91CF911F91089517
:10AE40001092EA0B0E94C256882331F08091241898
:10AE50008823F1F00C9406070E94DC56882369F0E1
:10AE60000E942B55882349F00E940756882329F019
:10AE70000E94F40681E08093EA0B809124188823D5
:10AE800039F08091EA0B81110C9494100C94D51038
:10AE900008950F931F93CF93DF931091E50B112328
:10AEA00089F0C2EFDDE10C2F005F0E94C674699348
:10AEB0000C13FBCF9091E40B9F5F9093E40B97FDF5
:10AEC0000E940756812FDF91CF911F910F91089516
:10AED00082EF9DE1089580E1E3EAFAE1A2EFBDE1AE
:10AEE00001900D928A95E1F70895FC01808191818E
:10AEF00090839281918393819283838308954F926B
:10AF00005F926F927F929F92AF92BF92CF92DF92A9
:10AF1000EF92FF920F931F93CF93DF9300D000D057
:10AF2000CDB7DEB78C01D62EBA01C22EE22EF12C9F
:10AF30005701AA0CBB1CAA0CBB1CA5010E94D8750A
:10AF4000A00EB11EF501349780819181A281B38159
:10AF500089839A83AB83BC832C2DBC2CA12CBD147C
:10AF600008F0B2C02C1145C0CE0101960E94755761
:10AF700049805A806B807C80872D9927AA27BB2720
:10AF8000FC01EB57FC4F2491462D50E0FA01EB57A2
:10AF9000FC4F4491852D90E0FC01EB57FC4F8491D0
:10AFA000552466247724F201EB57FC4F449050E07F
:10AFB00060E070E0BA0155274427722B442990E0E5
:10AFC000F82FEE27CF01AA2797FDA095BA2F482B7F
:10AFD000592B6A2B7B2B49835A836B837C83EA2D05
:10AFE000F0E0EB52FA4FE081E427E983A39420E0FC
:10AFF00042C0243009F03FC048E0C4123CC08981FF
:10B000009A81AB81BC814B2F552766277727FA01A0
:10B01000EB57FC4F34914A2F50E0FA01EB57FC4FAD
:10B020004490492F50E0FA01EB57FC4F9490992738
:10B03000AA27BB27FC01EB57FC4F8491512C612CB4
:10B04000712C320155244424732AB301A201482BE8
:10B05000DB01CA01492D50E0F42FEE27AF0166272E
:10B0600057FD6095762F842B952BA62BB72B8983C4
:10B070009A83AB83BC838B2D90E0FC01EE19FF0912
:10B08000EE0FFF1FEE0FFF1FE00FF11F40805180FA
:10B090006280738049815A816B817C81442555256A
:10B0A0006625772549835A836B837C83880F991F94
:10B0B000880F991FF801E80FF91F408351836283BD
:10B0C0007383B3942F5F4BCF0F900F900F900F901F
:10B0D000DF91CF911F910F91FF90EF90DF90CF9074
:10B0E000BF90AF909F907F906F905F904F9008952A
:10B0F000AB0128E06CE30C947F57AB0126E064E3DE
:10B100000C947F57AB0124E06CE20C947F579C01B8
:10B1100090E1915050F0D901A90FB11DEC91F0E0F0
:10B12000EB57FC4FE491EC93F4CF08959C0190E130
:10B13000915050F0D901A90FB11DEC91F0E0EB57FF
:10B14000FD4FE491EC93F4CF0895FC01818195814A
:10B150009183918595839585918785878281928555
:10B160009283828786819685968386878381978559
:10B170009383938597879781938787830895FC01AD
:10B180008381978193839385978397859387878717
:10B19000828192859283828786819685968386872F
:10B1A0008181958591839185958795819187858307
:10B1B00008958F929F92BF92CF92DF92EF92FF926B
:10B1C0000F931F93CF93DF93BC0184E0D82EDA94C2
:10B1D000BFEFDB1609F44FC084E0D89EF0011124C4
:10B1E0007B01EE0EFF1ED7011C91512F550F550B01
:10B1F0005B71912F990F5927EF012196C60FD71F29
:10B200000881402F440F440B4B71202F220F4227FF
:10B21000DF011296A60FB71F2C91C22EC0263396BF
:10B220004F01860E971EF4013081922F990F990BD2
:10B230009B71822F880F9827832F880F880B8B7123
:10B24000B32EBB0C8B25BC2CB326B526B426F70138
:10B25000B08223272127422749274883202F2127EF
:10B260003227392738273C939C2D9127952789270A
:10B27000D4018C93ACCFDF91CF911F910F91FF90B0
:10B28000EF90DF90CF90BF909F908F900895CF92D6
:10B29000DF92EF92FF920F931F93CF93DF93DC0126
:10B2A000EB0194E09150E8F084E0989F9001112424
:10B2B0008D01020F131F2C0F3D1FF801C080D1809C
:10B2C000E280F380F90140815181628173814C25D4
:10B2D0005D256E257F25F80140835183628373834A
:10B2E000E1CFDF91CF911F910F91FF90EF90DF9011
:10B2F000CF900895CF92DF92EF92FF920F931F931A
:10B30000CF93DF938C01EB01C42EBC01CE010E94D0
:10B310004759EE24E394F12CCE01EC14B8F40E94CA
:10B320008758CE010E94A558CE010E94D958B70176
:10B3300084E0660F771F8A95E1F7600F711FCE01D9
:10B340000E9447598FEFE81AF80AE6CF0E94875803
:10B35000CE010E94A558B80180E1E89E600D711DE4
:10B360001124CE01DF91CF911F910F91FF90EF90AB
:10B37000DF90CF900C9447594EE00C947A594CE0F2
:10B380000C947A594AE00C947A5920E0882369F0A9
:10B39000982F9170919596232927962F990F990BA5
:10B3A0009B71660F69278695F1CF822F08953F9292
:10B3B0004F925F926F927F928F929F92AF92BF92C5
:10B3C000CF92DF92EF92FF920F931F93CF93DF9371
:10B3D00000D000D01F92CDB7DEB77C0194E0915031
:10B3E00008F484C084E0989F900111243B832A8351
:10B3F00049018E0C9F1CF4011081612F8EE09D830A
:10B400000E94C559382EAA80BB80FFEFAF1ABF0A31
:10B41000AE0CBF1CF5015080652D8BE00E94C55914
:10B420003826CA80DB80F2E0CF0ED11CCE0CDF1CA8
:10B43000F6016080662D8DE00E94C55938262A816C
:10B440003B812D5F3F4F2E0D3F1DF9017080672D11
:10B4500089E029833C830E94C5593826612F89E001
:10B460000E94C559482E652D8EE00E94C559482678
:10B47000662D8BE00E94C5594826672D8DE00E94FD
:10B48000C5594826612F8DE00E94C559082F652DAA
:10B4900089E00E94C5590827662D8EE00E94C55993
:10B4A0000827672D8BE00E94C5590827612F8BE084
:10B4B0000E94C559182F652D8DE00E94C559182787
:10B4C000662D89E00E94C5591827672D8EE00E94DD
:10B4D000C559F4013082F5014082F60100838127CD
:10B4E00029813C81F90180839D8179CF0F900F9054
:10B4F0000F900F900F90DF91CF911F910F91FF90C0
:10B50000EF90DF90CF90BF90AF909F908F907F9003
:10B510006F905F904F903F900895BF92CF92DF92CF
:10B52000EF92FF920F931F93CF93DF937C01EB0178
:10B53000B42EC42ED12CBC0180E1489F600D711D3A
:10B540001124CE010E94475900E010E00F5F1F4F09
:10B55000CE010B15C0F40E94BF58CE010E94965830
:10B56000B601601B710B9B0184E0220F331F8A958B
:10B57000E1F7B701620F731FCE010E944759CE0158
:10B580000E94D759E3CF0E94BF58CE010E9496581F
:10B59000B701CE01DF91CF911F910F91FF90EF90F6
:10B5A000DF90CF90BF900C9447594EE00C948D5A89
:10B5B0004CE00C948D5A4AE00C948D5ABF92CF9275
:10B5C000DF92EF92FF920F931F93CF93DF93CDB74C
:10B5D000DEB7C054D1090FB6F894DEBF0FBECDBFA1
:10B5E0007C018E010F5F1F4F80E4F80111928A9554
:10B5F000E9F74130F2E05F0738F09A0140E050E0AF
:10B60000C8010E9400600AC0495F5F4F93E05695F1
:10B6100047959A95E1F7C8010E94D8756801F8012D
:10B6200096E380E4B82EB00E808189278193BE1204
:10B63000FBCFC7010E94955DB801C7010E94BB5DA9
:10B640009AE6F6018081892781936F01BE12F9CFB6
:10B65000F4E1EF0EF11CC7010E94955DB801C7012E
:10B660000E94BB5DC05CDF4F0FB6F894DEBF0FBE1B
:10B67000CDBFDF91CF911F910F91FF90EF90DF90A1
:10B68000CF90BF9008950C94BB5D0C94435F0F93D3
:10B690001F93CF93DF938C01EB010E94F85F6496B8
:10B6A00040E850E0B801CE010E94435FBE01C801EE
:10B6B000DF91CF911F910F910C94F85F2F923F92E1
:10B6C0004F925F926F927F928F929F92AF92BF92B2
:10B6D000CF92DF92EF92FF920F931F93CF93DF935E
:10B6E000CDB7DEB7C755D1090FB6F894DEBF0FBE90
:10B6F000CDBF5C014901170128018E010F5F1F4F6B
:10B7000080E4F80111928A95E9F74130F2E05F0791
:10B7100038F09A0140E050E0C8010E9400600AC081
:10B72000495F5F4FE3E056954795EA95E1F7C80119
:10B730000E94D87567961FAF0EAF6797F80196E322
:10B7400020E4200F68962FAF689780818927819326
:10B7500068962FAD68972E13F8CFCE018F5B9F4F61
:10B760000E94955DB801CE018F5B9F4F0E94BB5D2B
:10B77000720161013401C114F2E0DF06E104F10459
:10B7800070F0B301CE018F5B9F4F0E94BB5D80E4E0
:10B79000680E711CE2E0DE1AE108F108ECCFB2019C
:10B7A000A101517066277727D201C10129E0B69522
:10B7B000A795979587952A95D1F71C0136E0220C1D
:10B7C000331C3A95E1F7280C391CB101CE018F5B8F
:10B7D0009F4F0E94435F9AE66796EEADFFAD679775
:10B7E0008081892781936796FFAFEEAF6797689650
:10B7F0002FAD68972E13F0CFBE016F5B7F4FC50151
:10B800000E94F85FCE018F5B9F4F0E94955DB8014B
:10B81000CE018F5B9F4F0E94BB5D40E850E0B501B9
:10B82000CE018F5B9F4F0E94435FBE016F5B7F4FD6
:10B83000C5010E94F85FC95ADF4F0FB6F894DEBF0A
:10B840000FBECDBFDF91CF911F910F91FF90EF9071
:10B85000DF90CF90BF90AF909F908F907F906F9030
:10B860005F904F903F902F9008958F929F92AF924C
:10B87000BF92CF92DF92EF92FF920F931F934B01F3
:10B880005C0180949094A094B09467017801C820E2
:10B89000D920EA20FB20DC01CB0182239323A423BF
:10B8A000B523BC01CD016C297D298E299F291F91CB
:10B8B0000F91FF90EF90DF90CF90BF90AF909F904F
:10B8C0008F9008958F929F92AF92BF92EF92FF92C6
:10B8D0000F931F934701580180949094A094B094C3
:10B8E00082229322A422B522DC01CB018E219F214A
:10B8F000A023B123BC01CD01682979298A299B297C
:10B900001F910F91FF90EF90BF90AF909F908F90FD
:10B910000895AF92BF92CF92DF92EF92FF920F9372
:10B920001F9359016A01AE24BF24C026D1266A257F
:10B930007B258C259D251F910F91FF90EF90DF9027
:10B94000CF90BF90AF900895CF92DF92EF92FF9289
:10B950000F931F9367017801C094D094E094F09402
:10B96000DC01CB018C299D29AE29BF29BC01CD0169
:10B9700062277327842795271F910F91FF90EF90DF
:10B98000DF90CF9008952F923F924F925F926F92E7
:10B990007F928F929F92AF92BF92CF92DF92EF925F
:10B9A000FF920F931F93CF93DF93CDB7DEB72C9702
:10B9B0000FB6F894DEBF0FBECDBF4B01C22E098774
:10B9C000DE2C28E0EFEDF5E0DE01119601900D92FE
:10B9D0002A95E1F74370642F70E01C0124E0429F38
:10B9E000200C311C1124D1014D905D906D907C9004
:10B9F0005B01BFEFAB1ABB0AE3E0AE22BB24AA0C8B
:10BA0000BB1CAA0CBB1CA80EB91EFB013396E3702D
:10BA1000FF27EE0FFF1FEE0FFF1FE80FF91FE0805B
:10BA2000F180028113816E5F7F4F63707727660F0D
:10BA3000771F660F771FFC01E60FF71F208131810A
:10BA400042815381D5016D917D918D919C91FE0133
:10BA50003196ED0DF11DED0DF11D0190F081E02D00
:10BA600009952985B4E02B9FF0011124EB57FB4F7A
:10BA7000259135914591549129873A874B875C8769
:10BA8000D4010D911D912D913C91400E511E621ECD
:10BA9000731E460E571E681E791E29853A854B85F2
:10BAA0005C85420E531E641E751EB301A2010C2C50
:10BAB00004C0440F551F661F771F0A94D2F78C2DC0
:10BAC00081958F7104C076946794579447948A95B2
:10BAD000D2F7442A552A662A772AF5018081918176
:10BAE000A281B381480E591E6A1E7B1ED1014D9260
:10BAF0005D926D927C9213972C960FB6F894DEBFF0
:10BB00000FBECDBFDF91CF911F910F91FF90EF90AE
:10BB1000DF90CF90BF90AF909F908F907F906F906D
:10BB20005F904F903F902F900895FC01108A118AEA
:10BB3000128A138A81E093E2A5E4B7E680839183B9
:10BB4000A283B38389E89BEAADECBFEE848395833F
:10BB5000A683B7838EEF9CEDAAEBB8E98087918727
:10BB6000A287B38786E794E5A2E3B0E1848795874F
:10BB7000A687B78708952F923F924F925F926F9258
:10BB80007F928F929F92AF92BF92CF92DF92EF926D
:10BB9000FF920F931F93CF93DF93CDB7DEB7A1979B
:10BBA0000FB6F894DEBF0FBECDBF6C015B01FC0188
:10BBB00080819181A281B38189839A83AB83BC8385
:10BBC00084819581A681B7818D839E83AF83B88759
:10BBD00080859185A285B38589879A87AB87BC8745
:10BBE00084859585A685B7858D879E87AF87B88B19
:10BBF00087E08D8F8CE08E8F81E18F8F86E188A327
:10BC00002E01FDE14F0E511C342D3195812C912CCC
:10BC10001201612C712C14E0032F020DF10121910E
:10BC20001F01B301680D791D6A0D7B1DE12C412FA9
:10BC3000CE01019639A30E94C35C1150F4E06F0E4F
:10BC4000711C39A11111E8CF3C5F80E1880E911C75
:10BC5000E0E48E169104E1F685E0898F89E08A8F11
:10BC60008EE08B8F84E18C8F88248394912C2E011D
:10BC7000F9E14F0E511C8FE0F82EF4183401120137
:10BC800014E03F2D380D032F020DF10121911F010A
:10BC9000B3016F707727660F771F660F771F6A0DE6
:10BCA0007B1DEE24E394412FCE01019639A30E941F
:10BCB000C35C1150F5E06F0E711C39A11111E3CF77
:10BCC00084E0880E911CE1E18E169104B9F684E0BF
:10BCD0008D8B8BE08E8B80E18F8B87E1888F65E089
:10BCE000862E912C2E01F5E14F0E511C85E2F82E87
:10BCF000F4183401120114E03F2D3819032F020DFE
:10BD0000F10121911F01B3016F707727660F771F33
:10BD1000660F771F6A0D7B1D52E0E52E412FCE0185
:10BD2000019639A30E94C35C1150F3E06F0E711CA1
:10BD300039A11111E3CF84E0881A9108E5EF8E163E
:10BD4000EFEF9E06B1F686E0898B8AE08A8B8FE062
:10BD50008B8B85E18C8B812C912C2E01F1E14F0E88
:10BD6000511C80E3F82EF4183401120114E03F2D29
:10BD70003819032F020DF10121911F01B3016F70DA
:10BD80007727660F771F660F771F6A0D7B1D93E07D
:10BD9000E92E412FCE01019639A30E94C35C1150B8
:10BDA000F7E06F0E711C39A11111E3CF84E0881AFE
:10BDB0009108E0EF8E16EFEF9E06B1F6F601408196
:10BDC00051816281738189819A81AB81BC81840FA9
:10BDD000951FA61FB71F80839183A283B3834481DD
:10BDE0005581668177818D819E81AF81B885840F71
:10BDF000951FA61FB71F84839583A683B7834085AD
:10BE000051856285738589859A85AB85BC85840F4C
:10BE1000951FA61FB71F80879187A287B387448588
:10BE20005585668577858D859E85AF85B889840F14
:10BE3000951FA61FB71F84879587A687B787808918
:10BE40009189A289B3890196A11DB11D808B918B27
:10BE5000A28BB38BA1960FB6F894DEBF0FBECDBFF9
:10BE6000DF91CF911F910F91FF90EF90DF90CF90D6
:10BE7000BF90AF909F908F907F906F905F904F900A
:10BE80003F902F9008956F927F928F929F92AF92E2
:10BE9000BF92CF92DF92EF92FF920F931F93CF93B7
:10BEA000DF93CDB7DEB7C054D1090FB6F894DEBF2B
:10BEB0000FBECDBF8C016B014A017A015B01E11419
:10BEC000E2E0FE0650F0B501C8010E94BB5D82E0D1
:10BED000F81A90E4A90EB11CF2CF5401AB2CBB248C
:10BEE000A69446E0AA0CBB1C4A95E1F7AC0CBD1C1D
:10BEF0006401F1E0DF22CE0101967C0180E4F701CC
:10BF000011928A95E9F7360153E0769467945A9531
:10BF1000E1F7A301B501C7010E94D875F7E08F22B0
:10BF20009924F701E60DF71D8114910469F0D501FC
:10BF3000A60DB71D80E890E002C0959587958A947C
:10BF4000E2F79C91892B01C080E8808388E0680E2D
:10BF5000711C90E469167104A8F0B701C8010E9431
:10BF6000BB5DF80180899189A289B3890197A109F4
:10BF7000B109808B918BA28BB38B88E3F70111926F
:10BF80008A95E9F7F80180899189A289B38929E026
:10BF9000880F991FAA1FBB1F2A95D1F78C0D9D1DD5
:10BFA000A11DB11D9C01AD0189AF3AAF4BAF5CAF94
:10BFB0001DAE1EAE1FAE21961FAE2197B701C80160
:10BFC0000E94BB5DC05CDF4F0FB6F894DEBF0FBEB2
:10BFD000CDBFDF91CF911F910F91FF90EF90DF9038
:10BFE000CF90BF90AF909F908F907F906F9008956B
:10BFF000DC0190E1FB0101900D929A95E1F7089523
:10C000008F929F92AF92BF92CF92DF92EF92FF9268
:10C010000F931F93CF93DF93CDB7DEB768970FB61B
:10C02000F894DEBF0FBECDBF7C018B01CE0101961F
:10C030002D8B3E8B4F8B588F0E94955D2D893E89AD
:10C040004F89588D49015A016801811482E0980690
:10C05000A104B104A8F0B601CE0101962D8B3E8B50
:10C060004F8B588F0E94BB5D80E4C80ED11C82E0CC
:10C07000981AA108B108588D4F893E892D89E5CFBE
:10C08000DA01C9019170AA27BB27BA01A90129E0E9
:10C0900076956795579547952A95D1F79A0146E089
:10C0A000220F331F4A95E1F7B801620F731FAC01ED
:10C0B000CE0101960E94435FBE016F5F7F4FC701B3
:10C0C0000E94F85F68960FB6F894DEBF0FBECDBF32
:10C0D000DF91CF911F910F91FF90EF90DF90CF9064
:10C0E000BF90AF909F908F900895CF92DF92EF9284
:10C0F000FF920F931F93CF93DF931F92CDB7DEB7BD
:10C100007C01262F82E8860F87010B591D4F823054
:10C1100010F06B3149F4F801608171818BE190E09E
:10C1200029830E9474762981D701A559BD4F3C917E
:10C1300011964C911197822F90E0FC01E327EE0FAE
:10C14000FF1FEB57FA4F25913491C42ED12C2C258B
:10C150003D252D933C93F801608171810F90DF9113
:10C16000CF911F910F91FF90EF90DF90CF900C94A3
:10C170007476CF93DF93E2E7F2E0DC01EF011D92EA
:10C180002197E9F7FC01EB59FD4F5183408332972A
:10C19000718360833A963183208332972FEF3FEF8C
:10C1A00031832083329731832083389681E08083E6
:10C1B000DF91CF9108953F924F925F926F927F925D
:10C1C0008F929F92AF92BF92CF92DF92EF92FF92A7
:10C1D0000F931F93CF93DF932C013C012BE9621A3D
:10C1E0002DEF720A6C0140E9C41A4DEFD40AEC013C
:10C1F000C159DD4F8C0109591D4F7C0187E9E81AAF
:10C200008DEFF80A33243394AA24AA94BA2C42015D
:10C21000A3E98A1AADEF9A0AF301808191810E9405
:10C2200019768F3FFFEF9F0709F45CC0F60120816C
:10C2300021112CC08E379105F1F4D8018D919C917C
:10C24000049788F0F70180819181883B904F21F01D
:10C2500080911618882339F0D401ED91FC91309724
:10C2600011F0C20109953882F701B182A082D8018C
:10C270001D921C92D1CF8F37910511F41882CCCF2B
:10C280008B31910519F4F6013082C6CF2881222323
:10C2900031F1D8012D913C912336B2E03B07F0F407
:10C2A000A9014F5F5F4FF80151834083F201E20F14
:10C2B000F31F8083D7012D913C91F901E827FF27D7
:10C2C000EE0FFF1FEB57FA4F85919491232F3327E1
:10C2D00082279327F7019183808301C01882D601BA
:10C2E0001C929ACFDF91CF911F910F91FF90EF9009
:10C2F000DF90CF90BF90AF909F908F907F906F9086
:10C300005F904F903F9008956F927F928F929F928F
:10C31000AF92BF92CF92DF92EF92FF920F931F9353
:10C32000CF93DF93EC013B014A016C018FE8C81AFF
:10C330008DEFD80AF60110825E01F5E9AF1AFDEF24
:10C34000BF0A8FEF9FEFF501918380837E01FBE9A8
:10C35000EF1AFDEFFF0AF701608171818EE790E02F
:10C360000E9474768301860C971C0815190549F004
:10C37000F80161918F01CE010E9475600E94586A98
:10C38000F4CFF501608111816095CE010E94756046
:10C39000612F6095CE010E947560F7016081718107
:10C3A0008EE790E00E947476C8E0F70160817181A9
:10C3B0008EE790E00E947476C150B9F781E0F601F3
:10C3C0008083DF91CF911F910F91FF90EF90DF90CD
:10C3D000CF90BF90AF909F908F907F906F90089577
:10C3E0002FB7F894609134177091351780913617F4
:10C3F000909137172FBF0895FC012FB7F894A681AD
:10C40000B7816D937C9346815781828193814817D0
:10C41000590719F48081918103C086819781029622
:10C42000978386832FBF0895FC012FB7F894A481CA
:10C43000B58182819381A817B90719F48081918110
:10C4400004C0A481B581CD010296958384838D912A
:10C450009C912FBF0895CF93DF9390939A3A809346
:10C46000993A509375174093741770939C3A609360
:10C470009B3A80E797E1E0E2FFE1DF019C011D923A
:10C4800021503040E1F7C6EDD6E388E0DE01E82F29
:10C490001D92EA95E9F7A5E1B8E3FD0111928A95AD
:10C4A000E9F7EEECF6E3D183C083D783C683D58367
:10C4B000C48382EF96E393838283E0ECFAE3B18353
:10C4C000A083B783A683B583A48381E398E3938392
:10C4D0008283DF91CF9108951F93CF93DF9300D094
:10C4E000CDB7DEB70E940112182F882309F476C059
:10C4F00041E060E277E080E996E30E945035809366
:10C5000010388430D9F580E996E30E94D73E46E0A2
:10C5100060E277E080E996E30E945035809310381E
:10C52000811123C01092EC0B1092ED0B1092EE0BC8
:10C530001092EF0B1092113810921238109213389B
:10C54000109214381A8219829E012F5F3F4F44E0E7
:10C5500050E061E178E380E996E30E94823A8093BB
:10C56000103880E996E30E94D73E41E060E277E030
:10C5700080E996E30E9450358093103880911038FE
:10C5800081112CC01A8219829E012F5F3F4F44E017
:10C5900050E061E178E380E996E30E94AC38809353
:10C5A000103880E996E30E94D73E809110388111BF
:10C5B00015C089819A81049789F4809111389091EE
:10C5C0001238A0911338B09114388093EC0B9093EB
:10C5D000ED0BA093EE0BB093EF0B05C080E996E353
:10C5E0000E94D73E10E0812F0F900F90DF91CF91E6
:10C5F0001F910895CF93DF9300D0CDB7DEB742E00F
:10C6000060E277E080E996E30E945035809310382D
:10C61000811138C08091EC0B9091ED0BA091EE0B45
:10C62000B091EF0B0196A11DB11D8093EC0B90937F
:10C63000ED0BA093EE0BB093EF0B8093113890931A
:10C640001238A0931338B09314381A8219829E01BD
:10C650002F5F3F4F44E050E061E178E380E996E3EB
:10C660000E94823A8093103880E996E30E94D73E78
:10C6700080911038811106C089819A81049711F444
:10C6800081E001C080E00F900F90DF91CF9108957D
:10C690001F93CF93DF93CDB7DEB76A970FB6F894A9
:10C6A000DEBF0FBECDBF0E940112811102C010E09B
:10C6B000E6C066EF76E38BE397E00E942F4380931A
:10C6C00010388450823060F066EF76E385E497E0BE
:10C6D0000E942F43809310388450823090F409C018
:10C6E0008BE397E00E948E4680931038882361F395
:10C6F000DECF85E497E00E948E468093103881114A
:10C70000D6CF0E946C62182F882389F2EDE9FAE3F4
:10C7100080E2DF01282F1D922A95E9F79091EF0B17
:10C720009F939091EE0B9F939091ED0B9F9390911F
:10C73000EC0B9F9325E437E03F932F9323E537E0FD
:10C740003F932F931F928F93FF93EF930E94F07666
:10C750000E94FA6246E06DE97AE380E996E30E947E
:10C760005035809310380FB6F894DEBF0FBECDBFA2
:10C7700081119DCF84ED93ECA2EBB1EA898B9A8B6A
:10C78000AB8BBC8B82E090E09A8F898F84E090E045
:10C79000988F8F8B1D861E861F86188A19861A868B
:10C7A0001B861C8683E692E0A0E0B0E08D839E832A
:10C7B000AF83B88783E090E0A0E0B0E089839A83FC
:10C7C000AB83BC831E8A1D8A9E012B5E3F4F44E0D3
:10C7D00050E0BE016F5E7F4F80E996E30E94823A8F
:10C7E0009E012B5E3F4F42E050E0BE01675E7F4FEF
:10C7F00080E996E30E94823A9E012B5E3F4F42E021
:10C8000050E0BE01695E7F4F80E996E30E94823A64
:10C810009E012B5E3F4F44E050E0BE01635F7F4FBF
:10C8200080E996E30E94823A9E012B5E3F4F44E0EE
:10C8300050E0BE01675F7F4F80E996E30E94823A35
:10C840009E012B5E3F4F44E050E0BE016B5F7F4F87
:10C8500080E996E30E94823A9E012B5E3F4F44E0BE
:10C8600050E0BE016F5F7F4F80E996E30E94823AFD
:10C8700080E996E30E94D73E81E08093F00B812F00
:10C880006A960FB6F894DEBF0FBECDBFDF91CF9191
:10C890001F9108956F927F928F929F92AF92BF9255
:10C8A000CF92DF92EF92FF920F931F93CF93DF937C
:10C8B000CDB7DEB76E970FB6F894DEBF0FBECDBF13
:10C8C0008C010E94BD54980129593D4F6901811185
:10C8D00012C0609174177091751780EC90E00E94FF
:10C8E0007476609174177091751780E090E00E94E3
:10C8F0007476780179C0D901ED90FC90B3E3EB1622
:10C90000F10408F430C1F8019080B7016251710957
:10C91000FE01319680E1DF011D928A95E9F7D80189
:10C92000A60FB71F5F0140E1842E8E0E8D9181937B
:10C930008E12FCCFC8010E94A354E3EAFAE1D501AC
:10C940009D915D01819198130EC18A12F8CFD80193
:10C950001196E3EAFAE130E1A32EAE0E8D918193B8
:10C96000AE12FCCF0E946B570E94C054C701839740
:10C9700024E0969587952A95E1F7B82E3801812C09
:10C980008B14C0F4D3015196E3EAFAE18D918193BF
:10C99000AE12FCCF83EA9AE10E94F054D301E3EA9D
:10C9A000FAE181918D93AE12FCCF8394B0E16B0ECE
:10C9B000711CE6CFE1E2EE1AF108E918F108D601A0
:10C9C000ED92FC9286CFF70181917F01803CD9F4F2
:10C9D0008BED90E00E9474766091741770917517DA
:10C9E0008CED90E00E947476D6018D919C91029717
:10C9F00060917417709175179701201B310B2817E0
:10CA0000390708F30FC08B3D59F48BED90E00E947D
:10CA1000747660917417709175178DED90E0E2CF88
:10CA200090E0E0CF80EC90E00E94747680912E1729
:10CA3000882309F498C00E940112882309F493C046
:10CA40008091F00B882309F48AC042E36DE97AE310
:10CA500080E996E30E94503580931038811183C09D
:10CA60001E8E1D8E2FB7F89480916F1790917017BE
:10CA7000A0917117B09172172FBF80589C4BA2499B
:10CA8000B74C898F9A8FAB8FBC8F0E94F06120E0EA
:10CA90003BE440E050E00E948573675F7F4F8F4F1B
:10CAA0009F4F23E130E040E050E00E948573A8EE04
:10CAB000B3E00E945A736D8B7E8B8F8B988FF6013B
:10CAC000808191810297A0E0B0E0898B9A8BAB8B3B
:10CAD000BC8B89839A83AB83BC839E01235E3F4FCB
:10CAE00044E050E0BE01675E7F4F80E996E30E941C
:10CAF000823A9E01235E3F4F44E050E0BE016B5EF0
:10CB00007F4F80E996E30E94823A9E01235E3F4F69
:10CB100044E050E0BE016F5E7F4F80E996E30E94E3
:10CB2000823A9E01235E3F4F44E050E0BE016F5FBA
:10CB30007F4F80E996E30E94823AD6014D915C9145
:10CB4000425051099E01235E3F4FB80180E996E3B0
:10CB50000E94823A80E996E30E94D73E04C00E9478
:10CB60004863811172CF6E960FB6F894DEBF0FBE88
:10CB7000CDBFDF91CF911F910F91FF90EF90DF908C
:10CB8000CF90BF90AF909F908F907F906F900895BF
:10CB90002F923F924F925F926F927F928F929F92CD
:10CBA000AF92BF92CF92DF92EF92FF920F931F93BB
:10CBB000CF93DF93CDB7DEB766970FB6F894DEBF9D
:10CBC0000FBECDBF8091EB0B8111BCC181E0809382
:10CBD000EB0B212C312CE12CF12C83EA9AE130E192
:10CBE000C32EC80E8091FF0B90E02816390608F07E
:10CBF00090C18EEC96E30E9414625C0180EC9AE393
:10CC00000E9414628C01029708F47FC10E94BD54F7
:10CC1000882309F4C0C0802F8F7090E1D92ED81AD4
:10CC2000D91201C0D12C6D2C712C060D171D24E0DA
:10CC3000169507952A95E1F70B8B0E944957882393
:10CC400009F4A6C00E94C054D09235380E9468579B
:10CC5000E6E3F8E39C01205F3F4FDC014D91CD01FD
:10CC60004193A217B307C9F796E4492E98E3592ECA
:10CC7000812C912C1127C80101979D8B8C8BA0E1F1
:10CC8000B0E0A619B7093D0180E1482F4D198B8905
:10CC9000881608F052C08C899D898816990614F070
:10CCA000D11017C0E3EAFAE19501235A3A41C901CC
:10CCB0008E0F9F1F60E777E10E947173DC01A05E19
:10CCC000B04E8C918193CE12F2CF90E1A90EB11C9F
:10CCD00020C020E0822F90E08615970584F4FC01A7
:10CCE000ED55F54E8A0D9B1D60E777E10E9471734B
:10CCF000DC01A05EB04E8C9180832F5FEBCF842F40
:10CD00009FEFE82FF0E0ED55F54E90838F5F803177
:10CD1000C1F783EA9AE14E8B0E94D054D201E3EA34
:10CD2000FAE14E8981918D93CE12FCCFAFEF8A1A32
:10CD30009A0AB0E14B0E511CAACF84E0000F111FDC
:10CD40008A95E1F7580191E1A90EB11CB50185E37F
:10CD500098E30E94A354F501EB5CF74CA3EABAE117
:10CD60008D918193CA12FCCFA8014F5D5F4F87015F
:10CD70000F5F1F4F4436A2E05A0740F465E378E3A3
:10CD80008091993A90919A3A0E9484617801BDC04D
:10CD90000E94D510BAC0E5E3F8E395012553384366
:10CDA000C9018E0F9F1F60E777E10E947173DC015C
:10CDB000A05EB04E8C918193CF018553984380172C
:10CDC000910770F380912E17882309F492C00E9476
:10CDD0000112882309F48DC08091F00B882309F497
:10CDE00084C042E36DE97AE380E996E30E9450351E
:10CDF0008093103881117DC01A8A198A2FB7F89450
:10CE000080916F1790917017A0917117B091721760
:10CE10002FBF80589C4BA249B74C8D879E87AF8708
:10CE2000B88B0E94F06120E03BE440E050E00E94BB
:10CE30008573675F7F4F8F4F9F4F23E130E040E066
:10CE400050E00E948573A8EEB3E00E945A73698790
:10CE50007A878B879C87C801A0E0B0E08D839E8392
:10CE6000AF83B88789839A83AB83BC839E012F5E8F
:10CE70003F4F44E050E0BE01635F7F4F80E996E39F
:10CE80000E94823A9E012F5E3F4F44E050E0BE0177
:10CE9000675F7F4F80E996E30E94823A9E012F5E92
:10CEA0003F4F44E050E0BE016B5F7F4F80E996E367
:10CEB0000E94823A9E012F5E3F4F44E050E0BE0147
:10CEC0006F5F7F4F80E996E30E94823A9E012F5E5A
:10CED0003F4FA80165E378E380E996E30E94823A38
:10CEE00080E996E30E94D73E04C00E944863811106
:10CEF00078CFA80165E378E38091993A90919A3AC6
:10CF00000E948461BFEFEB1AFB0A8FEF281A380AE0
:10CF100069CE8091FF0B90E0E816F90658F48091F5
:10CF20007307811101C0299A809173078111F7CF8E
:10CF3000289AF5CF1092FF0B1092FE0B1092FD0B6A
:10CF40001092EB0B66960FB6F894DEBF0FBECDBF06
:10CF5000DF91CF911F910F91FF90EF90DF90CF90D5
:10CF6000BF90AF909F908F907F906F905F904F9009
:10CF70003F902F900895CF92DF92EF92FF92809191
:10CF8000FF0B882309F454C0E0919B3AF0919C3A3E
:10CF9000828981114DC0C090F50BD090F60BE090C6
:10CFA000F70BF090F80B0E94F0612EEBC20ED11C33
:10CFB000E11CF11CC616D706E806F906CCF58091EF
:10CFC000A21A8F3F31F4FF90EF90DF90CF900C9436
:10CFD000C8652091561730915717409158175091B6
:10CFE0005917A3E1B0E00E945A73C090F10BD090A2
:10CFF000F20BE090F30BF090F40BC60ED71EE81E78
:10D00000F91E0E94F061C616D706E806F90684F4F8
:10D010000E94C6748091A21A6817A8F20E94F0615B
:10D020006093F10B7093F20B8093F30B9093F40BDE
:10D03000FF90EF90DF90CF900895609174177091FA
:10D04000751780EC90E00E9474766091741770916F
:10D05000751784E190E00E94747660917417709166
:10D06000751783E090E00E94747660917417709158
:10D07000751780EC90E00C94747660917417709141
:10D08000751780EC90E00E9474766091741770912F
:10D09000751782E190E00E94747680916407609138
:10D0A000741770917517803C59F48BED90E00E94D5
:10D0B000747660917417709175178CED90E00EC0C6
:10D0C0008B3D59F48BED90E00E947476609174175B
:10D0D000709175178DED90E001C090E00E9474761C
:10D0E000609174177091751780EC90E00C947476D1
:10D0F000CF93DF939091BD3A992309F446C0803CC9
:10D1000009F051C080910301811142C01092BD3AD3
:10D110008091FF0B8F3008F0C8C18091FD0B90917A
:10D12000FE0B8037974108F0C0C16091F90B7091F8
:10D13000FA0B8091FB0B9091FC0B019710F48FE69A
:10D1400097E16817790709F4B0C16817790728F4DF
:10D15000861B970BEC01219605C0861B970BEC01F3
:10D16000CF58D84EC230D10508F49FC18091FF0B33
:10D170008F5F8093FF0B8EEC96E30E94FC61BE01F3
:10D1800080EC9AE30E94FC6121C0803C09F08DC1D3
:10D1900081E08093BD3A8EEF809303011092BF3AF5
:10D1A0001092BE3A82C12091BE3A3091BF3A2034EB
:10D1B00092E0390708F079C190910301232B79F4AB
:10D1C0009E3F69F48093030181116FC18091FB0B35
:10D1D0009091FC0B9093FA0B8093F90B66C191111F
:10D1E00046C08B3D21F481E08093983A5EC19091D6
:10D1F000983A992349F08C3D21F08D3D19F48BED3F
:10D2000001C080EC1092983A9091FF0B9F3008F08B
:10D210004CC12091FD0B3091FE0B2037374108F0B7
:10D2200044C12091FD0B3091FE0B2F5F3F4F309397
:10D23000FE0B2093FD0B2091FB0B3091FC0BA90101
:10D240004F5F5F4F5093FC0B4093FB0BF901E05E87
:10D25000F04E80838091FB0B9091FC0B80379741BF
:10D2600009F023C11092FC0B1092FB0B1EC19130F0
:10D2700079F4282F30E0AAE0B0E00E944B7360936D
:10D2800026187093271880932818909329180DC199
:10D29000943079F4282F30E0AAE0B0E00E944B737C
:10D2A00060931718709318188093191890931A1890
:10D2B000FCC0933079F4282F30E0AAE0B0E00E945F
:10D2C0004B7360935617709357178093581790932A
:10D2D0005917EBC0923019F48093A21AE6C0973028
:10D2E00021F4DF91CF910C94F206913139F48A390F
:10D2F00009F0DBC0DF91CF910C94F9069830A1F4CE
:10D300008B3D09F470CF9091983A992349F08C3D68
:10D3100021F08D3D19F48BED01C080EC1092983A0C
:10D32000DF91CF910C9421109930A1F48B3D09F439
:10D330005ACF9091983A992349F08C3D21F08D3D38
:10D3400019F48BED01C080EC1092983ADF91CF91E7
:10D350000C94F7049A30A1F48B3D09F444CF9091DA
:10D36000983A992349F08C3D21F08D3D19F48BEDCD
:10D3700001C080EC1092983ADF91CF910C94F9049F
:10D380009B30A1F48B3D09F42ECF9091983A9923CC
:10D3900049F08C3D21F08D3D19F48BED01C080ECFE
:10D3A0001092983ADF91CF910C94FB049C30A1F439
:10D3B0008B3D09F418CF9091983A992349F08C3D10
:10D3C00021F08D3D19F48BED01C080EC1092983A5C
:10D3D000DF91CF910C9404059D30A1F48B3D09F4AD
:10D3E00002CF9091983A992349F08C3D21F08D3DE0
:10D3F00019F48BED01C080EC1092983ADF91CF9137
:10D400000C940D059034A1F48B3D09F4ECCE909171
:10D41000983A992349F08C3D21F08D3D19F48BED1C
:10D4200001C080EC1092983ADF91CF910C941905CD
:10D430009E30A1F48B3D09F4D6CE9091983A992371
:10D4400049F08C3D21F08D3D19F48BED01C080EC4D
:10D450001092983ADF91CF910C942505903121F4E8
:10D46000DF91CF910C94F004903F19F40E941107C2
:10D4700018C0923131F48130C1F4DF91CF910C9416
:10D480003D68933151F4811104C0DF91CF910C9428
:10D490000E07DF91CF910C940A07943131F481117A
:10D4A00004C0DF91CF910C941D68DF91CF91089556
:10D4B0004FB7F89420912A1730912B1780912C1791
:10D4C00090912D174FBF2817390761F19FB7F89436
:10D4D000E0912A17F0912B172091281730912917E6
:10D4E000E217F30729F4209126173091271707C078
:10D4F000E0912A17F0912B179F012F5F3F4F309338
:10D500002B1720932A1780819FBF0E9478680E9462
:10D51000F0616093F50B7093F60B8093F70B90938B
:10D52000F80BC6CF0895EF92FF920F931F93CF93FE
:10D53000DF937C018B01609174177091751780ECFB
:10D5400090E00E947476609174177091751780E472
:10D5500090E00E947476E7010E0D1F1D6091741714
:10D5600070917517C017D107F9F08991803C59F473
:10D570008BED90E00E94747660917417709175172E
:10D580008CED90E00EC08B3D59F48BED90E00E9445
:10D59000747660917417709175178DED90E001C0ED
:10D5A00090E00E947476DACF80EC90E0DF91CF912A
:10D5B0001F910F91FF90EF900C947476EF92FF9271
:10D5C0000F931F93CF93DF937C018B0160917417AE
:10D5D0007091751780EC90E00E94747660917417DA
:10D5E0007091751780EF90E00E947476E7010E0D40
:10D5F0001F1D6091741770917517C017D107F9F04E
:10D600008991803C59F48BED90E00E947476609192
:10D610007417709175178CED90E00EC08B3D59F426
:10D620008BED90E00E94747660917417709175177D
:10D630008DED90E001C090E00E947476DACF80EC2E
:10D6400090E0DF91CF911F910F91FF90EF900C949C
:10D650007476CF92DF92EF92FF920F931F93CF9346
:10D66000DF93CDB7DEB728970FB6F894DEBF0FBEB5
:10D67000CDBF8B01FC01608171818281938120E8A3
:10D6800031E541E050E00E94857369017A012CE3A5
:10D6900030E040E050E00E947A7929833A834B835E
:10D6A0005C8389819A81AB81BC81F80160836CE3E2
:10D6B00070E00E946679DC01CB01F801A1838283CE
:10D6C000C601069667E070E00E94717384832DEABC
:10D6D0003EE840E050E0C701B6010E947A79298314
:10D6E0003A836D837E838F83988789819A8124E62C
:10D6F000289F6001299FD00C11246D817E818F812C
:10D70000988525EB35E040E050E00E947A79298346
:10D710003A836D837E83E980FA80EE0CFF1CEE0C69
:10D72000FF1CEC0CFD1C8D819E81F5E6EF16F104CB
:10D7300010F0019604C024E6E216F10419F021E08D
:10D7400030E002C020E030E0A90144595E4F4817A4
:10D75000590768F46DE671E0821B930B0E946679AD
:10D76000DC01CB01E80EF91ECD0120E030E044E6FB
:10D77000E40EF11CF801F782E68291878087255C30
:10D780003F4F8217930748F46FE170E00E9466797B
:10D79000DC01CB01F801858322C069E970E0821BBE
:10D7A000930B0E946679DC01CB01F82EFF0CFF0C75
:10D7B000F80E6DE370E0CD010E946679DC01CB01CB
:10D7C000E82EEE0C6FE170E0CD010E946679DC017D
:10D7D000CB0122E0280FF20EFE0CF801F582A383A4
:10D7E000F8011386128683818F5F838328960FB694
:10D7F000F894DEBF0FBECDBFDF91CF911F910F9187
:10D80000FF90EF90DF90CF900895CF92DF92EF924C
:10D81000FF920F931F93CF93DF9300D000D0CDB72B
:10D82000DEB78C010E94BE6C69837A838B839C83F4
:10D83000F8018285938597FF0EC0E091D23AF0916E
:10D84000D33A309741F06EEC7AE3CE010196099518
:10D85000F80193878287F801828593851816190647
:10D8600094F4AA2797FDA095BA2F49815A816B811C
:10D870007C816A017B01C81AD90AEA0AFB0AC982BB
:10D88000DA82EB82FC8289819A81AB81BC814091F2
:10D89000CE3A5091CF3A6091D03A7091D13A841BF0
:10D8A000950BA60BB70B89839A83AB83BC83B80116
:10D8B000CE0101960E946D6C69817A818B819C8179
:10D8C0000F900F900F900F90DF91CF911F910F91BC
:10D8D000FF90EF90DF90CF900895CF92DF92EF927C
:10D8E000FF920F931F93CF93DF9300D000D0CDB75B
:10D8F000DEB76C017B01E091D23AF091D33A3097D8
:10D9000029F06EEC7AE309958C0102C00FEF1FEF4E
:10D91000F60140815181628173818091CE3A90916C
:10D92000CF3AA091D03AB091D13A480F591F6A1F0F
:10D930007B1F101611064CF4C801AA2797FDA0956D
:10D94000BA2F480F591F6A1F7B1F49835A836B8365
:10D950007C83B701CE0101960E94296BF7011387E2
:10D9600002870F900F900F900F90DF91CF911F9132
:10D970000F91FF90EF90DF90CF9008958F929F923C
:10D98000AF92BF92CF92DF92EF92FF920F931F93CD
:10D99000CF93DF93EC01EE81FF818F0104561109D3
:10D9A000B9F0CF01855691096C0197FF03C023E0C0
:10D9B000C20ED11CD594C794D594C7946CE97FEF5F
:10D9C0000E946679C60ED71E8FEFC81AD80A02C009
:10D9D000C12CD12CEE24D7FCE094FE2C2DE631E0B6
:10D9E000D8010E944779C60ED71EE81EF91E8B810A
:10D9F000992787FD90958C01015011092D812230C6
:10DA00002CF4222379F1015E1F4F2CC0CF018459E1
:10DA1000984F0E947A6DE82FF0E0FB96E00FF11F1F
:10DA20008D81992787FD909502978530910514F097
:10DA3000E756FF4F65E070E00E9466799C0197FF12
:10DA400002C02F5F3F4F359527959DE3929FA00120
:10DA5000939F500D11248F01040F151F80FF02C0EA
:10DA6000015E1F4FA801662757FD6095762F9A012A
:10DA7000AB012C0D3D1D4E1D5F1D60E871E581E081
:10DA800090E00E9456796B017C01AA81BB27A7FD1B
:10DA9000B09520E13EE00E9447794B015C01A981ED
:10DAA000BB27A7FDB0952CE330E00E944779DC014D
:10DAB000CB01880D991DAA1DBB1D4881552747FD27
:10DAC0005095652F752F840F951FA61FB71FBC019A
:10DAD000CD016C0D7D1D8E1D9F1DDF91CF911F917E
:10DAE0000F91FF90EF90DF90CF90BF90AF909F90FD
:10DAF0008F9008959C0123703327232B59F464E6FB
:10DB000070E00E946679892B39F46370772781E091
:10DB1000672B19F080E0089581E008950E942004A9
:10DB20008BE298E10E94DB600E94586A0E94BB670A
:10DB30000E9435120E943154F3CF2F923F924F92A0
:10DB40005F926F927F928F929F92AF92BF92CF928D
:10DB5000DF92EF92FF920F931F93CF93DF93CDB796
:10DB6000DEB763970FB6F894DEBF0FBECDBF6C0172
:10DB70004B012A01FC0117821682838181FF43C376
:10DB8000AE014F5F5F4F3A01F6019381F40193FDBF
:10DB9000859193FF81914F01882309F430C3853229
:10DBA00039F493FD859193FF81914F01853239F4CA
:10DBB000B60190E00E94747652012501E5CF10E095
:10DBC000F12C20E02032A0F48B3269F030F4803266
:10DBD00059F0833269F420612CC08D3239F08033E2
:10DBE00039F4216026C02260246023C0286021C04F
:10DBF00027FD27C030ED380F3A3078F426FF06C0F5
:10DC0000FAE01F9F300D1124132F13C04AE0F49E39
:10DC1000300D1124F32E20620CC08E3221F426FD2B
:10DC2000EEC2206406C08C3611F4206802C088362B
:10DC300041F4F40193FD859193FF81914F0181118E
:10DC4000C1CF9BEB980F933018F42061805E06C023
:10DC50009BE9980F933008F071C12F7E26FF16E0E4
:10DC60002F73322E853619F42064322E08C0863682
:10DC700021F4F22FF0683F2E02C01111115037FE2F
:10DC800007C01C3350F4EE24E394E10E27E00BC0F0
:10DC9000183038F027E017E005C027E04CE3E42E09
:10DCA00002C0212FE12C520144E0A40EB11CF2016C
:10DCB00060817181828193810E2DA3010E94F57490
:10DCC0002C01098100FF02C003FF07C031FC08C01E
:10DCD00032FE09C030E2232E07C02DE2222E04C0FE
:10DCE0009BE2292E01C0212C802F8C7019F021106D
:10DCF00068C2A8C237FE0FC0E40C04FF04C08A81CA
:10DD0000813309F4EA941E1474F5F8E0FE1578F5F1
:10DD100088E0E82E2CC036FC2AC0812F90E08415C4
:10DD200095059CF02CEF42162FEF520674F0432D10
:10DD30004068342E0AC0E2E0F0E0EC0FFD1FE10F76
:10DD4000F11D8081803319F411501111F4CF37FE89
:10DD50000EC0EE24E394E10E812F90E048165906A0
:10DD60002CF4141904C0EE24E39401C010E037FE33
:10DD700006C01414150434F4C201019605C085E0F0
:10DD800090E002C081E090E021100196112331F073
:10DD9000212F30E02F5F3F4F820F931F2F2D30E058
:10DDA0008217930714F4F81A01C0F12C832D89709F
:10DDB00049F4FF2039F0B60180E290E00E947476C9
:10DDC000FA94F7CF222029F0B601822D90E00E942C
:10DDD000747633FC09C0FF2039F0B60180E390E08F
:10DDE0000E947476FA94F7CF37FE5AC0942D852D91
:10DDF00057FE02C090E080E0292E382E20E030E06F
:10DE0000A2014E1951095D874C87A201421953099D
:10DE10005F874E87612F70E044275527461B570BBD
:10DE2000598B488B5FEF2516350649F4B6018EE213
:10DE300090E02A8B3B8B0E9474763B892A8942149E
:10DE400053046CF04C855D854215530544F4EE8512
:10DE5000FF85E20FF31FE60DF71D818101C080E30E
:10DE600051E0251A31082F5F3F4F48895989241600
:10DE700035064CF0B60190E02A8B3B8B0E947476FD
:10DE80002A893B89CFCF2414350439F49A819633FB
:10DE900018F4953311F404FF81E3B60190E04BC010
:10DEA0008A81813309F00F7EB60190E00E9474767A
:10DEB000111105C034FC18C085E690E017C0B6010A
:10DEC0008EE290E00E94747682E0EE24E394E80E05
:10DED000F301E80FF11D8081B60190E00E94747695
:10DEE00011508E2D91F7E6CF85E490E0B6010E94A7
:10DEF000747657FC05C04114510439F404FF05C081
:10DF00005194419451088DE201C08BE2B60190E03A
:10DF10000E94747680E39AE0491651042CF08F5FDA
:10DF20005AE0451A5108F7CFB60190E00E94747686
:10DF3000B601C201C0960E94747657C1833631F093
:10DF4000833779F0833509F058C021C05201E2E0EF
:10DF5000AE0EB11CF2018081898301E010E0230143
:10DF600014C05201F2E0AF0EB11CF20140805180AA
:10DF700026FF03C0612F70E002C06FEF7FEFC20188
:10DF80002A8B0E94EC758C012A892F7715C05201CB
:10DF9000F2E0AF0EB11CF2014080518026FF03C0B9
:10DFA000612F70E002C06FEF7FEFC2012A8B0E94E9
:10DFB000CD758C012A892068322E23FD1AC08F2D41
:10DFC00090E008171907A8F4B60180E290E00E94DB
:10DFD0007476FA94F4CFF20137FC859137FE819183
:10DFE0002F01B60190E00E947476F110FA9401506E
:10DFF00011090115110579F7F8C0843611F0893639
:10E0000059F5520127FF09C0F4E0AF0EB11CF2012F
:10E0100060817181828193810AC0F2E0AF0EB11CF0
:10E02000F20160817181882777FD8095982F2F7686
:10E03000322E97FF09C090958095709561957F4F1E
:10E040008F4F9F4F2068322E2AE030E0A3010E94BC
:10E050002D77E82EE6183FC0022F853721F40F7E7A
:10E060002AE030E01DC0097F8F3691F018F4883522
:10E0700059F0C5C0803719F0883711F0C0C0006171
:10E0800004FF09C0046007C024FF08C0066006C082
:10E0900028E030E005C020E130E002C020E132E0BD
:10E0A000520107FF09C0F4E0AF0EB11CF20160811C
:10E0B00071818281938108C0F2E0AF0EB11CF20140
:10E0C0006081718180E090E0A3010E942D77E82EAD
:10E0D000E6180F77302E36FE0BC0332D3E7FE1164B
:10E0E00050F434FE0AC032FC08C0332D3E7E05C019
:10E0F0000E2D332D03C00E2D01C0012F34FF0CC097
:10E10000FE01EE0DF11D8081803311F4397E08C0CF
:10E1100032FF05C00E5F04C0832F867809F00F5FC1
:10E1200033FD13C030FF06C01E2D0F1518F41F0D50
:10E13000101B0F2D0F1568F4B60180E290E03B8BA9
:10E140000E9474760F5F3B89F5CF0F1510F4F01A1B
:10E1500001C0F12C34FF12C0B60180E390E03B8B8C
:10E160000E9474763B8932FF17C031FD03C088E7F7
:10E1700090E002C088E590E0B6010CC0832F86785D
:10E1800059F031FF02C08BE201C080E237FD8DE221
:10E19000B60190E00E947476E11638F4B60180E38F
:10E1A00090E00E9474761150F7CFEA94F301EE0DDF
:10E1B000F11D8081B60190E00E947476E110F5CFE8
:10E1C00014C0F4E0FF1558F584E0F81A33FE1EC0C1
:10E1D000211026C003FF2AC00CEB10E0F32DF071D4
:10E1E0003F2EF8018491811124C0FF2009F4E5CC71
:10E1F000B60180E290E00E947476FA94F6CFF601C0
:10E200008681978126C08FEF9FEF23C0B60180E201
:10E2100090E00E947476FA94F110F8CFD9CFF12CE7
:10E22000B601822D90E00E947476D4CF00EC10E00D
:10E23000D5CF31108052B60190E00E9474760F5F06
:10E240001F4FCFCF23E02F1510F483E0BECFF12C6A
:10E25000C1CF63960FB6F894DEBF0FBECDBFDF917E
:10E26000CF911F910F91FF90EF90DF90CF90BF90D3
:10E27000AF909F908F907F906F905F904F903F9066
:10E280002F9008955058BB27AA270E945A710C94CA
:10E29000A4720E94967238F00E949D7220F039F4A8
:10E2A0009F3F19F426F40C9493720EF4E095E7FB6B
:10E2B0000C948D72E92F0E94B57258F3BA17620759
:10E2C00073078407950720F079F4A6F50C94D772AC
:10E2D0000EF4E0950B2EBA2FA02D0B01B901900181
:10E2E0000C01CA01A0011124FF27591B99F0593FC5
:10E2F00050F4503E68F11A16F040A22F232F342F0D
:10E300004427585FF3CF469537952795A795F0405A
:10E310005395C9F77EF41F16BA0B620B730B840B6F
:10E32000BAF09150A1F0FF0FBB1F661F771F881F27
:10E33000C2F70EC0BA0F621F731F841F48F487957F
:10E3400077956795B795F7959E3F08F0B0CF939571
:10E35000880F08F09927EE0F9795879508950E94EA
:10E36000C3710C94A4720E949D7258F00E94967220
:10E3700040F029F45F3F29F00C948D7251110C94F8
:10E38000D8720C9493720E94B57268F39923B1F31A
:10E39000552391F3951B550BBB27AA2762177307CB
:10E3A000840738F09F5F5F4F220F331F441FAA1F5F
:10E3B000A9F335D00E2E3AF0E0E832D0915050401B
:10E3C000E695001CCAF72BD0FE2F29D0660F771FC9
:10E3D000881FBB1F261737074807AB07B0E809F0AF
:10E3E000BB0B802DBF01FF2793585F4F3AF09E3F34
:10E3F000510578F00C948D720C94D8725F3FE4F361
:10E40000983ED4F3869577956795B795F7959F5F76
:10E41000C9F7880F911D9695879597F90895E1E0C2
:10E42000660F771F881FBB1F621773078407BA0721
:10E4300020F0621B730B840BBA0BEE1F88F7E0957C
:10E4400008950E94BD7288F09F5798F0B92F9927C0
:10E45000B751B0F0E1F0660F771F881F991F1AF0CF
:10E46000BA95C9F714C0B13091F00E94D772B1E0EB
:10E4700008950C94D772672F782F8827B85F39F0EA
:10E48000B93FCCF3869577956795B395D9F73EF468
:10E4900090958095709561957F4F8F4F9F4F089510
:10E4A000E89409C097FB3EF490958095709561952E
:10E4B0007F4F8F4F9F4F9923A9F0F92F96E9BB27E4
:10E4C0009395F695879577956795B795F111F8CF60
:10E4D000FAF4BB0F11F460FF1BC06F5F7F4F8F4FCB
:10E4E0009F4F16C0882311F096E911C0772321F0C1
:10E4F0009EE8872F762F05C0662371F096E8862F59
:10E5000070E060E02AF09A95660F771F881FDAF7AF
:10E51000880F9695879597F9089597F99F6780E8F2
:10E5200070E060E008959FEF80EC089500240A9465
:10E530001616170618060906089500240A941216DE
:10E540001306140605060895092E0394000C11F411
:10E55000882352F0BB0F40F4BF2B11F460FF04C0BE
:10E560006F5F7F4F8F4F9F4F089557FD9058440F17
:10E57000551F59F05F3F71F04795880F97FB991F22
:10E5800061F09F3F79F087950895121613061406DF
:10E59000551FF2CF4695F1DF08C01616170618066C
:10E5A000991FF1CF86957105610508940895E89447
:10E5B000BB2766277727CB0197F908950E94F17250
:10E5C0000C94A4720E94967238F00E949D7220F002
:10E5D000952311F00C948D720C94937211240C9469
:10E5E000D8720E94B57270F3959FC1F3950F50E0F9
:10E5F000551F629FF001729FBB27F00DB11D639FF5
:10E60000AA27F00DB11DAA1F649F6627B00DA11D9A
:10E61000661F829F2227B00DA11D621F739FB00D40
:10E62000A11D621F839FA00D611D221F749F3327B0
:10E63000A00D611D231F849F600D211D822F762F49
:10E640006A2F11249F5750409AF0F1F088234AF026
:10E65000EE0FFF1FBB1F661F771F881F9150504092
:10E66000A9F79E3F510580F00C948D720C94D872DE
:10E670005F3FE4F3983ED4F3869577956795B79519
:10E68000F795E7959F5FC1F7FE2B880F911D969533
:10E69000879597F90895A29FB001B39FC001A39FEA
:10E6A000700D811D1124911DB29F700D811D1124CB
:10E6B000911D08950E944B73A59F900DB49F900DDE
:10E6C000A49F800D911D11240895991B79E004C029
:10E6D000991F961708F0961B881F7A95C9F78095A1
:10E6E0000895AA1BBB1B51E107C0AA1FBB1FA61799
:10E6F000B70710F0A61BB70B881F991F5A95A9F7EB
:10E7000080959095BC01CD010895A1E21A2EAA1B17
:10E71000BB1BFD010DC0AA1FBB1FEE1FFF1FA217D1
:10E72000B307E407F50720F0A21BB30BE40BF50BCE
:10E73000661F771F881F991F1A9469F76095709557
:10E74000809590959B01AC01BD01CF01089568941F
:10E7500001C0E8948F929F92CF93DF930E94B5738C
:10E76000DF91CF919F908F90089588249924F40190
:10E77000E401B0E49F93AA279A158B049C04ED054D
:10E78000FE05CF05D007A10798F4AD2FDC2FCF2FC2
:10E79000FE2FE92D982C892E982F872F762F652F05
:10E7A000542F432F322F2227B85031F7BF9127C063
:10E7B0001B2EBF91BB27220F331F441F551F661FFF
:10E7C000771F881F991F881C991CEE1FFF1FCC1FE5
:10E7D000DD1FAA1FBB1F8A149B04EC05FD05CE0597
:10E7E000DF05A007B10748F08A189B08EC09FD096E
:10E7F000CE09DF09A00BB10B21601A94E1F62EF4CB
:10E800009401AF01BE01CD01000C0895EE0FFF1F72
:10E810000024001C0BBE0790F691E02D09940F9385
:10E82000083090F0982F872F762F652F542F432F85
:10E83000322F22270850F4CF220F331F441F551FB9
:10E84000661F771F881F991F0A95B2F70F910895C9
:10E8500097FB10F8169400080F93083098F00850B2
:10E86000232F342F452F562F672F782F892F902D48
:10E87000F4CF059497958795779567955795479524
:10E88000379527950A95AAF70F9108952A0D3B1DF4
:10E890004C1D5D1D6E1D7F1D801F911F089500245E
:10E8A000A7FD00942A0F301D401D501D601D701DD6
:10E8B000801D901D08952A193B094C095D096E09B8
:10E8C0007F09800B910B08952A153B054C055D05CA
:10E8D0006E057F058007910708950024A7FD009429
:10E8E0002A17300540055005600570058005900524
:10E8F00008958F929F92AF92BF92CF92DF92EF9244
:10E90000FF92CF93DF93EC01688179818A819B81AB
:10E91000611571058105910521F464E279ED8BE5BE
:10E9200097E02DE133EF41E050E00E947A79490110
:10E930005A019B01AC01A7EAB1E40E945A736B0132
:10E940007C01ACEEB4EFA50194010E945179DC0189
:10E95000CB018C0D9D1DAE1DBF1DB7FF03C00197E0
:10E96000A109B04888839983AA83BB83BC01CD01E8
:10E970009F77DF91CF91FF90EF90DF90CF90BF9086
:10E98000AF909F908F9008950C94797484E091E0FB
:10E990000C947974609304017093050180930601CF
:10E9A000909307010895662777270C948B77FC01D5
:10E9B00088279927E89421912032E9F3293010F033
:10E9C0002E30C8F32B3241F02D3239F4689404C054
:10E9D0000E941176820F911D219120532A30C0F39D
:10E9E0001EF4909581959F4F0895283008F027E0F8
:10E9F0003327DA01990F311D87FD9160009661057B
:10EA0000710539F432602E5F3D9330E32A95E1F7CA
:10EA100008959F3F30F080387105610509F03C5F33
:10EA20003C5F3D93913008F08068911DDF93CF9358
:10EA30001F930F93FF92EF92192F987F9695E92FCE
:10EA400096959695E90FFF27E25EFE4F99273327AB
:10EA5000EE24FF24A701E70105900894079428F409
:10EA6000360FE71EF81E491F511D660F771F881FBE
:10EA7000991F0694A1F70590079428F4E70EF81E55
:10EA8000491F561FC11D770F881F991F661F0694C7
:10EA9000A1F70590079428F4F80E491F561FC71FC9
:10EAA000D11D880F991F661F771F0694A1F7059047
:10EAB000079420F4490F561FC71FD81F990F661FD0
:10EAC000771F881F0694A9F784911095177041F05D
:10EAD000D695C79557954795F794E7941A95C1F73A
:10EAE000E4ECF0E06894159015913591659195915D
:10EAF00005907FE27395E118F10A430B560BC90BA1
:10EB0000D009C0F7E10CF11E431F561FC91FD01DCD
:10EB10007EF4703311F48A95E6CFE894015030F01A
:10EB2000080F0AF40027021708F4202F2395022F5C
:10EB30007A3328F079E37D932A95E9F710C07D9325
:10EB40002A9589F6069497956795379517951794A2
:10EB5000E118F10A430B560BC90BD00998F0239525
:10EB60007E9173957A3308F070E37C932013B8F7A5
:10EB70007E9170617D9330F0839571E37D9370E3B6
:10EB80002A95E1F71124EF90FF900F911F91CF91FB
:10EB9000DF91992787FD90950895FC0105906150BC
:10EBA00070400110D8F7809590958E0F9F1F0895A3
:10EBB000FB01DC0102C001900D9241505040D8F79A
:10EBC0000895FC018191861721F08823D9F79927B0
:10EBD00008953197CF010895FC0161507040019074
:10EBE0000110D8F7809590958E0F9F1F0895FB0117
:10EBF00051915523A9F0BF01DC014D9145174111F9
:10EC0000E1F759F4CD010190002049F04D914015F4
:10EC10004111C9F3FB014111EFCF81E090E0019771
:10EC200008957AE0979F902D879F802D910D112454
:10EC30000895CF93DF93EC012B8120FF33C026FF93
:10EC40000AC02F7B2B838E819F8101969F838E83A9
:10EC50008A8190E029C022FF0FC0E881F98180817C
:10EC6000992787FD9095009719F420622B831AC08D
:10EC70003196F983E8830EC0EA85FB85099597FFF5
:10EC800009C02B81019611F080E201C080E1822B46
:10EC90008B8308C02E813F812F5F3F4F3F832E83A0
:10ECA000992702C08FEF9FEFDF91CF9108950F93C7
:10ECB0001F93CF93DF93CDB7DEB70F811885F8018F
:10ECC000838188608383AE01455F5F4F69857A8564
:10ECD000C8010E949D6DF8012381277F2383DF9166
:10ECE000CF911F910F9108950F931F93CF93DF93AF
:10ECF000FB01238121FD03C08FEF9FEF28C022FF7E
:10ED000016C046815781248135814217530744F448
:10ED1000A081B1819D012F5F3F4F318320838C9370
:10ED2000268137812F5F3F4F3783268310C0EB0149
:10ED3000092F182F0084F185E02D0995892BE1F624
:10ED40008E819F8101969F838E83812F902FDF91EB
:10ED5000CF911F910F910895CF93DF93CDB7DEB779
:10ED6000AE014B5F5F4FFA0161917191AF018091EC
:10ED7000CA3A9091CB3A0E949D6DDF91CF91089550
:10ED80000F931F93CF93DF93E091CA3AF091CB3A60
:10ED9000238121FF1BC08C01D0E0C0E0F8018191EC
:10EDA0008F016091CA3A7091CB3ADB011896ED91D0
:10EDB000FC911997882331F00995892B79F3DFEFBE
:10EDC000CFEFECCF8AE00995892B19F08FEF9FEFF9
:10EDD00002C08D2F9C2FDF91CF911F910F9108952D
:10EDE0000F931F93CF93DF93CDB7DEB72E970FB658
:10EDF000F894DEBF0FBECDBF0D891E898F89988D17
:10EE000026E02C831A83098397FF02C080E090E8F4
:10EE100001979E838D83AE01455E5F4F698D7A8D2C
:10EE2000CE0101960E949D6D4D815E8157FD0AC005
:10EE30002F813885421753070CF49A01F801E20F2D
:10EE4000F31F10822E960FB6F894DEBF0FBECDBF13
:10EE5000DF91CF911F910F910895FA01AA272830D1
:10EE600051F1203181F1E8946F936E7F6E5F7F4F97
:10EE70008F4F9F4FAF4FB1E03ED0B4E03CD0670F13
:10EE8000781F891F9A1FA11D680F791F8A1F911D66
:10EE9000A11D6A0F711D811D911DA11D20D009F4B6
:10EEA00068943F912AE0269F11243019305D3193F8
:10EEB000DEF6CF010895462F4770405D4193B3E0E1
:10EEC0000FD0C9F7F6CF462F4F70405D4A3318F088
:10EED000495D31FD4052419302D0A9F7EACFB4E039
:10EEE000A6959795879577956795BA95C9F70097F1
:10EEF0006105710508959B01AC010A2E0694579592
:10EF0000479537952795BA95C9F7620F731F841FE8
:10EF1000951FA01D08956F927F928F929F92AF923E
:10EF2000BF92CF92DF92EF92FF920F931F93CF93F6
:10EF3000DF93EC017B016115710519F0DB018D9305
:10EF40009C938E010F5F1F4F7880872D90E00E9469
:10EF5000FA78892B11F0E801F4CFBDE27B1205C0ED
:10EF60000F5F1F4F7980C1E008C0EBE27E1204C042
:10EF70008E010E5F1F4F7980C0E06801F1E0CF1A6B
:10EF8000D10843E050E066EC71E0C6010E940379CD
:10EF9000892BF1F4680122E0C20ED11C45E050E05B
:10EFA00061EC71E0C6010E940379892B21F46801AC
:10EFB00087E0C80ED11CE114F10419F0D701CD92FD
:10EFC000DC92C111FFC060E070E080E89FE703C100
:10EFD00043E050E06EEB71E0C6010E940379892B9B
:10EFE00051F4E114F10409F4F2C00E5F1F4FF70170
:10EFF00011830083ECC0680160E070E0CB0100E0A9
:10F0000010E0F601D0EDD70DDA3058F52C2F226044
:10F01000622E2C2F2870C2FF05C0211128C00F5F5F
:10F020001F4F25C0222311F001501109A5E0B0E0C7
:10F030009B01AC010E945A734B015C01880C991C26
:10F04000AA1CBB1CC501B4016D0F711D811D911D52
:10F050006839A9E97A078A07A9E19A0740F0C660EA
:10F0600005C0DE3F51F4C3FD44C0C8606C2EBFEF45
:10F07000CB1ADB0A7080C62DC4CF2D2F2F7D2531F2
:10F08000C1F540814D3211F4C06106C04B3221F010
:10F09000319621E030E006C03296D60111964C91AF
:10F0A00022E030E0A0EDA40FAA3018F0E21BF30B31
:10F0B00020C040E050E04038BCE05B075CF49A01BF
:10F0C000220F331F220F331F420F531F440F551FB0
:10F0D0004A0F511D3196DF0111972C91A0EDA20F1F
:10F0E000AA3048F3C4FF03C0519541955109040F5C
:10F0F000151FC1FF07C0E114F10421F03197D701BA
:10F10000ED93FC930E945072C370C33019F06B01F1
:10F110007C0106C06B017C01F7FAF094F7F8F094DB
:10F1200020E030E0A901C701B6010E941B798823C5
:10F1300009F445C017FF06C0119501951109CDEDE1
:10F14000D1E002C0C5EFD1E05E01B8E1AB1AB10871
:10F150004601BE2DAF2D90E2E92EF12C0E151F05B4
:10F1600084F0FE012591359145915491B4018B2F86
:10F170009A2F0E94DE724B01B82FA92F0E191F097A
:10F18000EDCF2497F594E794CA15DB0539F76401B0
:10F19000EB2EFA2E8E2D880F8F2D881F8F3F49F072
:10F1A00020E030E0A901C701B6010E941B7981115E
:10F1B00006C082E290E09093D53A8093D43AC7019A
:10F1C000B60109C060E070E080E89FEF04C060E035
:10F1D00070E080EC9FE7DF91CF911F910F91FF903E
:10F1E000EF90DF90CF90BF90AF909F908F907F90E7
:10F1F0006F90089591110C944479803219F08950E0
:10F200008550C8F70895FB01DC014150504088F05B
:10F210008D9181341CF08B350CF4805E65916134E6
:10F220001CF06B350CF4605E861B611171F3990B59
:10F230000895881BFCCF0E94207908F481E008958E
:10F24000990F0008550FAA0BE0E8FEEF16161706F7
:10F25000E807F907C0F012161306E407F50798F05F
:10F26000621B730B840B950B39F40A2661F0232B78
:10F27000242B252B21F408950A2609F4A140A695F4
:10F280008FEF811D811D08959927882708950E9479
:10F290004B73B7FF0895821B930B0895B7FF0C942F
:10F2A0005A730E945A73821B930B0895DB018F934C
:10F2B0009F930E945A73BF91AF91A29F800D911DA1
:10F2C000A39F900DB29F900D1124089597FB072ED8
:10F2D00016F4009407D077FD09D00E94717307FCE3
:10F2E00005D03EF4909581959F4F08957095619556
:10F2F0007F4F0895052E97FB1EF400940E9491798C
:10F3000057FD07D00E94857307FC03D04EF40C9480
:10F31000917950954095309521953F4F4F4F5F4FD4
:10F32000089590958095709561957F4F8F4F9F4F71
:06F330000895F894FFCFE0
:10F33600FF0101FE01000000808183848687898A9F
:10F346008C8E8F9192949597989A9B9D9EA0A2A33E
:10F35600A5A6A7A9AAACADAFB0B2B3B5B6B7B9BAB0
:10F36600BCBDBEC0C1C2C4C5C6C8C9CACBCDCECF3E
:10F37600D0D2D3D4D5D6D7D9DADBDCDDDEDFE0E1F7
:10F38600E2E3E4E5E6E7E8E9EAEAEBECEDEEEEEFE8
:10F39600F0F1F1F2F3F3F4F5F5F6F6F7F8F8F9F91A
:10F3A600FAFAFAFBFBFCFCFCFDFDFDFDFEFEFEFE93
:10F3B600FEFFFFFFFFFFFFFF2B2E2C3B3D5B5D2F6C
:10F3C6005C222A3A3C3E3F7C7F00809A90418E41E7
:10F3D6008F804545454949498E8F9092924F994F66
:10F3E600555559999A9B9C9D9E9F41494F55A5A558
:10F3F600A6A7A8A9AAABACADAEAFB0B1B2B3B4B52F
:10F40600B6B7B8B9BABBBCBDBEBFC0C1C2C3C4C51E
:10F41600C6C7C8C9CACBCCCDCECFD0D1D2D3D4D50E
:10F42600D6D7D8D9DADBDCDDDEDFE0E1E2E3E4E5FE
:10F43600E6E7E8E9EAEBECEDEEEFF0F1F2F3F4F5EE
:10F44600F6F7F8F9FAFBFCFDFEFF01030507090EC6
:10F4560010121416181C1E7D1D0100632C001E962A
:10F4660001A01E5A01001F0806101F0606201F08CD
:10F4760006301F0806401F0606511F0700591F5277
:10F486001F5B1F541F5D1F561F5F1F601F080670FE
:10F496001F0E00BA1FBB1FC81FC91FCA1FCB1FDA0A
:10F4A6001FDB1FF81FF91FEA1FEB1FFA1FFB1F8048
:10F4B6001F0806901F0806A01F0806B01F0400B804
:10F4C6001FB91FB21FBC1FCC1F0100C31FD01F02D4
:10F4D60006E01F0206E51F0100EC1FF31F0100FCFA
:10F4E6001F4E210100322170211002842101008368
:10F4F60021D0241A05302C2F04602C0201672C061B
:10F5060001752C0201802C6401002D260841FF1A8A
:10F5160003000061001A03E0001703F8000703FF69
:10F5260000010078010001300132010601390110A5
:10F53600014A012E017901060180014D0043028135
:10F546000182018201840184018601870187018984
:10F55600018A018B018B018D018E018F0190019132
:10F5660001910193019401F6019601970198019882
:10F57600013D029B019C019D0120029F01A001A06B
:10F5860001A201A201A401A401A601A701A701A944
:10F5960001AA01AB01AC01AC01AE01AF01AF01B1F3
:10F5A60001B201B301B301B501B501B701B801B8A4
:10F5B60001BA01BB01BC01BC01BE01F701C001C11A
:10F5C60001C201C301C401C501C401C701C801C705
:10F5D60001CA01CB01CA01CD011001DD0101008E76
:10F5E60001DE011201F3010300F101F401F401F857
:10F5F600012801220212013A020900652C3B023B56
:10F60600023D02662C3F0240024102410246020AC6
:10F61600015302400081018601550289018A015881
:10F62600028F015A0290015C025D025E025F029344
:10F636000161026202940164026502660267029732
:10F646000196016A02622C6C026D026E029C0170C8
:10F656000271029D01730274029F0176027702789D
:10F666000279027A027B027C02642C7E027F02A669
:10F676000181028202A9018402850286028702AE06
:10F68600014402B101B20145028D028E028F029041
:10F69600029102B7017B030300FD03FE03FF03ACE7
:10F6A6000304008603880389038A03B1031103C296
:10F6B600030200A303A303C4030803CC0303008CC3
:10F6C600038E038F03D8031801F2030A00F903F32C
:10F6D60003F403F503F603F703F703F903FA03FA52
:10F6E600033004200350041007600422018A043604
:10F6F60001C1040E01CF040100C004D0044401611D
:10F706000526040000C700FC00E900E200E400E072
:10F7160000E500E700EA00EB00E800EF00EE00EC91
:10F7260000C400C500C500E600C600F400F600F2FD
:10F7360000FB00F900FF00D600DC00F800A300D8AB
:10F7460000A7209201E100ED00F300FA00F100D1DC
:10F7560000AA00BA00BF001023AC00BD00BC00A187
:10F7660000AB00A40091259225932502252425614E
:10F77600256225562555256325512557255D255C8A
:10F786002558251025142534252C251C2500253C17
:10F79600255E255F255A2554256925662560255051
:10F7A600256C256725682564256525592558255224
:10F7B6002553256B256A2518250C25882584258C37
:10F7C6002590258025B103DF009303C003A303C35F
:10F7D60003B500C403A6039803A903B4031E22C6F7
:10F7E60003B50329226122B1006522642220232168
:10F7F60023F7004822B0001922B7001A227F20B250
:10F8060000A025A00001020408102040801B363508
:10F816005C625C895CA45C53797374656D20737457
:10F8260061727420686173206265656E2068616C20
:10F836007465640D00EB76904558464154202020AF
:10F846000046415400464154333200222A3A3C3E97
:10F856003F7C7F002B2C3B3D5B5D0041542B46419A
:10F8660043544F525952455345540D0041542B476A
:10F8760041504445564E414D453D4F70656E4D6F66
:10F8860064656D0D0041542B4D4F44455357495403
:10F896004348454E3D626C652C300D0041542B4D5E
:10F8A6004F4445535749544348454E3D6C6F636139
:10F8B6006C2C300D0041542B48574D4F44454C4558
:10F8C600443D300D0041542B424C45504F57455254
:10F8D6004C4556454C3D340D0041545A0D00257398
:10F8E6000A0D0024475047474100244750524D43D4
:10F8F600004F70656E4D6F64656D2F656E74726F27
:10F9060070792E696E646578004F70656E4D6F6410
:10F91600656D2F656E74726F70792E736F75726375
:10F9260065004F70656E4D6F64656D2F616573314F
:10F9360032382E64697361626C65004F70656E4D76
:10F946006F64656D2F6165733132382E6B65790092
:10F956004F70656E4D6F64656D2F4C6F672F7061CC
:10F96600636B65742E696E646578004F70656E4DC5
:10F976006F64656D004F70656E4D6F64656D2F4CDD
:10F986006F670025732F256C752E706361700000FC
:00000001FF
